 config_alm_overview

 Timestamp is 614c8101 (Thu Sep 23 13:28:33 2021)

 Preferred load address is 10000000

 Start         Length     Name                   Class
 0001:00000000 00000063H .text$di                CODE
 0001:00000070 0000547cH .text$mn                CODE
 0001:000054ec 00000d2aH .text$x                 CODE
 0001:00006216 00000021H .text$yd                CODE
 0002:00000000 00000a54H .idata$5                DATA
 0002:00000a54 00000004H .CRT$XCA                DATA
 0002:00000a58 0000000cH .CRT$XCU                DATA
 0002:00000a64 00000004H .CRT$XCZ                DATA
 0002:00000a68 00000004H .CRT$XIA                DATA
 0002:00000a6c 00000004H .CRT$XIAA               DATA
 0002:00000a70 00000004H .CRT$XIC                DATA
 0002:00000a74 00000004H .CRT$XIZ                DATA
 0002:00000a80 00002d18H .rdata                  DATA
 0002:00003798 00000fc4H .rdata$r                DATA
 0002:00004760 00000070H .rdata$sxdata           DATA
 0002:000047d0 00000004H .rtc$IAA                DATA
 0002:000047d4 00000004H .rtc$IZZ                DATA
 0002:000047d8 00000004H .rtc$TAA                DATA
 0002:000047dc 00000004H .rtc$TZZ                DATA
 0002:000047e0 00000be4H .xdata$x                DATA
 0002:000053d0 00000067H .edata                  DATA
 0002:00005438 00000064H .idata$2                DATA
 0002:0000549c 00000014H .idata$3                DATA
 0002:000054b0 00000a54H .idata$4                DATA
 0002:00005f04 00006aa4H .idata$6                DATA
 0003:00000000 000001d4H .data                   DATA
 0003:000001d4 00000554H .data$r                 DATA
 0003:00000728 0000039cH .bss                    DATA
 0004:00000000 000000a0H .rsrc$01                DATA
 0004:000000a0 00000638H .rsrc$02                DATA

  Address         Publics by Value              Rva+Base       Lib:Object

 0000:00000000       ___guard_fids_table        00000000     <absolute>
 0000:00000000       ___guard_flags             00000000     <absolute>
 0000:00000000       ___guard_fids_count        00000000     <absolute>
 0000:0000001c       ___safe_se_handler_count   0000001c     <absolute>
 0000:00000000       ___ImageBase               10000000     <linker-defined>
 0001:00000070       ??0?$QGuardedPtr@VQPopupMenu@@@@QAE@XZ 10001070 f i cfg_alarm_overview.obj
 0001:00000070       ??0?$QGuardedPtr@VQDockWindow@@@@QAE@XZ 10001070 f i cfg_alarm_overview.obj
 0001:000000b1       ??0cfg_alarm_overview@@QAE@ABVQString@@00@Z 100010b1 f   cfg_alarm_overview.obj
 0001:0000061e       ??0config_plugin_base@@QAE@ABVQString@@00@Z 1000161e f i cfg_alarm_overview.obj
 0001:000006ab       ??1?$QDict@VQAction@@@@UAE@XZ 100016ab f i cfg_alarm_overview.obj
 0001:000006de       ??1?$QGuardedPtr@VQPopupMenu@@@@QAE@XZ 100016de f i cfg_alarm_overview.obj
 0001:000006de       ??1?$QGuardedPtr@VQDockWindow@@@@QAE@XZ 100016de f i cfg_alarm_overview.obj
 0001:000006e3       ??1?$QPtrList@VCInputFile@@@@UAE@XZ 100016e3 f i cfg_alarm_overview.obj
 0001:00000716       ??1?$QPtrList@VCOutputFile@@@@UAE@XZ 10001716 f i cfg_alarm_overview.obj
 0001:00000749       ??1?$QPtrList@VQPopupMenu@@@@UAE@XZ 10001749 f i cfg_alarm_overview.obj
 0001:0000077c       ??1QDockWindowList@@UAE@XZ 1000177c f i cfg_alarm_overview.obj
 0001:000007c5       ??1QPopupMenuList@@UAE@XZ  100017c5 f i cfg_alarm_overview.obj
 0001:000007f7       ??1cfg_alarm_overview@@UAE@XZ 100017f7 f   cfg_alarm_overview.obj
 0001:000008f4       ??1config_plugin_base@@UAE@XZ 100018f4 f i cfg_alarm_overview.obj
 0001:0000094e       ??4?$QGuardedPtr@VQDockWindow@@@@QAEAAV0@PAVQDockWindow@@@Z 1000194e f i cfg_alarm_overview.obj
 0001:0000094e       ??4?$QGuardedPtr@VQPopupMenu@@@@QAEAAV0@PAVQPopupMenu@@@Z 1000194e f i cfg_alarm_overview.obj
 0001:000009ac       ??_EQPopupMenu@@WCI@AEPAXI@Z 100019ac f i cfg_alarm_overview.obj
 0001:000009b4       ??_EQPopupMenu@@WIM@AEPAXI@Z 100019b4 f i cfg_alarm_overview.obj
 0001:000009bf       ??_EQToolBar@@WCI@AEPAXI@Z 100019bf f i cfg_alarm_overview.obj
 0001:000009c7       ??_Ecfg_alarm_overview@@WCI@AEPAXI@Z 100019c7 f i cfg_alarm_overview.obj
 0001:000009cf       ??_Econfig_plugin_base@@WCI@AEPAXI@Z 100019cf f i cfg_alarm_overview.obj
 0001:000009d7       ??_G?$QDict@VQAction@@@@UAEPAXI@Z 100019d7 f i cfg_alarm_overview.obj
 0001:000009d7       ??_E?$QDict@VQAction@@@@UAEPAXI@Z 100019d7 f i cfg_alarm_overview.obj
 0001:000009f6       ??_G?$QPtrList@VCInputFile@@@@UAEPAXI@Z 100019f6 f i cfg_alarm_overview.obj
 0001:000009f6       ??_E?$QPtrList@VCInputFile@@@@UAEPAXI@Z 100019f6 f i cfg_alarm_overview.obj
 0001:00000a15       ??_G?$QPtrList@VCOutputFile@@@@UAEPAXI@Z 10001a15 f i cfg_alarm_overview.obj
 0001:00000a15       ??_E?$QPtrList@VCOutputFile@@@@UAEPAXI@Z 10001a15 f i cfg_alarm_overview.obj
 0001:00000a34       ??_G?$QPtrList@VQPopupMenu@@@@UAEPAXI@Z 10001a34 f i cfg_alarm_overview.obj
 0001:00000a34       ??_E?$QPtrList@VQPopupMenu@@@@UAEPAXI@Z 10001a34 f i cfg_alarm_overview.obj
 0001:00000a53       ??_EQAction@@UAEPAXI@Z     10001a53 f i cfg_alarm_overview.obj
 0001:00000a53       ??_GQAction@@UAEPAXI@Z     10001a53 f i cfg_alarm_overview.obj
 0001:00000a73       ??_EQDockWindowList@@UAEPAXI@Z 10001a73 f i cfg_alarm_overview.obj
 0001:00000a73       ??_GQDockWindowList@@UAEPAXI@Z 10001a73 f i cfg_alarm_overview.obj
 0001:00000a92       ??_EQGuardedPtrPrivate@@UAEPAXI@Z 10001a92 f i cfg_alarm_overview.obj
 0001:00000a92       ??_GQGuardedPtrPrivate@@UAEPAXI@Z 10001a92 f i cfg_alarm_overview.obj
 0001:00000ab2       ??_GQListViewItem@@UAEPAXI@Z 10001ab2 f i cfg_alarm_overview.obj
 0001:00000ab2       ??_EQListViewItem@@UAEPAXI@Z 10001ab2 f i cfg_alarm_overview.obj
 0001:00000ad2       ??_GQPopupMenu@@UAEPAXI@Z  10001ad2 f i cfg_alarm_overview.obj
 0001:00000ad2       ??_EQPopupMenu@@UAEPAXI@Z  10001ad2 f i cfg_alarm_overview.obj
 0001:00000af2       ??_EQPopupMenuList@@UAEPAXI@Z 10001af2 f i cfg_alarm_overview.obj
 0001:00000af2       ??_GQPopupMenuList@@UAEPAXI@Z 10001af2 f i cfg_alarm_overview.obj
 0001:00000b11       ??_GQToolBar@@UAEPAXI@Z    10001b11 f i cfg_alarm_overview.obj
 0001:00000b11       ??_EQToolBar@@UAEPAXI@Z    10001b11 f i cfg_alarm_overview.obj
 0001:00000b31       ??_Ecfg_alarm_overview@@UAEPAXI@Z 10001b31 f i cfg_alarm_overview.obj
 0001:00000b31       ??_Gcfg_alarm_overview@@UAEPAXI@Z 10001b31 f i cfg_alarm_overview.obj
 0001:00000b50       ??_Econfig_plugin_base@@UAEPAXI@Z 10001b50 f i cfg_alarm_overview.obj
 0001:00000b50       ??_Gconfig_plugin_base@@UAEPAXI@Z 10001b50 f i cfg_alarm_overview.obj
 0001:00000b6f       ?NavigateBNCSAcq@cfg_alarm_overview@@QAEXXZ 10001b6f f   cfg_alarm_overview.obj
 0001:00000bb1       ?NavigateBNCSOut@cfg_alarm_overview@@QAEXXZ 10001bb1 f   cfg_alarm_overview.obj
 0001:00000bf3       ?NavigateDatabaseOut@cfg_alarm_overview@@QAEXXZ 10001bf3 f   cfg_alarm_overview.obj
 0001:00000c35       ?NavigateProcs@cfg_alarm_overview@@QAEXXZ 10001c35 f   cfg_alarm_overview.obj
 0001:00000c35       ?NavigatetoProcs@cfg_alarm_overview@@QAEXXZ 10001c35 f   cfg_alarm_overview.obj
 0001:00000c77       ?NavigatetoInput@cfg_alarm_overview@@QAEXXZ 10001c77 f   cfg_alarm_overview.obj
 0001:00000dfa       ?NavigatetoOutput@cfg_alarm_overview@@QAEXXZ 10001dfa f   cfg_alarm_overview.obj
 0001:00000f7d       ?about@config_plugin_base@@UAE?AVQString@@XZ 10001f7d f i cfg_alarm_overview.obj
 0001:00000fd3       ?activate@cfg_alarm_overview@@UAEX_N@Z 10001fd3 f   cfg_alarm_overview.obj
 0001:00001082       ?activate@config_plugin_base@@UAEX_N@Z 10002082 f i cfg_alarm_overview.obj
 0001:00001082       ?reply@config_plugin_base@@UAEXPAVresponse@@@Z 10002082 f i cfg_alarm_overview.obj
 0001:00001085       ?apply@cfg_alarm_overview@@UAEXXZ 10002085 f   cfg_alarm_overview.obj
 0001:00001129       ?apply@config_plugin_base@@UAEXXZ 10002129 f i cfg_alarm_overview.obj
 0001:00001129       ?dummy@cfg_alarm_overview@@QAEXXZ 10002129 f i cfg_alarm_overview.obj
 0001:0000112a       ?clear@?$QDict@VQAction@@@@UAEXXZ 1000212a f i cfg_alarm_overview.obj
 0001:00001130       ?clear@?$QPtrList@VCInputFile@@@@UAEXXZ 10002130 f i cfg_alarm_overview.obj
 0001:00001130       ?clear@?$QPtrList@VQPopupMenu@@@@UAEXXZ 10002130 f i cfg_alarm_overview.obj
 0001:00001130       ?clear@?$QPtrList@VCOutputFile@@@@UAEXXZ 10002130 f i cfg_alarm_overview.obj
 0001:00001136       ?closeEvent@cfg_alarm_overview@@UAEXPAVQCloseEvent@@@Z 10002136 f   cfg_alarm_overview.obj
 0001:000011bb       ?closeEvent@config_plugin_base@@UAEXPAVQCloseEvent@@@Z 100021bb f i cfg_alarm_overview.obj
 0001:000011c9       ?count@?$QDict@VQAction@@@@UBEIXZ 100021c9 f i cfg_alarm_overview.obj
 0001:000011cd       ?count@?$QPtrList@VCOutputFile@@@@UBEIXZ 100021cd f i cfg_alarm_overview.obj
 0001:000011cd       ?count@?$QPtrList@VCInputFile@@@@UBEIXZ 100021cd f i cfg_alarm_overview.obj
 0001:000011cd       ?count@?$QPtrList@VQPopupMenu@@@@UBEIXZ 100021cd f i cfg_alarm_overview.obj
 0001:000011d1       ?createNewDirectory@cfg_alarm_overview@@QAE_NVQString@@@Z 100021d1 f   cfg_alarm_overview.obj
 0001:000016ab       ?createNewSystem@cfg_alarm_overview@@QAEXXZ 100026ab f   cfg_alarm_overview.obj
 0001:0000185a       ?deleteItem@?$QDict@VQAction@@@@EAEXPAX@Z 1000285a f i cfg_alarm_overview.obj
 0001:0000185a       ?deleteItem@?$QPtrList@VQPopupMenu@@@@EAEXPAX@Z 1000285a f i cfg_alarm_overview.obj
 0001:00001875       ?deleteItem@?$QPtrList@VCOutputFile@@@@EAEXPAX@Z 10002875 f i cfg_alarm_overview.obj
 0001:00001875       ?deleteItem@?$QPtrList@VCInputFile@@@@EAEXPAX@Z 10002875 f i cfg_alarm_overview.obj
 0001:0000188f       ?deref@?$QGuardedPtr@VQPopupMenu@@@@AAEXXZ 1000288f f i cfg_alarm_overview.obj
 0001:0000188f       ?deref@?$QGuardedPtr@VQDockWindow@@@@AAEXXZ 1000288f f i cfg_alarm_overview.obj
 0001:000018a4       ?validate@config_plugin_base@@UAE_NXZ 100028a4 f i cfg_alarm_overview.obj
 0001:000018a4       ?isDirty@config_plugin_base@@UAE_NXZ 100028a4 f i cfg_alarm_overview.obj
 0001:000018a4       ?isDirty@cfg_alarm_overview@@UAE_NXZ 100028a4 f i cfg_alarm_overview.obj
 0001:000018a7       ?markDirty@cfg_alarm_overview@@QAEXXZ 100028a7 f   cfg_alarm_overview.obj
 0001:00001905       ?menuNewSystem@cfg_alarm_overview@@QAEXXZ 10002905 f   cfg_alarm_overview.obj
 0001:00001912       ?menus@cfg_alarm_overview@@UAE?AVQPopupMenuList@@XZ 10002912 f   cfg_alarm_overview.obj
 0001:0000195c       ?menus@config_plugin_base@@UAE?AVQPopupMenuList@@XZ 1000295c f i cfg_alarm_overview.obj
 0001:0000197f       ?metaObject@cfg_alarm_overview@@UBEPAVQMetaObject@@XZ 1000297f f i cfg_alarm_overview.obj
 0001:00001984       ?navigate@cfg_alarm_overview@@UAEXABVQString@@0@Z 10002984 f   cfg_alarm_overview.obj
 0001:000019ad       ?navigate@config_plugin_base@@UAEXABVQString@@0@Z 100029ad f i cfg_alarm_overview.obj
 0001:000019b0       ?reply@cfg_alarm_overview@@UAEXPAVresponse@@@Z 100029b0 f   cfg_alarm_overview.obj
 0001:0000265d       ?resizeEvent@cfg_alarm_overview@@UAEXPAVQResizeEvent@@@Z 1000365d f   cfg_alarm_overview.obj
 0001:00002692       ?selectSystem@cfg_alarm_overview@@QAEXABVQString@@@Z 10003692 f   cfg_alarm_overview.obj
 0001:00002986       ?toolbars@cfg_alarm_overview@@UAE?AVQDockWindowList@@XZ 10003986 f   cfg_alarm_overview.obj
 0001:000029d0       ?toolbars@config_plugin_base@@UAE?AVQDockWindowList@@XZ 100039d0 f i cfg_alarm_overview.obj
 0001:000029f3       ??0dialog@@QAE@PAVQWidget@@PBDI@Z 100039f3 f   dialogimpl.obj
 0001:00002a1b       ??1dialog@@UAE@XZ          10003a1b f   dialogimpl.obj
 0001:00002a2d       ??_Edialog@@WCI@AEPAXI@Z   10003a2d f i dialogimpl.obj
 0001:00002a35       ??_Gdialog@@UAEPAXI@Z      10003a35 f i dialogimpl.obj
 0001:00002a35       ??_Edialog@@UAEPAXI@Z      10003a35 f i dialogimpl.obj
 0001:00002a54       ?metaObject@dialog@@UBEPAVQMetaObject@@XZ 10003a54 f i dialogimpl.obj
 0001:00002a59       ??0CInputFile@@QAE@XZ      10003a59 f   InputFile.obj
 0001:00002a9b       ??1CInputFile@@UAE@XZ      10003a9b f   InputFile.obj
 0001:00002ae2       ??_GCInputFile@@UAEPAXI@Z  10003ae2 f i InputFile.obj
 0001:00002ae2       ??_ECInputFile@@UAEPAXI@Z  10003ae2 f i InputFile.obj
 0001:00002b01       ??0COutputFile@@QAE@XZ     10003b01 f   OutputFile.obj
 0001:00002b43       ??1COutputFile@@UAE@XZ     10003b43 f   OutputFile.obj
 0001:00002b8a       ??_GCOutputFile@@UAEPAXI@Z 10003b8a f i OutputFile.obj
 0001:00002b8a       ??_ECOutputFile@@UAEPAXI@Z 10003b8a f i OutputFile.obj
 0001:00002ba9       ??_Gplugindesc@@UAEPAXI@Z  10003ba9 f i plugindesc.obj
 0001:00002ba9       ??_Eplugindesc@@UAEPAXI@Z  10003ba9 f i plugindesc.obj
 0001:00002ba9       ??_Econfig_plugin_desc_base@@UAEPAXI@Z 10003ba9 f i plugindesc.obj
 0001:00002ba9       ??_Gconfig_plugin_desc_base@@UAEPAXI@Z 10003ba9 f i plugindesc.obj
 0001:00002bc9       ?create@plugindesc@@UAEPAVconfig_plugin_base@@ABVQString@@00@Z 10003bc9 f   plugindesc.obj
 0001:00002c04       ?keys@plugindesc@@UAE?AVQStringList@@ABVQString@@0@Z 10003c04 f   plugindesc.obj
 0001:00002c5f       ?pixmap@plugindesc@@UAE?AVQPixmap@@ABVQString@@@Z 10003c5f f   plugindesc.obj
 0001:00002c7e       _load_bncs_config_plugin_desc 10003c7e f   plugindesc.obj
 0001:00002c94       ??0dialogBase@@QAE@PAVQWidget@@PBDI@Z 10003c94 f   dialog.obj
 0001:0000344b       ??1dialogBase@@UAE@XZ      1000444b f   dialog.obj
 0001:0000348b       ??_ECAlm_sys_select@@WCI@AEPAXI@Z 1000448b f i dialog.obj
 0001:00003493       ??_EQButtonGroup@@WCI@AEPAXI@Z 10004493 f i dialog.obj
 0001:0000349b       ??_EQHBoxLayout@@WCI@AEPAXI@Z 1000449b f i dialog.obj
 0001:000034a3       ??_EQLabel@@WCI@AEPAXI@Z   100044a3 f i dialog.obj
 0001:000034ab       ??_EQListView@@WCI@AEPAXI@Z 100044ab f i dialog.obj
 0001:000034b3       ??_EQPushButton@@WCI@AEPAXI@Z 100044b3 f i dialog.obj
 0001:000034bb       ??_EQVBoxLayout@@WCI@AEPAXI@Z 100044bb f i dialog.obj
 0001:000034c3       ??_EdialogBase@@WCI@AEPAXI@Z 100044c3 f i dialog.obj
 0001:000034cb       ??_ECAlm_sys_select@@UAEPAXI@Z 100044cb f i dialog.obj
 0001:000034cb       ??_GCAlm_sys_select@@UAEPAXI@Z 100044cb f i dialog.obj
 0001:000034eb       ??_EQButtonGroup@@UAEPAXI@Z 100044eb f i dialog.obj
 0001:000034eb       ??_GQButtonGroup@@UAEPAXI@Z 100044eb f i dialog.obj
 0001:0000350b       ??_EQHBoxLayout@@UAEPAXI@Z 1000450b f i dialog.obj
 0001:0000350b       ??_GQHBoxLayout@@UAEPAXI@Z 1000450b f i dialog.obj
 0001:0000352b       ??_EQLabel@@UAEPAXI@Z      1000452b f i dialog.obj
 0001:0000352b       ??_GQLabel@@UAEPAXI@Z      1000452b f i dialog.obj
 0001:0000354b       ??_GQListView@@UAEPAXI@Z   1000454b f i dialog.obj
 0001:0000354b       ??_EQListView@@UAEPAXI@Z   1000454b f i dialog.obj
 0001:0000356b       ??_GQPushButton@@UAEPAXI@Z 1000456b f i dialog.obj
 0001:0000356b       ??_EQPushButton@@UAEPAXI@Z 1000456b f i dialog.obj
 0001:0000358b       ??_GQSpacerItem@@UAEPAXI@Z 1000458b f i dialog.obj
 0001:0000358b       ??_EQSpacerItem@@UAEPAXI@Z 1000458b f i dialog.obj
 0001:000035ab       ??_EQVBoxLayout@@UAEPAXI@Z 100045ab f i dialog.obj
 0001:000035ab       ??_GQVBoxLayout@@UAEPAXI@Z 100045ab f i dialog.obj
 0001:000035cb       ??_EdialogBase@@UAEPAXI@Z  100045cb f i dialog.obj
 0001:000035cb       ??_GdialogBase@@UAEPAXI@Z  100045cb f i dialog.obj
 0001:000035ea       ?languageChange@dialogBase@@MAEXXZ 100045ea f   dialog.obj
 0001:000038de       ?metaObject@dialogBase@@UBEPAVQMetaObject@@XZ 100048de f i dialog.obj
 0001:000038e3       ?className@cfg_alarm_overview@@UBEPBDXZ 100048e3 f   moc_cfg_alarm_overview.obj
 0001:000038e9       ?command@cfg_alarm_overview@@IAEXVQString@@0@Z 100048e9 f   moc_cfg_alarm_overview.obj
 0001:000039a9       ?qt_cast@cfg_alarm_overview@@UAEPAXPBD@Z 100049a9 f   moc_cfg_alarm_overview.obj
 0001:000039d7       ?qt_emit@cfg_alarm_overview@@UAE_NHPAUQUObject@@@Z 100049d7 f   moc_cfg_alarm_overview.obj
 0001:00003a3b       ?qt_invoke@cfg_alarm_overview@@UAE_NHPAUQUObject@@@Z 10004a3b f   moc_cfg_alarm_overview.obj
 0001:00003b43       ?qt_property@cfg_alarm_overview@@UAE_NHHPAVQVariant@@@Z 10004b43 f   moc_cfg_alarm_overview.obj
 0001:00003b43       ?qt_property@dialogBase@@UAE_NHHPAVQVariant@@@Z 10004b43 f   moc_dialog.obj
 0001:00003b4d       ?staticMetaObject@cfg_alarm_overview@@SAPAVQMetaObject@@XZ 10004b4d f   moc_cfg_alarm_overview.obj
 0001:00003c50       ?className@dialogBase@@UBEPBDXZ 10004c50 f   moc_dialog.obj
 0001:00003c56       ?qt_cast@dialogBase@@UAEPAXPBD@Z 10004c56 f   moc_dialog.obj
 0001:00003c84       ?qt_emit@dialogBase@@UAE_NHPAUQUObject@@@Z 10004c84 f   moc_dialog.obj
 0001:00003c8e       ?qt_invoke@dialogBase@@UAE_NHPAUQUObject@@@Z 10004c8e f   moc_dialog.obj
 0001:00003cc0       ?staticMetaObject@dialogBase@@SAPAVQMetaObject@@XZ 10004cc0 f   moc_dialog.obj
 0001:00003d0a       ?tr@dialogBase@@SA?AVQString@@PBD0@Z 10004d0a f   moc_dialog.obj
 0001:00003d4d       ?className@dialog@@UBEPBDXZ 10004d4d f   moc_dialogimpl.obj
 0001:00003d53       ?qt_cast@dialog@@UAEPAXPBD@Z 10004d53 f   moc_dialogimpl.obj
 0001:00003d80       ?qt_emit@dialog@@UAE_NHPAUQUObject@@@Z 10004d80 f   moc_dialogimpl.obj
 0001:00003d89       ?qt_invoke@dialog@@UAE_NHPAUQUObject@@@Z 10004d89 f   moc_dialogimpl.obj
 0001:00003d92       ?qt_property@dialog@@UAE_NHHPAVQVariant@@@Z 10004d92 f   moc_dialogimpl.obj
 0001:00003d9b       ?staticMetaObject@dialog@@SAPAVQMetaObject@@XZ 10004d9b f   moc_dialogimpl.obj
 0001:00003de0       ?setName@QWidget@@UAEXPBD@Z 10004de0 f   qt-mt323:qt-mt323.dll
 0001:00003de6       ?acceptDrop@QListViewItem@@UBE_NPBVQMimeSource@@@Z 10004de6 f   qt-mt323:qt-mt323.dll
 0001:00003dec       ?activate@QListViewItem@@MAEXXZ 10004dec f   qt-mt323:qt-mt323.dll
 0001:00003df2       ?activateItemAt@QPopupMenu@@UAEXH@Z 10004df2 f   qt-mt323:qt-mt323.dll
 0001:00003df8       ?addTo@QAction@@UAE_NPAVQWidget@@@Z 10004df8 f   qt-mt323:qt-mt323.dll
 0001:00003dfe       ?addedTo@QAction@@MAEXHPAVQPopupMenu@@@Z 10004dfe f   qt-mt323:qt-mt323.dll
 0001:00003e04       ?addedTo@QAction@@MAEXPAVQWidget@@0@Z 10004e04 f   qt-mt323:qt-mt323.dll
 0001:00003e0a       ?adjustSize@QWidget@@UAEXXZ 10004e0a f   qt-mt323:qt-mt323.dll
 0001:00003e10       ?cancelRename@QListViewItem@@MAEXH@Z 10004e10 f   qt-mt323:qt-mt323.dll
 0001:00003e16       ?checkConnectArgs@QObject@@MAE_NPBDPBV1@0@Z 10004e16 f   qt-mt323:qt-mt323.dll
 0001:00003e1c       ?childEvent@QObject@@MAEXPAVQChildEvent@@@Z 10004e1c f   qt-mt323:qt-mt323.dll
 0001:00003e22       ?className@QAction@@UBEPBDXZ 10004e22 f   qt-mt323:qt-mt323.dll
 0001:00003e28       ?className@QGuardedPtrPrivate@@UBEPBDXZ 10004e28 f   qt-mt323:qt-mt323.dll
 0001:00003e2e       ?className@QPopupMenu@@UBEPBDXZ 10004e2e f   qt-mt323:qt-mt323.dll
 0001:00003e34       ?className@QToolBar@@UBEPBDXZ 10004e34 f   qt-mt323:qt-mt323.dll
 0001:00003e3a       ?className@QWidget@@UBEPBDXZ 10004e3a f   qt-mt323:qt-mt323.dll
 0001:00003e40       ?clear@?$QPtrList@VQDockWindow@@@@UAEXXZ 10004e40 f   qt-mt323:qt-mt323.dll
 0001:00003e46       ?clear@QToolBar@@UAEXXZ    10004e46 f   qt-mt323:qt-mt323.dll
 0001:00003e4c       ?close@QWidget@@UAE_N_N@Z  10004e4c f   qt-mt323:qt-mt323.dll
 0001:00003e52       ?closeEvent@QPopupMenu@@MAEXPAVQCloseEvent@@@Z 10004e52 f   qt-mt323:qt-mt323.dll
 0001:00003e58       ?closeEvent@QWidget@@MAEXPAVQCloseEvent@@@Z 10004e58 f   qt-mt323:qt-mt323.dll
 0001:00003e5e       ?cmd@QPaintDevice@@MAE_NHPAVQPainter@@PATQPDevCmdParam@@@Z 10004e5e f   qt-mt323:qt-mt323.dll
 0001:00003e64       ?compare@QListViewItem@@UBEHPAV1@H_N@Z 10004e64 f   qt-mt323:qt-mt323.dll
 0001:00003e6a       ?compareItems@QGList@@MAEHPAX0@Z 10004e6a f   qt-mt323:qt-mt323.dll
 0001:00003e70       ?connectNotify@QObject@@MAEXPBD@Z 10004e70 f   qt-mt323:qt-mt323.dll
 0001:00003e76       ?contextMenuEvent@QDockWindow@@MAEXPAVQContextMenuEvent@@@Z 10004e76 f   qt-mt323:qt-mt323.dll
 0001:00003e7c       ?contextMenuEvent@QWidget@@MAEXPAVQContextMenuEvent@@@Z 10004e7c f   qt-mt323:qt-mt323.dll
 0001:00003e82       ?count@?$QPtrList@VQDockWindow@@@@UBEIXZ 10004e82 f   qt-mt323:qt-mt323.dll
 0001:00003e88       ?create@QWidget@@MAEXPAUHWND__@@_N1@Z 10004e88 f   qt-mt323:qt-mt323.dll
 0001:00003e8e       ?customEvent@QObject@@MAEXPAVQCustomEvent@@@Z 10004e8e f   qt-mt323:qt-mt323.dll
 0001:00003e94       ?customWhatsThis@QPopupMenu@@UBE_NXZ 10004e94 f   qt-mt323:qt-mt323.dll
 0001:00003e9a       ?customWhatsThis@QWidget@@UBE_NXZ 10004e9a f   qt-mt323:qt-mt323.dll
 0001:00003ea0       ?deleteItem@?$QPtrList@VQDockWindow@@@@EAEXPAX@Z 10004ea0 f   qt-mt323:qt-mt323.dll
 0001:00003ea6       ?destroy@QWidget@@MAEX_N0@Z 10004ea6 f   qt-mt323:qt-mt323.dll
 0001:00003eac       ?disconnectNotify@QObject@@MAEXPBD@Z 10004eac f   qt-mt323:qt-mt323.dll
 0001:00003eb2       ?dock@QDockWindow@@UAEXXZ  10004eb2 f   qt-mt323:qt-mt323.dll
 0001:00003eb8       ?dragEnterEvent@QWidget@@MAEXPAVQDragEnterEvent@@@Z 10004eb8 f   qt-mt323:qt-mt323.dll
 0001:00003ebe       ?dragEntered@QListViewItem@@MAEXXZ 10004ebe f   qt-mt323:qt-mt323.dll
 0001:00003ec4       ?dragLeaveEvent@QWidget@@MAEXPAVQDragLeaveEvent@@@Z 10004ec4 f   qt-mt323:qt-mt323.dll
 0001:00003eca       ?dragLeft@QListViewItem@@MAEXXZ 10004eca f   qt-mt323:qt-mt323.dll
 0001:00003ed0       ?dragMoveEvent@QWidget@@MAEXPAVQDragMoveEvent@@@Z 10004ed0 f   qt-mt323:qt-mt323.dll
 0001:00003ed6       ?drawContents@QDockWindow@@MAEXPAVQPainter@@@Z 10004ed6 f   qt-mt323:qt-mt323.dll
 0001:00003edc       ?drawContents@QPopupMenu@@MAEXPAVQPainter@@@Z 10004edc f   qt-mt323:qt-mt323.dll
 0001:00003ee2       ?drawFrame@QDockWindow@@MAEXPAVQPainter@@@Z 10004ee2 f   qt-mt323:qt-mt323.dll
 0001:00003ee8       ?drawFrame@QFrame@@MAEXPAVQPainter@@@Z 10004ee8 f   qt-mt323:qt-mt323.dll
 0001:00003eee       ?dropEvent@QWidget@@MAEXPAVQDropEvent@@@Z 10004eee f   qt-mt323:qt-mt323.dll
 0001:00003ef4       ?dropped@QListViewItem@@MAEXPAVQDropEvent@@@Z 10004ef4 f   qt-mt323:qt-mt323.dll
 0001:00003efa       ?enabledChange@QPopupMenu@@MAEX_N@Z 10004efa f   qt-mt323:qt-mt323.dll
 0001:00003f00       ?enabledChange@QWidget@@MAEX_N@Z 10004f00 f   qt-mt323:qt-mt323.dll
 0001:00003f06       ?enforceSortOrder@QListViewItem@@MBEXXZ 10004f06 f   qt-mt323:qt-mt323.dll
 0001:00003f0c       ?enterEvent@QWidget@@MAEXPAVQEvent@@@Z 10004f0c f   qt-mt323:qt-mt323.dll
 0001:00003f12       ?event@QObject@@UAE_NPAVQEvent@@@Z 10004f12 f   qt-mt323:qt-mt323.dll
 0001:00003f18       ?event@QToolBar@@UAE_NPAVQEvent@@@Z 10004f18 f   qt-mt323:qt-mt323.dll
 0001:00003f1e       ?event@QWidget@@MAE_NPAVQEvent@@@Z 10004f1e f   qt-mt323:qt-mt323.dll
 0001:00003f24       ?eventFilter@QDockWindow@@UAE_NPAVQObject@@PAVQEvent@@@Z 10004f24 f   qt-mt323:qt-mt323.dll
 0001:00003f2a       ?eventFilter@QObject@@UAE_NPAV1@PAVQEvent@@@Z 10004f2a f   qt-mt323:qt-mt323.dll
 0001:00003f30       ?focusInEvent@QPopupMenu@@MAEXPAVQFocusEvent@@@Z 10004f30 f   qt-mt323:qt-mt323.dll
 0001:00003f36       ?focusInEvent@QWidget@@MAEXPAVQFocusEvent@@@Z 10004f36 f   qt-mt323:qt-mt323.dll
 0001:00003f3c       ?focusNextPrevChild@QPopupMenu@@MAE_N_N@Z 10004f3c f   qt-mt323:qt-mt323.dll
 0001:00003f42       ?focusNextPrevChild@QWidget@@MAE_N_N@Z 10004f42 f   qt-mt323:qt-mt323.dll
 0001:00003f48       ?focusOutEvent@QPopupMenu@@MAEXPAVQFocusEvent@@@Z 10004f48 f   qt-mt323:qt-mt323.dll
 0001:00003f4e       ?focusOutEvent@QWidget@@MAEXPAVQFocusEvent@@@Z 10004f4e f   qt-mt323:qt-mt323.dll
 0001:00003f54       ?fontChange@QWidget@@MAEXABVQFont@@@Z 10004f54 f   qt-mt323:qt-mt323.dll
 0001:00003f5a       ?fontInf@QPaintDevice@@MBEHPAVQFont@@H@Z 10004f5a f   qt-mt323:qt-mt323.dll
 0001:00003f60       ?fontMet@QPaintDevice@@MBEHPAVQFont@@HPBDH@Z 10004f60 f   qt-mt323:qt-mt323.dll
 0001:00003f66       ?frameChanged@QFrame@@MAEXXZ 10004f66 f   qt-mt323:qt-mt323.dll
 0001:00003f6c       ?frameChanged@QPopupMenu@@EAEXXZ 10004f6c f   qt-mt323:qt-mt323.dll
 0001:00003f72       ?handle@QPaintDevice@@UBEPAUHDC__@@XZ 10004f72 f   qt-mt323:qt-mt323.dll
 0001:00003f78       ?heightForWidth@QWidget@@UBEHH@Z 10004f78 f   qt-mt323:qt-mt323.dll
 0001:00003f7e       ?hide@QPopupMenu@@UAEXXZ   10004f7e f   qt-mt323:qt-mt323.dll
 0001:00003f84       ?hide@QToolBar@@UAEXXZ     10004f84 f   qt-mt323:qt-mt323.dll
 0001:00003f8a       ?hide@QWidget@@UAEXXZ      10004f8a f   qt-mt323:qt-mt323.dll
 0001:00003f90       ?hideEvent@QDockWindow@@MAEXPAVQHideEvent@@@Z 10004f90 f   qt-mt323:qt-mt323.dll
 0001:00003f96       ?hideEvent@QWidget@@MAEXPAVQHideEvent@@@Z 10004f96 f   qt-mt323:qt-mt323.dll
 0001:00003f9c       ?imComposeEvent@QWidget@@MAEXPAVQIMEvent@@@Z 10004f9c f   qt-mt323:qt-mt323.dll
 0001:00003fa2       ?imEndEvent@QWidget@@MAEXPAVQIMEvent@@@Z 10004fa2 f   qt-mt323:qt-mt323.dll
 0001:00003fa8       ?imStartEvent@QWidget@@MAEXPAVQIMEvent@@@Z 10004fa8 f   qt-mt323:qt-mt323.dll
 0001:00003fae       ?insertChild@QObject@@UAEXPAV1@@Z 10004fae f   qt-mt323:qt-mt323.dll
 0001:00003fb4       ?insertItem@QListViewItem@@UAEXPAV1@@Z 10004fb4 f   qt-mt323:qt-mt323.dll
 0001:00003fba       ?invalidateHeight@QListViewItem@@UAEXXZ 10004fba f   qt-mt323:qt-mt323.dll
 0001:00003fc0       ?key@QListViewItem@@UBE?AVQString@@H_N@Z 10004fc0 f   qt-mt323:qt-mt323.dll
 0001:00003fc6       ?keyPressEvent@QPopupMenu@@MAEXPAVQKeyEvent@@@Z 10004fc6 f   qt-mt323:qt-mt323.dll
 0001:00003fcc       ?keyPressEvent@QWidget@@MAEXPAVQKeyEvent@@@Z 10004fcc f   qt-mt323:qt-mt323.dll
 0001:00003fd2       ?keyReleaseEvent@QWidget@@MAEXPAVQKeyEvent@@@Z 10004fd2 f   qt-mt323:qt-mt323.dll
 0001:00003fd8       ?leaveEvent@QPopupMenu@@MAEXPAVQEvent@@@Z 10004fd8 f   qt-mt323:qt-mt323.dll
 0001:00003fde       ?leaveEvent@QWidget@@MAEXPAVQEvent@@@Z 10004fde f   qt-mt323:qt-mt323.dll
 0001:00003fe4       ?menuContentsChanged@QPopupMenu@@EAEXXZ 10004fe4 f   qt-mt323:qt-mt323.dll
 0001:00003fea       ?menuDelPopup@QPopupMenu@@EAEXPAV1@@Z 10004fea f   qt-mt323:qt-mt323.dll
 0001:00003ff0       ?menuInsPopup@QPopupMenu@@EAEXPAV1@@Z 10004ff0 f   qt-mt323:qt-mt323.dll
 0001:00003ff6       ?menuStateChanged@QPopupMenu@@EAEXXZ 10004ff6 f   qt-mt323:qt-mt323.dll
 0001:00003ffe       ?metaObject@QAction@@UBEPAVQMetaObject@@XZ 10004ffe f   qt-mt323:qt-mt323.dll
 0001:00004004       ?metaObject@QGuardedPtrPrivate@@UBEPAVQMetaObject@@XZ 10005004 f   qt-mt323:qt-mt323.dll
 0001:0000400a       ?metaObject@QPopupMenu@@UBEPAVQMetaObject@@XZ 1000500a f   qt-mt323:qt-mt323.dll
 0001:00004010       ?metaObject@QToolBar@@UBEPAVQMetaObject@@XZ 10005010 f   qt-mt323:qt-mt323.dll
 0001:00004016       ?metaObject@QWidget@@UBEPAVQMetaObject@@XZ 10005016 f   qt-mt323:qt-mt323.dll
 0001:0000401c       ?metric@QWidget@@MBEHH@Z   1000501c f   qt-mt323:qt-mt323.dll
 0001:00004022       ?minimumSizeHint@QToolBar@@UBE?AVQSize@@XZ 10005022 f   qt-mt323:qt-mt323.dll
 0001:00004028       ?minimumSizeHint@QWidget@@UBE?AVQSize@@XZ 10005028 f   qt-mt323:qt-mt323.dll
 0001:0000402e       ?mouseDoubleClickEvent@QWidget@@MAEXPAVQMouseEvent@@@Z 1000502e f   qt-mt323:qt-mt323.dll
 0001:00004034       ?mouseMoveEvent@QPopupMenu@@MAEXPAVQMouseEvent@@@Z 10005034 f   qt-mt323:qt-mt323.dll
 0001:0000403a       ?mouseMoveEvent@QWidget@@MAEXPAVQMouseEvent@@@Z 1000503a f   qt-mt323:qt-mt323.dll
 0001:00004040       ?mousePressEvent@QPopupMenu@@MAEXPAVQMouseEvent@@@Z 10005040 f   qt-mt323:qt-mt323.dll
 0001:00004046       ?mousePressEvent@QWidget@@MAEXPAVQMouseEvent@@@Z 10005046 f   qt-mt323:qt-mt323.dll
 0001:0000404c       ?mouseReleaseEvent@QPopupMenu@@MAEXPAVQMouseEvent@@@Z 1000504c f   qt-mt323:qt-mt323.dll
 0001:00004052       ?mouseReleaseEvent@QWidget@@MAEXPAVQMouseEvent@@@Z 10005052 f   qt-mt323:qt-mt323.dll
 0001:00004058       ?move@QWidget@@UAEXHH@Z    10005058 f   qt-mt323:qt-mt323.dll
 0001:0000405e       ?moveEvent@QWidget@@MAEXPAVQMoveEvent@@@Z 1000505e f   qt-mt323:qt-mt323.dll
 0001:00004064       ?newItem@QPtrCollection@@MAEPAXPAX@Z 10005064 f   qt-mt323:qt-mt323.dll
 0001:0000406a       ?okRename@QListViewItem@@MAEXH@Z 1000506a f   qt-mt323:qt-mt323.dll
 0001:00004070       ?paintBranches@QListViewItem@@UAEXPAVQPainter@@ABVQColorGroup@@HHH@Z 10005070 f   qt-mt323:qt-mt323.dll
 0001:00004076       ?paintCell@QListViewItem@@UAEXPAVQPainter@@ABVQColorGroup@@HHH@Z 10005076 f   qt-mt323:qt-mt323.dll
 0001:0000407c       ?paintEvent@QFrame@@MAEXPAVQPaintEvent@@@Z 1000507c f   qt-mt323:qt-mt323.dll
 0001:00004082       ?paintEvent@QPopupMenu@@MAEXPAVQPaintEvent@@@Z 10005082 f   qt-mt323:qt-mt323.dll
 0001:00004088       ?paintEvent@QWidget@@MAEXPAVQPaintEvent@@@Z 10005088 f   qt-mt323:qt-mt323.dll
 0001:0000408e       ?paintFocus@QListViewItem@@UAEXPAVQPainter@@ABVQColorGroup@@ABVQRect@@@Z 1000508e f   qt-mt323:qt-mt323.dll
 0001:00004094       ?paletteChange@QWidget@@MAEXABVQPalette@@@Z 10005094 f   qt-mt323:qt-mt323.dll
 0001:0000409a       ?pixmap@QListViewItem@@UBEPBVQPixmap@@H@Z 1000509a f   qt-mt323:qt-mt323.dll
 0001:000040a0       ?polish@QWidget@@UAEXXZ    100050a0 f   qt-mt323:qt-mt323.dll
 0001:000040a6       ?property@QObject@@UBE?AVQVariant@@PBD@Z 100050a6 f   qt-mt323:qt-mt323.dll
 0001:000040ac       ?qt_cast@QAction@@UAEPAXPBD@Z 100050ac f   qt-mt323:qt-mt323.dll
 0001:000040b2       ?qt_cast@QGuardedPtrPrivate@@UAEPAXPBD@Z 100050b2 f   qt-mt323:qt-mt323.dll
 0001:000040b8       ?qt_cast@QPopupMenu@@UAEPAXPBD@Z 100050b8 f   qt-mt323:qt-mt323.dll
 0001:000040be       ?qt_cast@QToolBar@@UAEPAXPBD@Z 100050be f   qt-mt323:qt-mt323.dll
 0001:000040c4       ?qt_cast@QWidget@@UAEPAXPBD@Z 100050c4 f   qt-mt323:qt-mt323.dll
 0001:000040ca       ?qt_emit@QAction@@UAE_NHPAUQUObject@@@Z 100050ca f   qt-mt323:qt-mt323.dll
 0001:000040d0       ?qt_emit@QGuardedPtrPrivate@@UAE_NHPAUQUObject@@@Z 100050d0 f   qt-mt323:qt-mt323.dll
 0001:000040d6       ?qt_emit@QPopupMenu@@UAE_NHPAUQUObject@@@Z 100050d6 f   qt-mt323:qt-mt323.dll
 0001:000040dc       ?qt_emit@QToolBar@@UAE_NHPAUQUObject@@@Z 100050dc f   qt-mt323:qt-mt323.dll
 0001:000040e2       ?qt_emit@QWidget@@UAE_NHPAUQUObject@@@Z 100050e2 f   qt-mt323:qt-mt323.dll
 0001:000040e8       ?qt_invoke@QAction@@UAE_NHPAUQUObject@@@Z 100050e8 f   qt-mt323:qt-mt323.dll
 0001:000040ee       ?qt_invoke@QGuardedPtrPrivate@@UAE_NHPAUQUObject@@@Z 100050ee f   qt-mt323:qt-mt323.dll
 0001:000040f4       ?qt_invoke@QPopupMenu@@UAE_NHPAUQUObject@@@Z 100050f4 f   qt-mt323:qt-mt323.dll
 0001:000040fa       ?qt_invoke@QToolBar@@UAE_NHPAUQUObject@@@Z 100050fa f   qt-mt323:qt-mt323.dll
 0001:00004100       ?qt_invoke@QWidget@@UAE_NHPAUQUObject@@@Z 10005100 f   qt-mt323:qt-mt323.dll
 0001:00004106       ?qt_property@QAction@@UAE_NHHPAVQVariant@@@Z 10005106 f   qt-mt323:qt-mt323.dll
 0001:0000410c       ?qt_property@QGuardedPtrPrivate@@UAE_NHHPAVQVariant@@@Z 1000510c f   qt-mt323:qt-mt323.dll
 0001:00004112       ?qt_property@QPopupMenu@@UAE_NHHPAVQVariant@@@Z 10005112 f   qt-mt323:qt-mt323.dll
 0001:00004118       ?qt_property@QToolBar@@UAE_NHHPAVQVariant@@@Z 10005118 f   qt-mt323:qt-mt323.dll
 0001:0000411e       ?qt_property@QWidget@@UAE_NHHPAVQVariant@@@Z 1000511e f   qt-mt323:qt-mt323.dll
 0001:00004124       ?read@QGDict@@MAEAAVQDataStream@@AAV2@AAPAX@Z 10005124 f   qt-mt323:qt-mt323.dll
 0001:0000412a       ?read@QGList@@MAEAAVQDataStream@@AAV2@AAPAX@Z 1000512a f   qt-mt323:qt-mt323.dll
 0001:00004130       ?removeChild@QObject@@UAEXPAV1@@Z 10005130 f   qt-mt323:qt-mt323.dll
 0001:00004136       ?removeFrom@QAction@@UAE_NPAVQWidget@@@Z 10005136 f   qt-mt323:qt-mt323.dll
 0001:0000413c       ?removeItem@QListViewItem@@UAEXPAV1@@Z 1000513c f   qt-mt323:qt-mt323.dll
 0001:00004142       ?reparent@QWidget@@UAEXPAV1@IABVQPoint@@_N@Z 10005142 f   qt-mt323:qt-mt323.dll
 0001:00004148       ?resize@QWidget@@UAEXHH@Z  10005148 f   qt-mt323:qt-mt323.dll
 0001:0000414e       ?resizeEvent@QFrame@@MAEXPAVQResizeEvent@@@Z 1000514e f   qt-mt323:qt-mt323.dll
 0001:00004154       ?resizeEvent@QToolBar@@MAEXPAVQResizeEvent@@@Z 10005154 f   qt-mt323:qt-mt323.dll
 0001:0000415a       ?resizeEvent@QWidget@@MAEXPAVQResizeEvent@@@Z 1000515a f   qt-mt323:qt-mt323.dll
 0001:00004160       ?resolution@QPaintDevice@@UBEHXZ 10005160 f   qt-mt323:qt-mt323.dll
 0001:00004166       ?rtti@QListViewItem@@UBEHXZ 10005166 f   qt-mt323:qt-mt323.dll
 0001:0000416c       ?setAccel@QAction@@UAEXABVQKeySequence@@@Z 1000516c f   qt-mt323:qt-mt323.dll
 0001:00004172       ?setAcceptDrops@QWidget@@UAEX_N@Z 10005172 f   qt-mt323:qt-mt323.dll
 0001:00004178       ?setActiveItem@QPopupMenu@@UAEXH@Z 10005178 f   qt-mt323:qt-mt323.dll
 0001:0000417e       ?setActiveWindow@QWidget@@UAEXXZ 1000517e f   qt-mt323:qt-mt323.dll
 0001:00004184       ?setAutoMask@QWidget@@UAEX_N@Z 10005184 f   qt-mt323:qt-mt323.dll
 0001:0000418a       ?setBackgroundColor@QWidget@@UAEXABVQColor@@@Z 1000518a f   qt-mt323:qt-mt323.dll
 0001:00004190       ?setBackgroundMode@QWidget@@UAEXW4BackgroundMode@Qt@@@Z 10005190 f   qt-mt323:qt-mt323.dll
 0001:00004196       ?setBackgroundOrigin@QWidget@@UAEXW4BackgroundOrigin@1@@Z 10005196 f   qt-mt323:qt-mt323.dll
 0001:0000419c       ?setBackgroundPixmap@QWidget@@UAEXABVQPixmap@@@Z 1000519c f   qt-mt323:qt-mt323.dll
 0001:000041a2       ?setCaption@QDockWindow@@UAEXABVQString@@@Z 100051a2 f   qt-mt323:qt-mt323.dll
 0001:000041a8       ?setCaption@QWidget@@UAEXABVQString@@@Z 100051a8 f   qt-mt323:qt-mt323.dll
 0001:000041ae       ?setCheckable@QPopupMenu@@UAEX_N@Z 100051ae f   qt-mt323:qt-mt323.dll
 0001:000041b4       ?setCloseMode@QDockWindow@@UAEXH@Z 100051b4 f   qt-mt323:qt-mt323.dll
 0001:000041ba       ?setCursor@QWidget@@UAEXABVQCursor@@@Z 100051ba f   qt-mt323:qt-mt323.dll
 0001:000041c0       ?setDragEnabled@QListViewItem@@UAEX_N@Z 100051c0 f   qt-mt323:qt-mt323.dll
 0001:000041c6       ?setDropEnabled@QListViewItem@@UAEX_N@Z 100051c6 f   qt-mt323:qt-mt323.dll
 0001:000041cc       ?setEnabled@QAction@@UAEX_N@Z 100051cc f   qt-mt323:qt-mt323.dll
 0001:000041d2       ?setEnabled@QListViewItem@@UAEX_N@Z 100051d2 f   qt-mt323:qt-mt323.dll
 0001:000041d8       ?setEnabled@QWidget@@UAEX_N@Z 100051d8 f   qt-mt323:qt-mt323.dll
 0001:000041de       ?setEraseColor@QWidget@@UAEXABVQColor@@@Z 100051de f   qt-mt323:qt-mt323.dll
 0001:000041e4       ?setErasePixmap@QWidget@@UAEXABVQPixmap@@@Z 100051e4 f   qt-mt323:qt-mt323.dll
 0001:000041ea       ?setExpandable@QListViewItem@@UAEX_N@Z 100051ea f   qt-mt323:qt-mt323.dll
 0001:000041f0       ?setFirstItemActive@QPopupMenu@@EAEXXZ 100051f0 f   qt-mt323:qt-mt323.dll
 0001:000041f6       ?setFixedExtentHeight@QDockWindow@@UAEXH@Z 100051f6 f   qt-mt323:qt-mt323.dll
 0001:000041fc       ?setFixedExtentWidth@QDockWindow@@UAEXH@Z 100051fc f   qt-mt323:qt-mt323.dll
 0001:00004202       ?setFocus@QWidget@@UAEXXZ  10005202 f   qt-mt323:qt-mt323.dll
 0001:00004208       ?setFocusPolicy@QWidget@@UAEXW4FocusPolicy@1@@Z 10005208 f   qt-mt323:qt-mt323.dll
 0001:0000420e       ?setFocusProxy@QWidget@@UAEXPAV1@@Z 1000520e f   qt-mt323:qt-mt323.dll
 0001:00004214       ?setFont@QPopupMenu@@UAEXABVQFont@@@Z 10005214 f   qt-mt323:qt-mt323.dll
 0001:0000421a       ?setFont@QWidget@@UAEXABVQFont@@@Z 1000521a f   qt-mt323:qt-mt323.dll
 0001:00004220       ?setFrameRect@QFrame@@UAEXABVQRect@@@Z 10005220 f   qt-mt323:qt-mt323.dll
 0001:00004226       ?setFrameStyle@QFrame@@UAEXH@Z 10005226 f   qt-mt323:qt-mt323.dll
 0001:0000422c       ?setGeometry@QWidget@@UAEXABVQRect@@@Z 1000522c f   qt-mt323:qt-mt323.dll
 0001:00004232       ?setGeometry@QWidget@@UAEXHHHH@Z 10005232 f   qt-mt323:qt-mt323.dll
 0001:00004238       ?setHeight@QListViewItem@@MAEXH@Z 10005238 f   qt-mt323:qt-mt323.dll
 0001:0000423e       ?setHorizontallyStretchable@QDockWindow@@UAEX_N@Z 1000523e f   qt-mt323:qt-mt323.dll
 0001:00004244       ?setIcon@QWidget@@UAEXABVQPixmap@@@Z 10005244 f   qt-mt323:qt-mt323.dll
 0001:0000424a       ?setIconSet@QAction@@UAEXABVQIconSet@@@Z 1000524a f   qt-mt323:qt-mt323.dll
 0001:00004250       ?setIconText@QWidget@@UAEXABVQString@@@Z 10005250 f   qt-mt323:qt-mt323.dll
 0001:00004256       ?setId@QMenuData@@UAEXHH@Z 10005256 f   qt-mt323:qt-mt323.dll
 0001:0000425c       ?setKeyCompression@QWidget@@MAEX_N@Z 1000525c f   qt-mt323:qt-mt323.dll
 0001:00004262       ?setLabel@QToolBar@@UAEXABVQString@@@Z 10005262 f   qt-mt323:qt-mt323.dll
 0001:00004268       ?setLineWidth@QFrame@@UAEXH@Z 10005268 f   qt-mt323:qt-mt323.dll
 0001:0000426e       ?setMargin@QFrame@@UAEXH@Z 1000526e f   qt-mt323:qt-mt323.dll
 0001:00004274       ?setMask@QWidget@@UAEXABVQBitmap@@@Z 10005274 f   qt-mt323:qt-mt323.dll
 0001:0000427a       ?setMask@QWidget@@UAEXABVQRegion@@@Z 1000527a f   qt-mt323:qt-mt323.dll
 0001:00004280       ?setMaximumSize@QWidget@@UAEXHH@Z 10005280 f   qt-mt323:qt-mt323.dll
 0001:00004286       ?setMenuText@QAction@@UAEXABVQString@@@Z 10005286 f   qt-mt323:qt-mt323.dll
 0001:0000428c       ?setMicroFocusHint@QWidget@@MAEXHHHH_NPAVQFont@@@Z 1000528c f   qt-mt323:qt-mt323.dll
 0001:00004292       ?setMidLineWidth@QFrame@@UAEXH@Z 10005292 f   qt-mt323:qt-mt323.dll
 0001:00004298       ?setMinimumSize@QToolBar@@UAEXHH@Z 10005298 f   qt-mt323:qt-mt323.dll
 0001:0000429e       ?setMinimumSize@QWidget@@UAEXHH@Z 1000529e f   qt-mt323:qt-mt323.dll
 0001:000042a4       ?setMouseTracking@QWidget@@UAEX_N@Z 100052a4 f   qt-mt323:qt-mt323.dll
 0001:000042aa       ?setMovingEnabled@QDockWindow@@UAEX_N@Z 100052aa f   qt-mt323:qt-mt323.dll
 0001:000042b0       ?setMultiLinesEnabled@QListViewItem@@UAEX_N@Z 100052b0 f   qt-mt323:qt-mt323.dll
 0001:000042b6       ?setName@QObject@@UAEXPBD@Z 100052b6 f   qt-mt323:qt-mt323.dll
 0001:000042bc       ?setNewLine@QDockWindow@@UAEX_N@Z 100052bc f   qt-mt323:qt-mt323.dll
 0001:000042c2       ?setOffset@QDockWindow@@UAEXH@Z 100052c2 f   qt-mt323:qt-mt323.dll
 0001:000042c8       ?setOn@QAction@@UAEX_N@Z   100052c8 f   qt-mt323:qt-mt323.dll
 0001:000042ce       ?setOpaqueMoving@QDockWindow@@UAEX_N@Z 100052ce f   qt-mt323:qt-mt323.dll
 0001:000042d4       ?setOpen@QListViewItem@@UAEX_N@Z 100052d4 f   qt-mt323:qt-mt323.dll
 0001:000042da       ?setOrientation@QToolBar@@UAEXW4Orientation@Qt@@@Z 100052da f   qt-mt323:qt-mt323.dll
 0001:000042e0       ?setPalette@QWidget@@UAEXABVQPalette@@@Z 100052e0 f   qt-mt323:qt-mt323.dll
 0001:000042e6       ?setPaletteBackgroundColor@QWidget@@UAEXABVQColor@@@Z 100052e6 f   qt-mt323:qt-mt323.dll
 0001:000042ec       ?setPaletteBackgroundPixmap@QWidget@@UAEXABVQPixmap@@@Z 100052ec f   qt-mt323:qt-mt323.dll
 0001:000042f2       ?setPixmap@QListViewItem@@UAEXHABVQPixmap@@@Z 100052f2 f   qt-mt323:qt-mt323.dll
 0001:000042f8       ?setProperty@QObject@@UAE_NPBDABVQVariant@@@Z 100052f8 f   qt-mt323:qt-mt323.dll
 0001:000042fe       ?setRenameEnabled@QListViewItem@@UAEXH_N@Z 100052fe f   qt-mt323:qt-mt323.dll
 0001:00004304       ?setResizeEnabled@QDockWindow@@UAEX_N@Z 10005304 f   qt-mt323:qt-mt323.dll
 0001:0000430a       ?setResolution@QPaintDevice@@UAEXH@Z 1000530a f   qt-mt323:qt-mt323.dll
 0001:00004310       ?setSelectable@QListViewItem@@UAEX_N@Z 10005310 f   qt-mt323:qt-mt323.dll
 0001:00004316       ?setSelected@QListViewItem@@UAEX_N@Z 10005316 f   qt-mt323:qt-mt323.dll
 0001:0000431c       ?setSizeIncrement@QWidget@@UAEXHH@Z 1000531c f   qt-mt323:qt-mt323.dll
 0001:00004322       ?setSizePolicy@QWidget@@UAEXVQSizePolicy@@@Z 10005322 f   qt-mt323:qt-mt323.dll
 0001:00004328       ?setStatusTip@QAction@@UAEXABVQString@@@Z 10005328 f   qt-mt323:qt-mt323.dll
 0001:0000432e       ?setStretchableWidget@QToolBar@@UAEXPAVQWidget@@@Z 1000532e f   qt-mt323:qt-mt323.dll
 0001:00004334       ?setText@QAction@@UAEXABVQString@@@Z 10005334 f   qt-mt323:qt-mt323.dll
 0001:0000433a       ?setText@QListViewItem@@UAEXHABVQString@@@Z 1000533a f   qt-mt323:qt-mt323.dll
 0001:00004340       ?setToggleAction@QAction@@UAEX_N@Z 10005340 f   qt-mt323:qt-mt323.dll
 0001:00004346       ?setToolTip@QAction@@UAEXABVQString@@@Z 10005346 f   qt-mt323:qt-mt323.dll
 0001:0000434c       ?setUpdatesEnabled@QWidget@@UAEX_N@Z 1000534c f   qt-mt323:qt-mt323.dll
 0001:00004352       ?setVerticallyStretchable@QDockWindow@@UAEX_N@Z 10005352 f   qt-mt323:qt-mt323.dll
 0001:00004358       ?setWFlags@QWidget@@MAEXI@Z 10005358 f   qt-mt323:qt-mt323.dll
 0001:0000435e       ?setWState@QWidget@@MAEXI@Z 1000535e f   qt-mt323:qt-mt323.dll
 0001:00004364       ?setWhatsThis@QAction@@UAEXABVQString@@@Z 10005364 f   qt-mt323:qt-mt323.dll
 0001:0000436a       ?setWidget@QDockWindow@@UAEXPAVQWidget@@@Z 1000536a f   qt-mt323:qt-mt323.dll
 0001:00004370       ?setup@QListViewItem@@UAEXXZ 10005370 f   qt-mt323:qt-mt323.dll
 0001:00004376       ?show@QPopupMenu@@UAEXXZ   10005376 f   qt-mt323:qt-mt323.dll
 0001:0000437c       ?show@QToolBar@@UAEXXZ     1000537c f   qt-mt323:qt-mt323.dll
 0001:00004382       ?show@QWidget@@UAEXXZ      10005382 f   qt-mt323:qt-mt323.dll
 0001:00004388       ?showEvent@QDockWindow@@MAEXPAVQShowEvent@@@Z 10005388 f   qt-mt323:qt-mt323.dll
 0001:0000438e       ?showEvent@QWidget@@MAEXPAVQShowEvent@@@Z 1000538e f   qt-mt323:qt-mt323.dll
 0001:00004394       ?showMaximized@QWidget@@UAEXXZ 10005394 f   qt-mt323:qt-mt323.dll
 0001:0000439a       ?showMinimized@QWidget@@UAEXXZ 1000539a f   qt-mt323:qt-mt323.dll
 0001:000043a0       ?showNormal@QWidget@@UAEXXZ 100053a0 f   qt-mt323:qt-mt323.dll
 0001:000043a6       ?sizeHint@QDockWindow@@UBE?AVQSize@@XZ 100053a6 f   qt-mt323:qt-mt323.dll
 0001:000043ac       ?sizeHint@QPopupMenu@@UBE?AVQSize@@XZ 100053ac f   qt-mt323:qt-mt323.dll
 0001:000043b2       ?sizeHint@QWidget@@UBE?AVQSize@@XZ 100053b2 f   qt-mt323:qt-mt323.dll
 0001:000043b8       ?sizePolicy@QWidget@@UBE?AVQSizePolicy@@XZ 100053b8 f   qt-mt323:qt-mt323.dll
 0001:000043be       ?sort@QListViewItem@@UAEXXZ 100053be f   qt-mt323:qt-mt323.dll
 0001:000043c4       ?sortChildItems@QListViewItem@@UAEXH_N@Z 100053c4 f   qt-mt323:qt-mt323.dll
 0001:000043ca       ?startRename@QListViewItem@@UAEXH@Z 100053ca f   qt-mt323:qt-mt323.dll
 0001:000043d0       ?styleChange@QPopupMenu@@MAEXAAVQStyle@@@Z 100053d0 f   qt-mt323:qt-mt323.dll
 0001:000043d6       ?styleChange@QToolBar@@MAEXAAVQStyle@@@Z 100053d6 f   qt-mt323:qt-mt323.dll
 0001:000043dc       ?styleChange@QWidget@@MAEXAAVQStyle@@@Z 100053dc f   qt-mt323:qt-mt323.dll
 0001:000043e2       ?tabletEvent@QWidget@@MAEXPAVQTabletEvent@@@Z 100053e2 f   qt-mt323:qt-mt323.dll
 0001:000043e8       ?takeItem@QListViewItem@@UAEXPAV1@@Z 100053e8 f   qt-mt323:qt-mt323.dll
 0001:000043ee       ?text@QListViewItem@@UBE?AVQString@@H@Z 100053ee f   qt-mt323:qt-mt323.dll
 0001:000043f4       ?timerEvent@QObject@@MAEXPAVQTimerEvent@@@Z 100053f4 f   qt-mt323:qt-mt323.dll
 0001:000043fa       ?timerEvent@QPopupMenu@@MAEXPAVQTimerEvent@@@Z 100053fa f   qt-mt323:qt-mt323.dll
 0001:00004400       ?undock@QDockWindow@@UAEXPAVQWidget@@@Z 10005400 f   qt-mt323:qt-mt323.dll
 0001:00004406       ?undock@QDockWindow@@UAEXXZ 10005406 f   qt-mt323:qt-mt323.dll
 0001:0000440c       ?unsetCursor@QWidget@@UAEXXZ 1000540c f   qt-mt323:qt-mt323.dll
 0001:00004412       ?updateItem@QPopupMenu@@UAEXH@Z 10005412 f   qt-mt323:qt-mt323.dll
 0001:00004418       ?updateMask@QWidget@@MAEXXZ 10005418 f   qt-mt323:qt-mt323.dll
 0001:0000441e       ?wheelEvent@QWidget@@MAEXPAVQWheelEvent@@@Z 1000541e f   qt-mt323:qt-mt323.dll
 0001:00004424       ?width@QListViewItem@@UBEHABVQFontMetrics@@PBVQListView@@H@Z 10005424 f   qt-mt323:qt-mt323.dll
 0001:0000442a       ?winEvent@QWidget@@MAE_NPAUtagMSG@@@Z 1000542a f   qt-mt323:qt-mt323.dll
 0001:00004430       ?windowActivationChange@QWidget@@MAEX_N@Z 10005430 f   qt-mt323:qt-mt323.dll
 0001:00004436       ?write@QGDict@@MBEAAVQDataStream@@AAV2@PAX@Z 10005436 f   qt-mt323:qt-mt323.dll
 0001:0000443c       ?write@QGList@@MBEAAVQDataStream@@AAV2@PAX@Z 1000543c f   qt-mt323:qt-mt323.dll
 0001:00004442       ?addChild@QScrollView@@UAEXPAVQWidget@@HH@Z 10005442 f   qt-mt323:qt-mt323.dll
 0001:00004448       ?addColumn@QListView@@UAEHABVQIconSet@@ABVQString@@H@Z 10005448 f   qt-mt323:qt-mt323.dll
 0001:0000444e       ?addColumn@QListView@@UAEHABVQString@@H@Z 1000544e f   qt-mt323:qt-mt323.dll
 0001:00004454       ?addItem@QBoxLayout@@UAEXPAVQLayoutItem@@@Z 10005454 f   qt-mt323:qt-mt323.dll
 0001:0000445a       ?childEvent@QGroupBox@@MAEXPAVQChildEvent@@@Z 1000545a f   qt-mt323:qt-mt323.dll
 0001:00004460       ?childEvent@QLayout@@MAEXPAVQChildEvent@@@Z 10005460 f   qt-mt323:qt-mt323.dll
 0001:00004466       ?className@QButtonGroup@@UBEPBDXZ 10005466 f   qt-mt323:qt-mt323.dll
 0001:0000446c       ?className@QHBoxLayout@@UBEPBDXZ 1000546c f   qt-mt323:qt-mt323.dll
 0001:00004472       ?className@QLabel@@UBEPBDXZ 10005472 f   qt-mt323:qt-mt323.dll
 0001:00004478       ?className@QListView@@UBEPBDXZ 10005478 f   qt-mt323:qt-mt323.dll
 0001:0000447e       ?className@QPushButton@@UBEPBDXZ 1000547e f   qt-mt323:qt-mt323.dll
 0001:00004484       ?className@QVBoxLayout@@UBEPBDXZ 10005484 f   qt-mt323:qt-mt323.dll
 0001:0000448a       ?clear@QListView@@UAEXXZ   1000548a f   qt-mt323:qt-mt323.dll
 0001:00004490       ?clearSelection@QListView@@UAEXXZ 10005490 f   qt-mt323:qt-mt323.dll
 0001:00004496       ?contentsContextMenuEvent@QListView@@MAEXPAVQContextMenuEvent@@@Z 10005496 f   qt-mt323:qt-mt323.dll
 0001:0000449c       ?contentsDragEnterEvent@QListView@@MAEXPAVQDragEnterEvent@@@Z 1000549c f   qt-mt323:qt-mt323.dll
 0001:000044a2       ?contentsDragLeaveEvent@QListView@@MAEXPAVQDragLeaveEvent@@@Z 100054a2 f   qt-mt323:qt-mt323.dll
 0001:000044a8       ?contentsDragMoveEvent@QListView@@MAEXPAVQDragMoveEvent@@@Z 100054a8 f   qt-mt323:qt-mt323.dll
 0001:000044ae       ?contentsDropEvent@QListView@@MAEXPAVQDropEvent@@@Z 100054ae f   qt-mt323:qt-mt323.dll
 0001:000044b4       ?contentsMouseDoubleClickEvent@QListView@@MAEXPAVQMouseEvent@@@Z 100054b4 f   qt-mt323:qt-mt323.dll
 0001:000044ba       ?contentsMouseMoveEvent@QListView@@MAEXPAVQMouseEvent@@@Z 100054ba f   qt-mt323:qt-mt323.dll
 0001:000044c0       ?contentsMousePressEvent@QListView@@MAEXPAVQMouseEvent@@@Z 100054c0 f   qt-mt323:qt-mt323.dll
 0001:000044c6       ?contentsMouseReleaseEvent@QListView@@MAEXPAVQMouseEvent@@@Z 100054c6 f   qt-mt323:qt-mt323.dll
 0001:000044cc       ?contentsWheelEvent@QScrollView@@MAEXPAVQWheelEvent@@@Z 100054cc f   qt-mt323:qt-mt323.dll
 0001:000044d2       ?contextMenuEvent@QScrollView@@MAEXPAVQContextMenuEvent@@@Z 100054d2 f   qt-mt323:qt-mt323.dll
 0001:000044d8       ?dragObject@QListView@@MAEPAVQDragObject@@XZ 100054d8 f   qt-mt323:qt-mt323.dll
 0001:000044de       ?drawButton@QPushButton@@MAEXPAVQPainter@@@Z 100054de f   qt-mt323:qt-mt323.dll
 0001:000044e4       ?drawButtonLabel@QPushButton@@MAEXPAVQPainter@@@Z 100054e4 f   qt-mt323:qt-mt323.dll
 0001:000044ea       ?drawContents@QFrame@@MAEXPAVQPainter@@@Z 100054ea f   qt-mt323:qt-mt323.dll
 0001:000044f0       ?drawContents@QLabel@@MAEXPAVQPainter@@@Z 100054f0 f   qt-mt323:qt-mt323.dll
 0001:000044f6       ?drawContents@QScrollView@@EAEXPAVQPainter@@@Z 100054f6 f   qt-mt323:qt-mt323.dll
 0001:000044fc       ?drawContents@QScrollView@@MAEXPAVQPainter@@HHHH@Z 100054fc f   qt-mt323:qt-mt323.dll
 0001:00004502       ?drawContentsOffset@QListView@@MAEXPAVQPainter@@HHHHHH@Z 10005502 f   qt-mt323:qt-mt323.dll
 0001:00004508       ?enabledChange@QButton@@MAEX_N@Z 10005508 f   qt-mt323:qt-mt323.dll
 0001:0000450e       ?event@QButtonGroup@@MAE_NPAVQEvent@@@Z 1000550e f   qt-mt323:qt-mt323.dll
 0001:00004514       ?eventFilter@QLayout@@MAE_NPAVQObject@@PAVQEvent@@@Z 10005514 f   qt-mt323:qt-mt323.dll
 0001:0000451a       ?eventFilter@QListView@@UAE_NPAVQObject@@PAVQEvent@@@Z 1000551a f   qt-mt323:qt-mt323.dll
 0001:00004520       ?expanding@QBoxLayout@@UBE?AW4ExpandData@QSizePolicy@@XZ 10005520 f   qt-mt323:qt-mt323.dll
 0001:00004526       ?expanding@QSpacerItem@@UBE?AW4ExpandData@QSizePolicy@@XZ 10005526 f   qt-mt323:qt-mt323.dll
 0001:0000452c       ?focusInEvent@QGroupBox@@MAEXPAVQFocusEvent@@@Z 1000552c f   qt-mt323:qt-mt323.dll
 0001:00004532       ?focusInEvent@QListView@@MAEXPAVQFocusEvent@@@Z 10005532 f   qt-mt323:qt-mt323.dll
 0001:00004538       ?focusInEvent@QPushButton@@MAEXPAVQFocusEvent@@@Z 10005538 f   qt-mt323:qt-mt323.dll
 0001:0000453e       ?focusNextPrevChild@QScrollView@@MAE_N_N@Z 1000553e f   qt-mt323:qt-mt323.dll
 0001:00004544       ?focusOutEvent@QListView@@MAEXPAVQFocusEvent@@@Z 10005544 f   qt-mt323:qt-mt323.dll
 0001:0000454a       ?focusOutEvent@QPushButton@@MAEXPAVQFocusEvent@@@Z 1000554a f   qt-mt323:qt-mt323.dll
 0001:00004550       ?fontChange@QGroupBox@@MAEXABVQFont@@@Z 10005550 f   qt-mt323:qt-mt323.dll
 0001:00004556       ?fontChange@QLabel@@MAEXABVQFont@@@Z 10005556 f   qt-mt323:qt-mt323.dll
 0001:0000455c       ?fontChange@QScrollView@@MAEXABVQFont@@@Z 1000555c f   qt-mt323:qt-mt323.dll
 0001:00004562       ?frameChanged@QHBox@@MAEXXZ 10005562 f   qt-mt323:qt-mt323.dll
 0001:00004568       ?frameChanged@QScrollView@@MAEXXZ 10005568 f   qt-mt323:qt-mt323.dll
 0001:0000456e       ?geometry@QLayout@@UBE?AVQRect@@XZ 1000556e f   qt-mt323:qt-mt323.dll
 0001:00004574       ?geometry@QSpacerItem@@UBE?AVQRect@@XZ 10005574 f   qt-mt323:qt-mt323.dll
 0001:0000457a       ?hasHeightForWidth@QBoxLayout@@UBE_NXZ 1000557a f   qt-mt323:qt-mt323.dll
 0001:00004580       ?hasHeightForWidth@QLayoutItem@@UBE_NXZ 10005580 f   qt-mt323:qt-mt323.dll
 0001:00004586       ?heightForWidth@QBoxLayout@@UBEHH@Z 10005586 f   qt-mt323:qt-mt323.dll
 0001:0000458c       ?heightForWidth@QLabel@@UBEHH@Z 1000558c f   qt-mt323:qt-mt323.dll
 0001:00004592       ?heightForWidth@QLayoutItem@@UBEHH@Z 10005592 f   qt-mt323:qt-mt323.dll
 0001:00004598       ?hitButton@QButton@@MBE_NABVQPoint@@@Z 10005598 f   qt-mt323:qt-mt323.dll
 0001:0000459e       ?insertItem@QListView@@UAEXPAVQListViewItem@@@Z 1000559e f   qt-mt323:qt-mt323.dll
 0001:000045a4       ?invalidate@QBoxLayout@@UAEXXZ 100055a4 f   qt-mt323:qt-mt323.dll
 0001:000045aa       ?invalidate@QLayoutItem@@UAEXXZ 100055aa f   qt-mt323:qt-mt323.dll
 0001:000045b0       ?invertSelection@QListView@@UAEXXZ 100055b0 f   qt-mt323:qt-mt323.dll
 0001:000045b6       ?isEmpty@QLayout@@UBE_NXZ  100055b6 f   qt-mt323:qt-mt323.dll
 0001:000045bc       ?isEmpty@QSpacerItem@@UBE_NXZ 100055bc f   qt-mt323:qt-mt323.dll
 0001:000045c2       ?iterator@QBoxLayout@@UAE?AVQLayoutIterator@@XZ 100055c2 f   qt-mt323:qt-mt323.dll
 0001:000045c8       ?iterator@QLayoutItem@@UAE?AVQLayoutIterator@@XZ 100055c8 f   qt-mt323:qt-mt323.dll
 0001:000045ce       ?keyPressEvent@QButton@@MAEXPAVQKeyEvent@@@Z 100055ce f   qt-mt323:qt-mt323.dll
 0001:000045d4       ?keyPressEvent@QListView@@MAEXPAVQKeyEvent@@@Z 100055d4 f   qt-mt323:qt-mt323.dll
 0001:000045da       ?keyReleaseEvent@QButton@@MAEXPAVQKeyEvent@@@Z 100055da f   qt-mt323:qt-mt323.dll
 0001:000045e0       ?layout@QLayout@@UAEPAV1@XZ 100055e0 f   qt-mt323:qt-mt323.dll
 0001:000045e6       ?layout@QLayoutItem@@UAEPAVQLayout@@XZ 100055e6 f   qt-mt323:qt-mt323.dll
 0001:000045ec       ?maximumSize@QBoxLayout@@UBE?AVQSize@@XZ 100055ec f   qt-mt323:qt-mt323.dll
 0001:000045f2       ?maximumSize@QSpacerItem@@UBE?AVQSize@@XZ 100055f2 f   qt-mt323:qt-mt323.dll
 0001:000045f8       ?metaObject@QButtonGroup@@UBEPAVQMetaObject@@XZ 100055f8 f   qt-mt323:qt-mt323.dll
 0001:000045fe       ?metaObject@QHBoxLayout@@UBEPAVQMetaObject@@XZ 100055fe f   qt-mt323:qt-mt323.dll
 0001:00004604       ?metaObject@QLabel@@UBEPAVQMetaObject@@XZ 10005604 f   qt-mt323:qt-mt323.dll
 0001:0000460a       ?metaObject@QListView@@UBEPAVQMetaObject@@XZ 1000560a f   qt-mt323:qt-mt323.dll
 0001:00004610       ?metaObject@QPushButton@@UBEPAVQMetaObject@@XZ 10005610 f   qt-mt323:qt-mt323.dll
 0001:00004616       ?metaObject@QVBoxLayout@@UBEPAVQMetaObject@@XZ 10005616 f   qt-mt323:qt-mt323.dll
 0001:0000461c       ?minimumSize@QBoxLayout@@UBE?AVQSize@@XZ 1000561c f   qt-mt323:qt-mt323.dll
 0001:00004622       ?minimumSize@QSpacerItem@@UBE?AVQSize@@XZ 10005622 f   qt-mt323:qt-mt323.dll
 0001:00004628       ?minimumSizeHint@QLabel@@UBE?AVQSize@@XZ 10005628 f   qt-mt323:qt-mt323.dll
 0001:0000462e       ?minimumSizeHint@QListView@@UBE?AVQSize@@XZ 1000562e f   qt-mt323:qt-mt323.dll
 0001:00004634       ?mouseDoubleClickEvent@QScrollView@@MAEXPAVQMouseEvent@@@Z 10005634 f   qt-mt323:qt-mt323.dll
 0001:0000463a       ?mouseMoveEvent@QButton@@MAEXPAVQMouseEvent@@@Z 1000563a f   qt-mt323:qt-mt323.dll
 0001:00004640       ?mouseMoveEvent@QScrollView@@MAEXPAVQMouseEvent@@@Z 10005640 f   qt-mt323:qt-mt323.dll
 0001:00004646       ?mousePressEvent@QButton@@MAEXPAVQMouseEvent@@@Z 10005646 f   qt-mt323:qt-mt323.dll
 0001:0000464c       ?mousePressEvent@QScrollView@@MAEXPAVQMouseEvent@@@Z 1000564c f   qt-mt323:qt-mt323.dll
 0001:00004652       ?mouseReleaseEvent@QButton@@MAEXPAVQMouseEvent@@@Z 10005652 f   qt-mt323:qt-mt323.dll
 0001:00004658       ?mouseReleaseEvent@QScrollView@@MAEXPAVQMouseEvent@@@Z 10005658 f   qt-mt323:qt-mt323.dll
 0001:0000465e       ?move@QPushButton@@UAEXHH@Z 1000565e f   qt-mt323:qt-mt323.dll
 0001:00004664       ?moveChild@QScrollView@@UAEXPAVQWidget@@HH@Z 10005664 f   qt-mt323:qt-mt323.dll
 0001:0000466a       ?moveFocus@QButtonGroup@@UAEXH@Z 1000566a f   qt-mt323:qt-mt323.dll
 0001:00004670       ?paintEmptyArea@QListView@@MAEXPAVQPainter@@ABVQRect@@@Z 10005670 f   qt-mt323:qt-mt323.dll
 0001:00004676       ?paintEvent@QButton@@MAEXPAVQPaintEvent@@@Z 10005676 f   qt-mt323:qt-mt323.dll
 0001:0000467c       ?paintEvent@QGroupBox@@MAEXPAVQPaintEvent@@@Z 1000567c f   qt-mt323:qt-mt323.dll
 0001:00004682       ?qt_cast@QButtonGroup@@UAEPAXPBD@Z 10005682 f   qt-mt323:qt-mt323.dll
 0001:00004688       ?qt_cast@QHBoxLayout@@UAEPAXPBD@Z 10005688 f   qt-mt323:qt-mt323.dll
 0001:0000468e       ?qt_cast@QLabel@@UAEPAXPBD@Z 1000568e f   qt-mt323:qt-mt323.dll
 0001:00004694       ?qt_cast@QListView@@UAEPAXPBD@Z 10005694 f   qt-mt323:qt-mt323.dll
 0001:0000469a       ?qt_cast@QPushButton@@UAEPAXPBD@Z 1000569a f   qt-mt323:qt-mt323.dll
 0001:000046a0       ?qt_cast@QVBoxLayout@@UAEPAXPBD@Z 100056a0 f   qt-mt323:qt-mt323.dll
 0001:000046a6       ?qt_emit@QButtonGroup@@UAE_NHPAUQUObject@@@Z 100056a6 f   qt-mt323:qt-mt323.dll
 0001:000046ac       ?qt_emit@QHBoxLayout@@UAE_NHPAUQUObject@@@Z 100056ac f   qt-mt323:qt-mt323.dll
 0001:000046b2       ?qt_emit@QLabel@@UAE_NHPAUQUObject@@@Z 100056b2 f   qt-mt323:qt-mt323.dll
 0001:000046b8       ?qt_emit@QListView@@UAE_NHPAUQUObject@@@Z 100056b8 f   qt-mt323:qt-mt323.dll
 0001:000046be       ?qt_emit@QPushButton@@UAE_NHPAUQUObject@@@Z 100056be f   qt-mt323:qt-mt323.dll
 0001:000046c4       ?qt_emit@QVBoxLayout@@UAE_NHPAUQUObject@@@Z 100056c4 f   qt-mt323:qt-mt323.dll
 0001:000046ca       ?qt_invoke@QButtonGroup@@UAE_NHPAUQUObject@@@Z 100056ca f   qt-mt323:qt-mt323.dll
 0001:000046d0       ?qt_invoke@QHBoxLayout@@UAE_NHPAUQUObject@@@Z 100056d0 f   qt-mt323:qt-mt323.dll
 0001:000046d6       ?qt_invoke@QLabel@@UAE_NHPAUQUObject@@@Z 100056d6 f   qt-mt323:qt-mt323.dll
 0001:000046dc       ?qt_invoke@QListView@@UAE_NHPAUQUObject@@@Z 100056dc f   qt-mt323:qt-mt323.dll
 0001:000046e2       ?qt_invoke@QPushButton@@UAE_NHPAUQUObject@@@Z 100056e2 f   qt-mt323:qt-mt323.dll
 0001:000046e8       ?qt_invoke@QVBoxLayout@@UAE_NHPAUQUObject@@@Z 100056e8 f   qt-mt323:qt-mt323.dll
 0001:000046ee       ?qt_property@QButtonGroup@@UAE_NHHPAVQVariant@@@Z 100056ee f   qt-mt323:qt-mt323.dll
 0001:000046f4       ?qt_property@QHBoxLayout@@UAE_NHHPAVQVariant@@@Z 100056f4 f   qt-mt323:qt-mt323.dll
 0001:000046fa       ?qt_property@QLabel@@UAE_NHHPAVQVariant@@@Z 100056fa f   qt-mt323:qt-mt323.dll
 0001:00004700       ?qt_property@QListView@@UAE_NHHPAVQVariant@@@Z 10005700 f   qt-mt323:qt-mt323.dll
 0001:00004706       ?qt_property@QPushButton@@UAE_NHHPAVQVariant@@@Z 10005706 f   qt-mt323:qt-mt323.dll
 0001:0000470c       ?qt_property@QVBoxLayout@@UAE_NHHPAVQVariant@@@Z 1000570c f   qt-mt323:qt-mt323.dll
 0001:00004712       ?removeChild@QScrollView@@UAEXPAVQObject@@@Z 10005712 f   qt-mt323:qt-mt323.dll
 0001:00004718       ?removeColumn@QListView@@UAEXH@Z 10005718 f   qt-mt323:qt-mt323.dll
 0001:0000471e       ?removeItem@QListView@@UAEXPAVQListViewItem@@@Z 1000571e f   qt-mt323:qt-mt323.dll
 0001:00004724       ?resize@QPushButton@@UAEXHH@Z 10005724 f   qt-mt323:qt-mt323.dll
 0001:0000472a       ?resize@QScrollView@@UAEXHH@Z 1000572a f   qt-mt323:qt-mt323.dll
 0001:00004730       ?resizeContents@QScrollView@@UAEXHH@Z 10005730 f   qt-mt323:qt-mt323.dll
 0001:00004736       ?resizeEvent@QGroupBox@@MAEXPAVQResizeEvent@@@Z 10005736 f   qt-mt323:qt-mt323.dll
 0001:0000473c       ?resizeEvent@QLabel@@MAEXPAVQResizeEvent@@@Z 1000573c f   qt-mt323:qt-mt323.dll
 0001:00004742       ?resizeEvent@QListView@@MAEXPAVQResizeEvent@@@Z 10005742 f   qt-mt323:qt-mt323.dll
 0001:00004748       ?resizeEvent@QPushButton@@MAEXPAVQResizeEvent@@@Z 10005748 f   qt-mt323:qt-mt323.dll
 0001:0000474e       ?selectAll@QListView@@UAEX_N@Z 1000574e f   qt-mt323:qt-mt323.dll
 0001:00004754       ?setAccel@QButton@@UAEXABVQKeySequence@@@Z 10005754 f   qt-mt323:qt-mt323.dll
 0001:0000475a       ?setAlignment@QGroupBox@@UAEXH@Z 1000575a f   qt-mt323:qt-mt323.dll
 0001:00004760       ?setAlignment@QLabel@@UAEXH@Z 10005760 f   qt-mt323:qt-mt323.dll
 0001:00004766       ?setAlignment@QLayoutItem@@UAEXH@Z 10005766 f   qt-mt323:qt-mt323.dll
 0001:0000476c       ?setAllColumnsShowFocus@QListView@@UAEX_N@Z 1000576c f   qt-mt323:qt-mt323.dll
 0001:00004772       ?setAutoAdd@QLayout@@UAEX_N@Z 10005772 f   qt-mt323:qt-mt323.dll
 0001:00004778       ?setAutoDefault@QPushButton@@UAEX_N@Z 10005778 f   qt-mt323:qt-mt323.dll
 0001:0000477e       ?setAutoRepeat@QButton@@UAEX_N@Z 1000577e f   qt-mt323:qt-mt323.dll
 0001:00004784       ?setAutoResize@QLabel@@UAEX_N@Z 10005784 f   qt-mt323:qt-mt323.dll
 0001:0000478a       ?setBuddy@QLabel@@UAEXPAVQWidget@@@Z 1000578a f   qt-mt323:qt-mt323.dll
 0001:00004790       ?setButton@QButtonGroup@@UAEXH@Z 10005790 f   qt-mt323:qt-mt323.dll
 0001:00004796       ?setColumnAlignment@QListView@@UAEXHH@Z 10005796 f   qt-mt323:qt-mt323.dll
 0001:0000479c       ?setColumnLayout@QGroupBox@@UAEXHW4Orientation@Qt@@@Z 1000579c f   qt-mt323:qt-mt323.dll
 0001:000047a2       ?setColumnText@QListView@@UAEXHABVQIconSet@@ABVQString@@@Z 100057a2 f   qt-mt323:qt-mt323.dll
 0001:000047a8       ?setColumnText@QListView@@UAEXHABVQString@@@Z 100057a8 f   qt-mt323:qt-mt323.dll
 0001:000047ae       ?setColumnWidth@QListView@@UAEXHH@Z 100057ae f   qt-mt323:qt-mt323.dll
 0001:000047b4       ?setColumnWidthMode@QListView@@UAEXHW4WidthMode@1@@Z 100057b4 f   qt-mt323:qt-mt323.dll
 0001:000047ba       ?setContentsPos@QListView@@UAEXHH@Z 100057ba f   qt-mt323:qt-mt323.dll
 0001:000047c0       ?setCornerWidget@QScrollView@@UAEXPAVQWidget@@@Z 100057c0 f   qt-mt323:qt-mt323.dll
 0001:000047c6       ?setCurrentItem@QListView@@UAEXPAVQListViewItem@@@Z 100057c6 f   qt-mt323:qt-mt323.dll
 0001:000047cc       ?setDefault@QPushButton@@UAEX_N@Z 100057cc f   qt-mt323:qt-mt323.dll
 0001:000047d2       ?setDefaultRenameAction@QListView@@UAEXW4RenameAction@1@@Z 100057d2 f   qt-mt323:qt-mt323.dll
 0001:000047d8       ?setDown@QButton@@UAEX_N@Z 100057d8 f   qt-mt323:qt-mt323.dll
 0001:000047de       ?setDragAutoScroll@QScrollView@@UAEX_N@Z 100057de f   qt-mt323:qt-mt323.dll
 0001:000047e4       ?setEnabled@QGroupBox@@UAEX_N@Z 100057e4 f   qt-mt323:qt-mt323.dll
 0001:000047ea       ?setEnabled@QScrollView@@UAEX_N@Z 100057ea f   qt-mt323:qt-mt323.dll
 0001:000047f0       ?setExclusive@QButtonGroup@@UAEX_N@Z 100057f0 f   qt-mt323:qt-mt323.dll
 0001:000047f6       ?setFont@QLabel@@UAEXABVQFont@@@Z 100057f6 f   qt-mt323:qt-mt323.dll
 0001:000047fc       ?setFont@QListView@@UAEXABVQFont@@@Z 100057fc f   qt-mt323:qt-mt323.dll
 0001:00004802       ?setGeometry@QBoxLayout@@UAEXABVQRect@@@Z 10005802 f   qt-mt323:qt-mt323.dll
 0001:00004808       ?setGeometry@QPushButton@@UAEXABVQRect@@@Z 10005808 f   qt-mt323:qt-mt323.dll
 0001:0000480e       ?setGeometry@QPushButton@@UAEXHHHH@Z 1000580e f   qt-mt323:qt-mt323.dll
 0001:00004814       ?setGeometry@QSpacerItem@@UAEXABVQRect@@@Z 10005814 f   qt-mt323:qt-mt323.dll
 0001:0000481a       ?setGroup@QButton@@EAEXPAVQButtonGroup@@@Z 1000581a f   qt-mt323:qt-mt323.dll
 0001:00004820       ?setHBarGeometry@QScrollView@@MAEXAAVQScrollBar@@HHHH@Z 10005820 f   qt-mt323:qt-mt323.dll
 0001:00004826       ?setHScrollBarMode@QScrollView@@UAEXW4ScrollBarMode@1@@Z 10005826 f   qt-mt323:qt-mt323.dll
 0001:0000482c       ?setIsMenuButton@QPushButton@@UAEX_N@Z 1000582c f   qt-mt323:qt-mt323.dll
 0001:00004832       ?setItemMargin@QListView@@UAEXH@Z 10005832 f   qt-mt323:qt-mt323.dll
 0001:00004838       ?setMargin@QLayout@@UAEXH@Z 10005838 f   qt-mt323:qt-mt323.dll
 0001:0000483e       ?setMargins@QScrollView@@MAEXHHHH@Z 1000583e f   qt-mt323:qt-mt323.dll
 0001:00004844       ?setMenuBar@QLayout@@UAEXPAVQMenuBar@@@Z 10005844 f   qt-mt323:qt-mt323.dll
 0001:0000484a       ?setMovie@QLabel@@UAEXABVQMovie@@@Z 1000584a f   qt-mt323:qt-mt323.dll
 0001:00004850       ?setMultiSelection@QListView@@UAEX_N@Z 10005850 f   qt-mt323:qt-mt323.dll
 0001:00004856       ?setNum@QLabel@@UAEXH@Z    10005856 f   qt-mt323:qt-mt323.dll
 0001:0000485c       ?setNum@QLabel@@UAEXN@Z    1000585c f   qt-mt323:qt-mt323.dll
 0001:00004862       ?setOn@QPushButton@@UAEX_N@Z 10005862 f   qt-mt323:qt-mt323.dll
 0001:00004868       ?setOpen@QListView@@UAEXPAVQListViewItem@@_N@Z 10005868 f   qt-mt323:qt-mt323.dll
 0001:0000486e       ?setPalette@QListView@@UAEXABVQPalette@@@Z 1000586e f   qt-mt323:qt-mt323.dll
 0001:00004874       ?setPicture@QLabel@@UAEXABVQPicture@@@Z 10005874 f   qt-mt323:qt-mt323.dll
 0001:0000487a       ?setPixmap@QButton@@UAEXABVQPixmap@@@Z 1000587a f   qt-mt323:qt-mt323.dll
 0001:00004880       ?setPixmap@QLabel@@UAEXABVQPixmap@@@Z 10005880 f   qt-mt323:qt-mt323.dll
 0001:00004886       ?setRadioButtonExclusive@QButtonGroup@@UAEX_N@Z 10005886 f   qt-mt323:qt-mt323.dll
 0001:0000488c       ?setResizeMode@QListView@@UAEXW4ResizeMode@1@@Z 1000588c f   qt-mt323:qt-mt323.dll
 0001:00004892       ?setResizePolicy@QScrollView@@UAEXW4ResizePolicy@1@@Z 10005892 f   qt-mt323:qt-mt323.dll
 0001:00004898       ?setRootIsDecorated@QListView@@UAEX_N@Z 10005898 f   qt-mt323:qt-mt323.dll
 0001:0000489e       ?setSelected@QListView@@UAEXPAVQListViewItem@@_N@Z 1000589e f   qt-mt323:qt-mt323.dll
 0001:000048a4       ?setShowSortIndicator@QListView@@UAEX_N@Z 100058a4 f   qt-mt323:qt-mt323.dll
 0001:000048aa       ?setShowToolTips@QListView@@UAEX_N@Z 100058aa f   qt-mt323:qt-mt323.dll
 0001:000048b0       ?setSorting@QListView@@UAEXH_N@Z 100058b0 f   qt-mt323:qt-mt323.dll
 0001:000048b6       ?setSpacing@QLayout@@UAEXH@Z 100058b6 f   qt-mt323:qt-mt323.dll
 0001:000048bc       ?setState@QButton@@MAEXW4ToggleState@1@@Z 100058bc f   qt-mt323:qt-mt323.dll
 0001:000048c2       ?setText@QButton@@UAEXABVQString@@@Z 100058c2 f   qt-mt323:qt-mt323.dll
 0001:000048c8       ?setText@QLabel@@UAEXABVQString@@@Z 100058c8 f   qt-mt323:qt-mt323.dll
 0001:000048ce       ?setTitle@QGroupBox@@UAEXABVQString@@@Z 100058ce f   qt-mt323:qt-mt323.dll
 0001:000048d4       ?setToggleType@QButton@@MAEXW4ToggleType@1@@Z 100058d4 f   qt-mt323:qt-mt323.dll
 0001:000048da       ?setTreeStepSize@QListView@@UAEXH@Z 100058da f   qt-mt323:qt-mt323.dll
 0001:000048e0       ?setVBarGeometry@QScrollView@@MAEXAAVQScrollBar@@HHHH@Z 100058e0 f   qt-mt323:qt-mt323.dll
 0001:000048e6       ?setVScrollBarMode@QScrollView@@UAEXW4ScrollBarMode@1@@Z 100058e6 f   qt-mt323:qt-mt323.dll
 0001:000048ec       ?show@QListView@@UAEXXZ    100058ec f   qt-mt323:qt-mt323.dll
 0001:000048f2       ?showEvent@QListView@@MAEXPAVQShowEvent@@@Z 100058f2 f   qt-mt323:qt-mt323.dll
 0001:000048f8       ?sizeHint@QBoxLayout@@UBE?AVQSize@@XZ 100058f8 f   qt-mt323:qt-mt323.dll
 0001:000048fe       ?sizeHint@QGroupBox@@UBE?AVQSize@@XZ 100058fe f   qt-mt323:qt-mt323.dll
 0001:00004904       ?sizeHint@QHBox@@UBE?AVQSize@@XZ 10005904 f   qt-mt323:qt-mt323.dll
 0001:0000490a       ?sizeHint@QLabel@@UBE?AVQSize@@XZ 1000590a f   qt-mt323:qt-mt323.dll
 0001:00004910       ?sizeHint@QListView@@UBE?AVQSize@@XZ 10005910 f   qt-mt323:qt-mt323.dll
 0001:00004916       ?sizeHint@QPushButton@@UBE?AVQSize@@XZ 10005916 f   qt-mt323:qt-mt323.dll
 0001:0000491c       ?sizeHint@QSpacerItem@@UBE?AVQSize@@XZ 1000591c f   qt-mt323:qt-mt323.dll
 0001:00004922       ?sort@QListView@@UAEXXZ    10005922 f   qt-mt323:qt-mt323.dll
 0001:00004928       ?spacerItem@QLayoutItem@@UAEPAVQSpacerItem@@XZ 10005928 f   qt-mt323:qt-mt323.dll
 0001:0000492e       ?spacerItem@QSpacerItem@@UAEPAV1@XZ 1000592e f   qt-mt323:qt-mt323.dll
 0001:00004934       ?startDrag@QListView@@MAEXXZ 10005934 f   qt-mt323:qt-mt323.dll
 0001:0000493a       ?styleChange@QFrame@@MAEXAAVQStyle@@@Z 1000593a f   qt-mt323:qt-mt323.dll
 0001:00004940       ?styleChange@QListView@@MAEXAAVQStyle@@@Z 10005940 f   qt-mt323:qt-mt323.dll
 0001:00004946       ?takeItem@QListView@@UAEXPAVQListViewItem@@@Z 10005946 f   qt-mt323:qt-mt323.dll
 0001:0000494c       ?updateMask@QPushButton@@MAEXXZ 1000594c f   qt-mt323:qt-mt323.dll
 0001:00004952       ?viewportContextMenuEvent@QScrollView@@MAEXPAVQContextMenuEvent@@@Z 10005952 f   qt-mt323:qt-mt323.dll
 0001:00004958       ?viewportDragEnterEvent@QScrollView@@MAEXPAVQDragEnterEvent@@@Z 10005958 f   qt-mt323:qt-mt323.dll
 0001:0000495e       ?viewportDragLeaveEvent@QScrollView@@MAEXPAVQDragLeaveEvent@@@Z 1000595e f   qt-mt323:qt-mt323.dll
 0001:00004964       ?viewportDragMoveEvent@QScrollView@@MAEXPAVQDragMoveEvent@@@Z 10005964 f   qt-mt323:qt-mt323.dll
 0001:0000496a       ?viewportDropEvent@QScrollView@@MAEXPAVQDropEvent@@@Z 1000596a f   qt-mt323:qt-mt323.dll
 0001:00004970       ?viewportMouseDoubleClickEvent@QScrollView@@MAEXPAVQMouseEvent@@@Z 10005970 f   qt-mt323:qt-mt323.dll
 0001:00004976       ?viewportMouseMoveEvent@QScrollView@@MAEXPAVQMouseEvent@@@Z 10005976 f   qt-mt323:qt-mt323.dll
 0001:0000497c       ?viewportMousePressEvent@QScrollView@@MAEXPAVQMouseEvent@@@Z 1000597c f   qt-mt323:qt-mt323.dll
 0001:00004982       ?viewportMouseReleaseEvent@QScrollView@@MAEXPAVQMouseEvent@@@Z 10005982 f   qt-mt323:qt-mt323.dll
 0001:00004988       ?viewportPaintEvent@QScrollView@@MAEXPAVQPaintEvent@@@Z 10005988 f   qt-mt323:qt-mt323.dll
 0001:0000498e       ?viewportResizeEvent@QListView@@MAEXPAVQResizeEvent@@@Z 1000598e f   qt-mt323:qt-mt323.dll
 0001:00004994       ?viewportWheelEvent@QScrollView@@MAEXPAVQWheelEvent@@@Z 10005994 f   qt-mt323:qt-mt323.dll
 0001:0000499a       ?wheelEvent@QScrollView@@MAEXPAVQWheelEvent@@@Z 1000599a f   qt-mt323:qt-mt323.dll
 0001:000049a0       ?widget@QLayoutItem@@UAEPAVQWidget@@XZ 100059a0 f   qt-mt323:qt-mt323.dll
 0001:000049a6       ?windowActivationChange@QListView@@MAEX_N@Z 100059a6 f   qt-mt323:qt-mt323.dll
 0001:000049ac       ?className@CAlm_sys_select@@UBEPBDXZ 100059ac f   alm_sys_select:alm_sys_select.dll
 0001:000049b2       ?metaObject@CAlm_sys_select@@UBEPAVQMetaObject@@XZ 100059b2 f   alm_sys_select:alm_sys_select.dll
 0001:000049b8       ?qt_cast@CAlm_sys_select@@UAEPAXPBD@Z 100059b8 f   alm_sys_select:alm_sys_select.dll
 0001:000049be       ?qt_emit@CAlm_sys_select@@UAE_NHPAUQUObject@@@Z 100059be f   alm_sys_select:alm_sys_select.dll
 0001:000049c4       ?qt_invoke@CAlm_sys_select@@UAE_NHPAUQUObject@@@Z 100059c4 f   alm_sys_select:alm_sys_select.dll
 0001:000049ca       ?qt_property@CAlm_sys_select@@UAE_NHHPAVQVariant@@@Z 100059ca f   alm_sys_select:alm_sys_select.dll
 0001:000049d0       ??2@YAPAXI@Z               100059d0 f   MSVCRT:MSVCR120.dll
 0001:000049d6       ??3@YAXPAX@Z               100059d6 f   MSVCRT:MSVCR120.dll
 0001:000049dc       @__security_check_cookie@4 100059dc f   MSVCRT:secchk.obj
 0001:000049eb       __EH_epilog3               100059eb f   MSVCRT:ehprolg3.obj
 0001:000049ff       __EH_epilog3_GS            100059ff f   MSVCRT:ehprolg3.obj
 0001:00004a0e       __EH_prolog3               10005a0e f   MSVCRT:ehprolg3.obj
 0001:00004a41       __EH_prolog3_GS            10005a41 f   MSVCRT:ehprolg3.obj
 0001:00004a78       ___CxxFrameHandler3        10005a78 f   MSVCRT:MSVCR120.dll
 0001:00004a7e       ??_Etype_info@@UAEPAXI@Z   10005a7e f i MSVCRT:ti_inst.obj
 0001:00004ac8       __purecall                 10005ac8 f   MSVCRT:MSVCR120.dll
 0001:00004ace       ??_L@YGXPAXIHP6EX0@Z1@Z    10005ace f   MSVCRT:ehvecctr.obj
 0001:00004b30       ??_M@YGXPAXIHP6EX0@Z@Z     10005b30 f   MSVCRT:ehvecdtr.obj
 0001:00004b9f       ?__ArrayUnwind@@YGXPAXIHP6EX0@Z@Z 10005b9f f   MSVCRT:ehvecdtr.obj
 0001:00004bfd       ___atonexitinit            10005bfd f   MSVCRT:atonexit.obj
 0001:00004c39       __onexit                   10005c39 f   MSVCRT:atonexit.obj
 0001:00004ce2       _atexit                    10005ce2 f   MSVCRT:atonexit.obj
 0001:00004d43       __CRT_INIT@12              10005d43 f   MSVCRT:crtdll.obj
 0001:00004f3a       __DllMainCRTStartup@12     10005f3a f   MSVCRT:crtdll.obj
 0001:00005090       ___raise_securityfailure   10006090 f   MSVCRT:gs_report.obj
 0001:000050cd       ___report_gsfailure        100060cd f   MSVCRT:gs_report.obj
 0001:000051c8       ??1type_info@@UAE@XZ       100061c8 f   MSVCRT:MSVCR120.dll
 0001:000051d0       __SEH_prolog4              100061d0 f   MSVCRT:sehprolg4.obj
 0001:00005215       __SEH_epilog4              10006215 f   MSVCRT:sehprolg4.obj
 0001:00005229       __except_handler4          10006229 f   MSVCRT:chandler4gs.obj
 0001:0000524c       ?terminate@@YAXXZ          1000624c f   MSVCRT:MSVCR120.dll
 0001:00005252       __lock                     10006252 f   MSVCRT:MSVCR120.dll
 0001:00005258       __unlock                   10006258 f   MSVCRT:MSVCR120.dll
 0001:0000525e       ___dllonexit               1000625e f   MSVCRT:MSVCR120.dll
 0001:00005264       ___CppXcptFilter           10006264 f   MSVCRT:MSVCR120.dll
 0001:0000526a       __amsg_exit                1000626a f   MSVCRT:MSVCR120.dll
 0001:00005270       __FindPESection            10006270 f   MSVCRT:pesect.obj
 0001:000052c0       __IsNonwritableInCurrentImage 100062c0 f   MSVCRT:pesect.obj
 0001:00005380       __ValidateImageBase        10006380 f   MSVCRT:pesect.obj
 0001:000053b1       ___security_init_cookie    100063b1 f   MSVCRT:gs_support.obj
 0001:0000544d       _DllMain@12                1000644d f   MSVCRT:dllmain.obj
 0001:0000546f       __RTC_Initialize           1000646f f   MSVCRT:initsect.obj
 0001:0000548f       __RTC_Terminate            1000648f f   MSVCRT:initsect.obj
 0001:000054b0       __initterm                 100064b0 f   MSVCRT:MSVCR120.dll
 0001:000054b6       __initterm_e               100064b6 f   MSVCRT:MSVCR120.dll
 0001:000054bc       ___clean_type_info_names   100064bc f   MSVCRT:tncleanup.obj
 0001:000054c8       __crt_debugger_hook        100064c8 f   MSVCRT:MSVCR120.dll
 0001:000054ce       ___crtUnhandledException   100064ce f   MSVCRT:MSVCR120.dll
 0001:000054d4       ___crtTerminateProcess     100064d4 f   MSVCRT:MSVCR120.dll
 0001:000054da       __except_handler4_common   100064da f   MSVCRT:MSVCR120.dll
 0001:000054e0       ___clean_type_info_names_internal 100064e0 f   MSVCRT:MSVCR120.dll
 0001:000054e6       _IsProcessorFeaturePresent@4 100064e6 f   kernel32:KERNEL32.dll
 0002:00000000       __imp__DisableThreadLibraryCalls@4 10008000     kernel32:KERNEL32.dll
 0002:00000004       __imp__GetCurrentThreadId@0 10008004     kernel32:KERNEL32.dll
 0002:00000008       __imp__GetCurrentProcessId@0 10008008     kernel32:KERNEL32.dll
 0002:0000000c       __imp__QueryPerformanceCounter@4 1000800c     kernel32:KERNEL32.dll
 0002:00000010       __imp__IsProcessorFeaturePresent@4 10008010     kernel32:KERNEL32.dll
 0002:00000014       __imp__IsDebuggerPresent@0 10008014     kernel32:KERNEL32.dll
 0002:00000018       __imp__DecodePointer@4     10008018     kernel32:KERNEL32.dll
 0002:0000001c       __imp__EncodePointer@4     1000801c     kernel32:KERNEL32.dll
 0002:00000020       __imp__GetPrivateProfileStringA@24 10008020     kernel32:KERNEL32.dll
 0002:00000024       __imp__GetSystemTimeAsFileTime@4 10008024     kernel32:KERNEL32.dll
 0002:00000028       \177KERNEL32_NULL_THUNK_DATA 10008028     kernel32:KERNEL32.dll
 0002:0000002c       __imp____clean_type_info_names_internal 1000802c     MSVCRT:MSVCR120.dll
 0002:00000030       __imp____crtTerminateProcess 10008030     MSVCRT:MSVCR120.dll
 0002:00000034       __imp____crtUnhandledException 10008034     MSVCRT:MSVCR120.dll
 0002:00000038       __imp___crt_debugger_hook  10008038     MSVCRT:MSVCR120.dll
 0002:0000003c       __imp___initterm_e         1000803c     MSVCRT:MSVCR120.dll
 0002:00000040       __imp___initterm           10008040     MSVCRT:MSVCR120.dll
 0002:00000044       __imp___malloc_crt         10008044     MSVCRT:MSVCR120.dll
 0002:00000048       __imp__free                10008048     MSVCRT:MSVCR120.dll
 0002:0000004c       __imp___amsg_exit          1000804c     MSVCRT:MSVCR120.dll
 0002:00000050       __imp____CppXcptFilter     10008050     MSVCRT:MSVCR120.dll
 0002:00000054       __imp___onexit             10008054     MSVCRT:MSVCR120.dll
 0002:00000058       __imp____dllonexit         10008058     MSVCRT:MSVCR120.dll
 0002:0000005c       __imp___calloc_crt         1000805c     MSVCRT:MSVCR120.dll
 0002:00000060       __imp___unlock             10008060     MSVCRT:MSVCR120.dll
 0002:00000064       __imp___lock               10008064     MSVCRT:MSVCR120.dll
 0002:00000068       __imp_?terminate@@YAXXZ    10008068     MSVCRT:MSVCR120.dll
 0002:0000006c       __imp_??1type_info@@UAE@XZ 1000806c     MSVCRT:MSVCR120.dll
 0002:00000070       __imp___purecall           10008070     MSVCRT:MSVCR120.dll
 0002:00000074       __imp____CxxFrameHandler3  10008074     MSVCRT:MSVCR120.dll
 0002:00000078       __imp_??3@YAXPAX@Z         10008078     MSVCRT:MSVCR120.dll
 0002:0000007c       __imp_??2@YAPAXI@Z         1000807c     MSVCRT:MSVCR120.dll
 0002:00000080       __imp___except_handler4_common 10008080     MSVCRT:MSVCR120.dll
 0002:00000084       \177MSVCR120_NULL_THUNK_DATA 10008084     MSVCRT:MSVCR120.dll
 0002:00000088       __imp_?qt_invoke@CAlm_sys_select@@UAE_NHPAUQUObject@@@Z 10008088     alm_sys_select:alm_sys_select.dll
 0002:0000008c       __imp_?qt_emit@CAlm_sys_select@@UAE_NHPAUQUObject@@@Z 1000808c     alm_sys_select:alm_sys_select.dll
 0002:00000090       __imp_?qt_cast@CAlm_sys_select@@UAEPAXPBD@Z 10008090     alm_sys_select:alm_sys_select.dll
 0002:00000094       __imp_?metaObject@CAlm_sys_select@@UBEPAVQMetaObject@@XZ 10008094     alm_sys_select:alm_sys_select.dll
 0002:00000098       __imp_?className@CAlm_sys_select@@UBEPBDXZ 10008098     alm_sys_select:alm_sys_select.dll
 0002:0000009c       __imp_??1CAlm_sys_select@@UAE@XZ 1000809c     alm_sys_select:alm_sys_select.dll
 0002:000000a0       __imp_??0CAlm_sys_select@@QAE@PAVQWidget@@PBD@Z 100080a0     alm_sys_select:alm_sys_select.dll
 0002:000000a4       __imp_?setSystemNames@CAlm_sys_select@@QAE_NVQString@@@Z 100080a4     alm_sys_select:alm_sys_select.dll
 0002:000000a8       __imp_?getSystemName@CAlm_sys_select@@QAE?AVQString@@XZ 100080a8     alm_sys_select:alm_sys_select.dll
 0002:000000ac       __imp_?qt_property@CAlm_sys_select@@UAE_NHHPAVQVariant@@@Z 100080ac     alm_sys_select:alm_sys_select.dll
 0002:000000b0       \177alm_sys_select_NULL_THUNK_DATA 100080b0     alm_sys_select:alm_sys_select.dll
 0002:000000b4       __imp_?fnConfig_icons@@YAPAPBDPBD@Z 100080b4     config_icons:config_icons.dll
 0002:000000b8       \177config_icons_NULL_THUNK_DATA 100080b8     config_icons:config_icons.dll
 0002:000000bc       __imp_??1QAction@@UAE@XZ   100080bc     qt-mt323:qt-mt323.dll
 0002:000000c0       __imp_??1?$QPtrList@VQDockWindow@@@@UAE@XZ 100080c0     qt-mt323:qt-mt323.dll
 0002:000000c4       __imp_??0QToolBar@@QAE@PAVQMainWindow@@PBD@Z 100080c4     qt-mt323:qt-mt323.dll
 0002:000000c8       __imp_??1QToolBar@@UAE@XZ  100080c8     qt-mt323:qt-mt323.dll
 0002:000000cc       __imp_??0QFile@@QAE@ABVQString@@@Z 100080cc     qt-mt323:qt-mt323.dll
 0002:000000d0       __imp_??1QFile@@UAE@XZ     100080d0     qt-mt323:qt-mt323.dll
 0002:000000d4       __imp_?open@QFile@@UAE_NH@Z 100080d4     qt-mt323:qt-mt323.dll
 0002:000000d8       __imp_?close@QFile@@UAEXXZ 100080d8     qt-mt323:qt-mt323.dll
 0002:000000dc       __imp_??0QListViewItem@@QAE@PAVQListView@@VQString@@1111111@Z 100080dc     qt-mt323:qt-mt323.dll
 0002:000000e0       __imp_??1QListViewItem@@UAE@XZ 100080e0     qt-mt323:qt-mt323.dll
 0002:000000e4       __imp_?selectedItem@QListView@@QBEPAVQListViewItem@@XZ 100080e4     qt-mt323:qt-mt323.dll
 0002:000000e8       __imp_?getText@QInputDialog@@SA?AVQString@@ABV2@0W4EchoMode@QLineEdit@@0PA_NPAVQWidget@@PBD@Z 100080e8     qt-mt323:qt-mt323.dll
 0002:000000ec       __imp_??0QFileInfo@@QAE@XZ 100080ec     qt-mt323:qt-mt323.dll
 0002:000000f0       __imp_??1QFileInfo@@QAE@XZ 100080f0     qt-mt323:qt-mt323.dll
 0002:000000f4       __imp_??0QDir@@QAE@XZ      100080f4     qt-mt323:qt-mt323.dll
 0002:000000f8       __imp_??1QDir@@UAE@XZ      100080f8     qt-mt323:qt-mt323.dll
 0002:000000fc       __imp_?setPath@QDir@@UAEXABVQString@@@Z 100080fc     qt-mt323:qt-mt323.dll
 0002:00000100       __imp_?mkdir@QDir@@UBE_NABVQString@@_N@Z 10008100     qt-mt323:qt-mt323.dll
 0002:00000104       __imp_?exists@QDir@@UBE_NXZ 10008104     qt-mt323:qt-mt323.dll
 0002:00000108       __imp_??0QPopupMenu@@QAE@PAVQWidget@@PBD@Z 10008108     qt-mt323:qt-mt323.dll
 0002:0000010c       __imp_??1QPopupMenu@@UAE@XZ 1000810c     qt-mt323:qt-mt323.dll
 0002:00000110       __imp_??0QGuardedPtrPrivate@@QAE@PAVQObject@@@Z 10008110     qt-mt323:qt-mt323.dll
 0002:00000114       __imp_??1QGuardedPtrPrivate@@UAE@XZ 10008114     qt-mt323:qt-mt323.dll
 0002:00000118       __imp_?reconnect@QGuardedPtrPrivate@@QAEXPAVQObject@@@Z 10008118     qt-mt323:qt-mt323.dll
 0002:0000011c       __imp_??0QGDict@@IAE@IW4KeyType@0@_N1@Z 1000811c     qt-mt323:qt-mt323.dll
 0002:00000120       __imp_??1QGDict@@MAE@XZ    10008120     qt-mt323:qt-mt323.dll
 0002:00000124       __imp_?clear@QGDict@@MAEXXZ 10008124     qt-mt323:qt-mt323.dll
 0002:00000128       __imp_?acceptDrop@QListViewItem@@UBE_NPBVQMimeSource@@@Z 10008128     qt-mt323:qt-mt323.dll
 0002:0000012c       __imp_?activate@QListViewItem@@MAEXXZ 1000812c     qt-mt323:qt-mt323.dll
 0002:00000130       __imp_?activateItemAt@QPopupMenu@@UAEXH@Z 10008130     qt-mt323:qt-mt323.dll
 0002:00000134       __imp_?addTo@QAction@@UAE_NPAVQWidget@@@Z 10008134     qt-mt323:qt-mt323.dll
 0002:00000138       __imp_?addedTo@QAction@@MAEXHPAVQPopupMenu@@@Z 10008138     qt-mt323:qt-mt323.dll
 0002:0000013c       __imp_?addedTo@QAction@@MAEXPAVQWidget@@0@Z 1000813c     qt-mt323:qt-mt323.dll
 0002:00000140       __imp_?adjustSize@QWidget@@UAEXXZ 10008140     qt-mt323:qt-mt323.dll
 0002:00000144       __imp_?cancelRename@QListViewItem@@MAEXH@Z 10008144     qt-mt323:qt-mt323.dll
 0002:00000148       __imp_?checkConnectArgs@QObject@@MAE_NPBDPBV1@0@Z 10008148     qt-mt323:qt-mt323.dll
 0002:0000014c       __imp_?childEvent@QObject@@MAEXPAVQChildEvent@@@Z 1000814c     qt-mt323:qt-mt323.dll
 0002:00000150       __imp_?className@QAction@@UBEPBDXZ 10008150     qt-mt323:qt-mt323.dll
 0002:00000154       __imp_?className@QGuardedPtrPrivate@@UBEPBDXZ 10008154     qt-mt323:qt-mt323.dll
 0002:00000158       __imp_?className@QPopupMenu@@UBEPBDXZ 10008158     qt-mt323:qt-mt323.dll
 0002:0000015c       __imp_?className@QToolBar@@UBEPBDXZ 1000815c     qt-mt323:qt-mt323.dll
 0002:00000160       __imp_?className@QWidget@@UBEPBDXZ 10008160     qt-mt323:qt-mt323.dll
 0002:00000164       __imp_?clear@?$QPtrList@VQDockWindow@@@@UAEXXZ 10008164     qt-mt323:qt-mt323.dll
 0002:00000168       __imp_?clear@QToolBar@@UAEXXZ 10008168     qt-mt323:qt-mt323.dll
 0002:0000016c       __imp_?close@QWidget@@UAE_N_N@Z 1000816c     qt-mt323:qt-mt323.dll
 0002:00000170       __imp_?closeEvent@QPopupMenu@@MAEXPAVQCloseEvent@@@Z 10008170     qt-mt323:qt-mt323.dll
 0002:00000174       __imp_?closeEvent@QWidget@@MAEXPAVQCloseEvent@@@Z 10008174     qt-mt323:qt-mt323.dll
 0002:00000178       __imp_?cmd@QPaintDevice@@MAE_NHPAVQPainter@@PATQPDevCmdParam@@@Z 10008178     qt-mt323:qt-mt323.dll
 0002:0000017c       __imp_?compare@QListViewItem@@UBEHPAV1@H_N@Z 1000817c     qt-mt323:qt-mt323.dll
 0002:00000180       __imp_?compareItems@QGList@@MAEHPAX0@Z 10008180     qt-mt323:qt-mt323.dll
 0002:00000184       __imp_?connectNotify@QObject@@MAEXPBD@Z 10008184     qt-mt323:qt-mt323.dll
 0002:00000188       __imp_?contextMenuEvent@QDockWindow@@MAEXPAVQContextMenuEvent@@@Z 10008188     qt-mt323:qt-mt323.dll
 0002:0000018c       __imp_?contextMenuEvent@QWidget@@MAEXPAVQContextMenuEvent@@@Z 1000818c     qt-mt323:qt-mt323.dll
 0002:00000190       __imp_?count@?$QPtrList@VQDockWindow@@@@UBEIXZ 10008190     qt-mt323:qt-mt323.dll
 0002:00000194       __imp_?create@QWidget@@MAEXPAUHWND__@@_N1@Z 10008194     qt-mt323:qt-mt323.dll
 0002:00000198       __imp_?customEvent@QObject@@MAEXPAVQCustomEvent@@@Z 10008198     qt-mt323:qt-mt323.dll
 0002:0000019c       __imp_?customWhatsThis@QPopupMenu@@UBE_NXZ 1000819c     qt-mt323:qt-mt323.dll
 0002:000001a0       __imp_?customWhatsThis@QWidget@@UBE_NXZ 100081a0     qt-mt323:qt-mt323.dll
 0002:000001a4       __imp_?deleteItem@?$QPtrList@VQDockWindow@@@@EAEXPAX@Z 100081a4     qt-mt323:qt-mt323.dll
 0002:000001a8       __imp_?destroy@QWidget@@MAEX_N0@Z 100081a8     qt-mt323:qt-mt323.dll
 0002:000001ac       __imp_?disconnectNotify@QObject@@MAEXPBD@Z 100081ac     qt-mt323:qt-mt323.dll
 0002:000001b0       __imp_?dock@QDockWindow@@UAEXXZ 100081b0     qt-mt323:qt-mt323.dll
 0002:000001b4       __imp_?dragEnterEvent@QWidget@@MAEXPAVQDragEnterEvent@@@Z 100081b4     qt-mt323:qt-mt323.dll
 0002:000001b8       __imp_?dragEntered@QListViewItem@@MAEXXZ 100081b8     qt-mt323:qt-mt323.dll
 0002:000001bc       __imp_?dragLeaveEvent@QWidget@@MAEXPAVQDragLeaveEvent@@@Z 100081bc     qt-mt323:qt-mt323.dll
 0002:000001c0       __imp_?dragLeft@QListViewItem@@MAEXXZ 100081c0     qt-mt323:qt-mt323.dll
 0002:000001c4       __imp_?dragMoveEvent@QWidget@@MAEXPAVQDragMoveEvent@@@Z 100081c4     qt-mt323:qt-mt323.dll
 0002:000001c8       __imp_?drawContents@QDockWindow@@MAEXPAVQPainter@@@Z 100081c8     qt-mt323:qt-mt323.dll
 0002:000001cc       __imp_?drawContents@QPopupMenu@@MAEXPAVQPainter@@@Z 100081cc     qt-mt323:qt-mt323.dll
 0002:000001d0       __imp_?drawFrame@QDockWindow@@MAEXPAVQPainter@@@Z 100081d0     qt-mt323:qt-mt323.dll
 0002:000001d4       __imp_?drawFrame@QFrame@@MAEXPAVQPainter@@@Z 100081d4     qt-mt323:qt-mt323.dll
 0002:000001d8       __imp_?dropEvent@QWidget@@MAEXPAVQDropEvent@@@Z 100081d8     qt-mt323:qt-mt323.dll
 0002:000001dc       __imp_?dropped@QListViewItem@@MAEXPAVQDropEvent@@@Z 100081dc     qt-mt323:qt-mt323.dll
 0002:000001e0       __imp_?enabledChange@QPopupMenu@@MAEX_N@Z 100081e0     qt-mt323:qt-mt323.dll
 0002:000001e4       __imp_?enabledChange@QWidget@@MAEX_N@Z 100081e4     qt-mt323:qt-mt323.dll
 0002:000001e8       __imp_?enforceSortOrder@QListViewItem@@MBEXXZ 100081e8     qt-mt323:qt-mt323.dll
 0002:000001ec       __imp_?enterEvent@QWidget@@MAEXPAVQEvent@@@Z 100081ec     qt-mt323:qt-mt323.dll
 0002:000001f0       __imp_?event@QObject@@UAE_NPAVQEvent@@@Z 100081f0     qt-mt323:qt-mt323.dll
 0002:000001f4       __imp_?event@QToolBar@@UAE_NPAVQEvent@@@Z 100081f4     qt-mt323:qt-mt323.dll
 0002:000001f8       __imp_?event@QWidget@@MAE_NPAVQEvent@@@Z 100081f8     qt-mt323:qt-mt323.dll
 0002:000001fc       __imp_?eventFilter@QDockWindow@@UAE_NPAVQObject@@PAVQEvent@@@Z 100081fc     qt-mt323:qt-mt323.dll
 0002:00000200       __imp_?eventFilter@QObject@@UAE_NPAV1@PAVQEvent@@@Z 10008200     qt-mt323:qt-mt323.dll
 0002:00000204       __imp_?focusInEvent@QPopupMenu@@MAEXPAVQFocusEvent@@@Z 10008204     qt-mt323:qt-mt323.dll
 0002:00000208       __imp_?focusInEvent@QWidget@@MAEXPAVQFocusEvent@@@Z 10008208     qt-mt323:qt-mt323.dll
 0002:0000020c       __imp_?focusNextPrevChild@QPopupMenu@@MAE_N_N@Z 1000820c     qt-mt323:qt-mt323.dll
 0002:00000210       __imp_?focusNextPrevChild@QWidget@@MAE_N_N@Z 10008210     qt-mt323:qt-mt323.dll
 0002:00000214       __imp_?focusOutEvent@QPopupMenu@@MAEXPAVQFocusEvent@@@Z 10008214     qt-mt323:qt-mt323.dll
 0002:00000218       __imp_?focusOutEvent@QWidget@@MAEXPAVQFocusEvent@@@Z 10008218     qt-mt323:qt-mt323.dll
 0002:0000021c       __imp_?fontChange@QWidget@@MAEXABVQFont@@@Z 1000821c     qt-mt323:qt-mt323.dll
 0002:00000220       __imp_?fontInf@QPaintDevice@@MBEHPAVQFont@@H@Z 10008220     qt-mt323:qt-mt323.dll
 0002:00000224       __imp_?fontMet@QPaintDevice@@MBEHPAVQFont@@HPBDH@Z 10008224     qt-mt323:qt-mt323.dll
 0002:00000228       __imp_?frameChanged@QFrame@@MAEXXZ 10008228     qt-mt323:qt-mt323.dll
 0002:0000022c       __imp_?frameChanged@QPopupMenu@@EAEXXZ 1000822c     qt-mt323:qt-mt323.dll
 0002:00000230       __imp_?handle@QPaintDevice@@UBEPAUHDC__@@XZ 10008230     qt-mt323:qt-mt323.dll
 0002:00000234       __imp_?heightForWidth@QWidget@@UBEHH@Z 10008234     qt-mt323:qt-mt323.dll
 0002:00000238       __imp_?hide@QPopupMenu@@UAEXXZ 10008238     qt-mt323:qt-mt323.dll
 0002:0000023c       __imp_?hide@QToolBar@@UAEXXZ 1000823c     qt-mt323:qt-mt323.dll
 0002:00000240       __imp_?hide@QWidget@@UAEXXZ 10008240     qt-mt323:qt-mt323.dll
 0002:00000244       __imp_?hideEvent@QDockWindow@@MAEXPAVQHideEvent@@@Z 10008244     qt-mt323:qt-mt323.dll
 0002:00000248       __imp_?hideEvent@QWidget@@MAEXPAVQHideEvent@@@Z 10008248     qt-mt323:qt-mt323.dll
 0002:0000024c       __imp_?imComposeEvent@QWidget@@MAEXPAVQIMEvent@@@Z 1000824c     qt-mt323:qt-mt323.dll
 0002:00000250       __imp_?imEndEvent@QWidget@@MAEXPAVQIMEvent@@@Z 10008250     qt-mt323:qt-mt323.dll
 0002:00000254       __imp_?imStartEvent@QWidget@@MAEXPAVQIMEvent@@@Z 10008254     qt-mt323:qt-mt323.dll
 0002:00000258       __imp_?insertChild@QObject@@UAEXPAV1@@Z 10008258     qt-mt323:qt-mt323.dll
 0002:0000025c       __imp_?insertItem@QListViewItem@@UAEXPAV1@@Z 1000825c     qt-mt323:qt-mt323.dll
 0002:00000260       __imp_?invalidateHeight@QListViewItem@@UAEXXZ 10008260     qt-mt323:qt-mt323.dll
 0002:00000264       __imp_?key@QListViewItem@@UBE?AVQString@@H_N@Z 10008264     qt-mt323:qt-mt323.dll
 0002:00000268       __imp_?keyPressEvent@QPopupMenu@@MAEXPAVQKeyEvent@@@Z 10008268     qt-mt323:qt-mt323.dll
 0002:0000026c       __imp_?keyPressEvent@QWidget@@MAEXPAVQKeyEvent@@@Z 1000826c     qt-mt323:qt-mt323.dll
 0002:00000270       __imp_?keyReleaseEvent@QWidget@@MAEXPAVQKeyEvent@@@Z 10008270     qt-mt323:qt-mt323.dll
 0002:00000274       __imp_?leaveEvent@QPopupMenu@@MAEXPAVQEvent@@@Z 10008274     qt-mt323:qt-mt323.dll
 0002:00000278       __imp_?leaveEvent@QWidget@@MAEXPAVQEvent@@@Z 10008278     qt-mt323:qt-mt323.dll
 0002:0000027c       __imp_?menuContentsChanged@QPopupMenu@@EAEXXZ 1000827c     qt-mt323:qt-mt323.dll
 0002:00000280       __imp_?menuDelPopup@QPopupMenu@@EAEXPAV1@@Z 10008280     qt-mt323:qt-mt323.dll
 0002:00000284       __imp_?menuInsPopup@QPopupMenu@@EAEXPAV1@@Z 10008284     qt-mt323:qt-mt323.dll
 0002:00000288       __imp_?menuStateChanged@QPopupMenu@@EAEXXZ 10008288     qt-mt323:qt-mt323.dll
 0002:0000028c       __imp_?metaObject@QAction@@UBEPAVQMetaObject@@XZ 1000828c     qt-mt323:qt-mt323.dll
 0002:00000290       __imp_?metaObject@QGuardedPtrPrivate@@UBEPAVQMetaObject@@XZ 10008290     qt-mt323:qt-mt323.dll
 0002:00000294       __imp_?metaObject@QPopupMenu@@UBEPAVQMetaObject@@XZ 10008294     qt-mt323:qt-mt323.dll
 0002:00000298       __imp_?metaObject@QToolBar@@UBEPAVQMetaObject@@XZ 10008298     qt-mt323:qt-mt323.dll
 0002:0000029c       __imp_?metaObject@QWidget@@UBEPAVQMetaObject@@XZ 1000829c     qt-mt323:qt-mt323.dll
 0002:000002a0       __imp_?metric@QWidget@@MBEHH@Z 100082a0     qt-mt323:qt-mt323.dll
 0002:000002a4       __imp_?minimumSizeHint@QToolBar@@UBE?AVQSize@@XZ 100082a4     qt-mt323:qt-mt323.dll
 0002:000002a8       __imp_?minimumSizeHint@QWidget@@UBE?AVQSize@@XZ 100082a8     qt-mt323:qt-mt323.dll
 0002:000002ac       __imp_?mouseDoubleClickEvent@QWidget@@MAEXPAVQMouseEvent@@@Z 100082ac     qt-mt323:qt-mt323.dll
 0002:000002b0       __imp_?mouseMoveEvent@QPopupMenu@@MAEXPAVQMouseEvent@@@Z 100082b0     qt-mt323:qt-mt323.dll
 0002:000002b4       __imp_?mouseMoveEvent@QWidget@@MAEXPAVQMouseEvent@@@Z 100082b4     qt-mt323:qt-mt323.dll
 0002:000002b8       __imp_?mousePressEvent@QPopupMenu@@MAEXPAVQMouseEvent@@@Z 100082b8     qt-mt323:qt-mt323.dll
 0002:000002bc       __imp_?mousePressEvent@QWidget@@MAEXPAVQMouseEvent@@@Z 100082bc     qt-mt323:qt-mt323.dll
 0002:000002c0       __imp_?mouseReleaseEvent@QPopupMenu@@MAEXPAVQMouseEvent@@@Z 100082c0     qt-mt323:qt-mt323.dll
 0002:000002c4       __imp_?mouseReleaseEvent@QWidget@@MAEXPAVQMouseEvent@@@Z 100082c4     qt-mt323:qt-mt323.dll
 0002:000002c8       __imp_?move@QWidget@@UAEXHH@Z 100082c8     qt-mt323:qt-mt323.dll
 0002:000002cc       __imp_?moveEvent@QWidget@@MAEXPAVQMoveEvent@@@Z 100082cc     qt-mt323:qt-mt323.dll
 0002:000002d0       __imp_?newItem@QPtrCollection@@MAEPAXPAX@Z 100082d0     qt-mt323:qt-mt323.dll
 0002:000002d4       __imp_?okRename@QListViewItem@@MAEXH@Z 100082d4     qt-mt323:qt-mt323.dll
 0002:000002d8       __imp_?paintBranches@QListViewItem@@UAEXPAVQPainter@@ABVQColorGroup@@HHH@Z 100082d8     qt-mt323:qt-mt323.dll
 0002:000002dc       __imp_?paintCell@QListViewItem@@UAEXPAVQPainter@@ABVQColorGroup@@HHH@Z 100082dc     qt-mt323:qt-mt323.dll
 0002:000002e0       __imp_?paintEvent@QFrame@@MAEXPAVQPaintEvent@@@Z 100082e0     qt-mt323:qt-mt323.dll
 0002:000002e4       __imp_?paintEvent@QPopupMenu@@MAEXPAVQPaintEvent@@@Z 100082e4     qt-mt323:qt-mt323.dll
 0002:000002e8       __imp_?paintEvent@QWidget@@MAEXPAVQPaintEvent@@@Z 100082e8     qt-mt323:qt-mt323.dll
 0002:000002ec       __imp_?paintFocus@QListViewItem@@UAEXPAVQPainter@@ABVQColorGroup@@ABVQRect@@@Z 100082ec     qt-mt323:qt-mt323.dll
 0002:000002f0       __imp_?paletteChange@QWidget@@MAEXABVQPalette@@@Z 100082f0     qt-mt323:qt-mt323.dll
 0002:000002f4       __imp_?pixmap@QListViewItem@@UBEPBVQPixmap@@H@Z 100082f4     qt-mt323:qt-mt323.dll
 0002:000002f8       __imp_?polish@QWidget@@UAEXXZ 100082f8     qt-mt323:qt-mt323.dll
 0002:000002fc       __imp_?property@QObject@@UBE?AVQVariant@@PBD@Z 100082fc     qt-mt323:qt-mt323.dll
 0002:00000300       __imp_?qt_cast@QAction@@UAEPAXPBD@Z 10008300     qt-mt323:qt-mt323.dll
 0002:00000304       __imp_?qt_cast@QGuardedPtrPrivate@@UAEPAXPBD@Z 10008304     qt-mt323:qt-mt323.dll
 0002:00000308       __imp_?qt_cast@QPopupMenu@@UAEPAXPBD@Z 10008308     qt-mt323:qt-mt323.dll
 0002:0000030c       __imp_?qt_cast@QToolBar@@UAEPAXPBD@Z 1000830c     qt-mt323:qt-mt323.dll
 0002:00000310       __imp_?qt_cast@QWidget@@UAEPAXPBD@Z 10008310     qt-mt323:qt-mt323.dll
 0002:00000314       __imp_?qt_emit@QAction@@UAE_NHPAUQUObject@@@Z 10008314     qt-mt323:qt-mt323.dll
 0002:00000318       __imp_?qt_emit@QGuardedPtrPrivate@@UAE_NHPAUQUObject@@@Z 10008318     qt-mt323:qt-mt323.dll
 0002:0000031c       __imp_?qt_emit@QPopupMenu@@UAE_NHPAUQUObject@@@Z 1000831c     qt-mt323:qt-mt323.dll
 0002:00000320       __imp_?qt_emit@QToolBar@@UAE_NHPAUQUObject@@@Z 10008320     qt-mt323:qt-mt323.dll
 0002:00000324       __imp_?qt_emit@QWidget@@UAE_NHPAUQUObject@@@Z 10008324     qt-mt323:qt-mt323.dll
 0002:00000328       __imp_?qt_invoke@QAction@@UAE_NHPAUQUObject@@@Z 10008328     qt-mt323:qt-mt323.dll
 0002:0000032c       __imp_?qt_invoke@QGuardedPtrPrivate@@UAE_NHPAUQUObject@@@Z 1000832c     qt-mt323:qt-mt323.dll
 0002:00000330       __imp_?qt_invoke@QPopupMenu@@UAE_NHPAUQUObject@@@Z 10008330     qt-mt323:qt-mt323.dll
 0002:00000334       __imp_?qt_invoke@QToolBar@@UAE_NHPAUQUObject@@@Z 10008334     qt-mt323:qt-mt323.dll
 0002:00000338       __imp_?qt_invoke@QWidget@@UAE_NHPAUQUObject@@@Z 10008338     qt-mt323:qt-mt323.dll
 0002:0000033c       __imp_?qt_property@QAction@@UAE_NHHPAVQVariant@@@Z 1000833c     qt-mt323:qt-mt323.dll
 0002:00000340       __imp_?qt_property@QGuardedPtrPrivate@@UAE_NHHPAVQVariant@@@Z 10008340     qt-mt323:qt-mt323.dll
 0002:00000344       __imp_?qt_property@QPopupMenu@@UAE_NHHPAVQVariant@@@Z 10008344     qt-mt323:qt-mt323.dll
 0002:00000348       __imp_?qt_property@QToolBar@@UAE_NHHPAVQVariant@@@Z 10008348     qt-mt323:qt-mt323.dll
 0002:0000034c       __imp_?qt_property@QWidget@@UAE_NHHPAVQVariant@@@Z 1000834c     qt-mt323:qt-mt323.dll
 0002:00000350       __imp_?read@QGDict@@MAEAAVQDataStream@@AAV2@AAPAX@Z 10008350     qt-mt323:qt-mt323.dll
 0002:00000354       __imp_?read@QGList@@MAEAAVQDataStream@@AAV2@AAPAX@Z 10008354     qt-mt323:qt-mt323.dll
 0002:00000358       __imp_?removeChild@QObject@@UAEXPAV1@@Z 10008358     qt-mt323:qt-mt323.dll
 0002:0000035c       __imp_?removeFrom@QAction@@UAE_NPAVQWidget@@@Z 1000835c     qt-mt323:qt-mt323.dll
 0002:00000360       __imp_?removeItem@QListViewItem@@UAEXPAV1@@Z 10008360     qt-mt323:qt-mt323.dll
 0002:00000364       __imp_?reparent@QWidget@@UAEXPAV1@IABVQPoint@@_N@Z 10008364     qt-mt323:qt-mt323.dll
 0002:00000368       __imp_?resize@QWidget@@UAEXHH@Z 10008368     qt-mt323:qt-mt323.dll
 0002:0000036c       __imp_?resizeEvent@QFrame@@MAEXPAVQResizeEvent@@@Z 1000836c     qt-mt323:qt-mt323.dll
 0002:00000370       __imp_?resizeEvent@QToolBar@@MAEXPAVQResizeEvent@@@Z 10008370     qt-mt323:qt-mt323.dll
 0002:00000374       __imp_?resizeEvent@QWidget@@MAEXPAVQResizeEvent@@@Z 10008374     qt-mt323:qt-mt323.dll
 0002:00000378       __imp_?resolution@QPaintDevice@@UBEHXZ 10008378     qt-mt323:qt-mt323.dll
 0002:0000037c       __imp_?rtti@QListViewItem@@UBEHXZ 1000837c     qt-mt323:qt-mt323.dll
 0002:00000380       __imp_?setAccel@QAction@@UAEXABVQKeySequence@@@Z 10008380     qt-mt323:qt-mt323.dll
 0002:00000384       __imp_?setAcceptDrops@QWidget@@UAEX_N@Z 10008384     qt-mt323:qt-mt323.dll
 0002:00000388       __imp_?setActiveItem@QPopupMenu@@UAEXH@Z 10008388     qt-mt323:qt-mt323.dll
 0002:0000038c       __imp_?setActiveWindow@QWidget@@UAEXXZ 1000838c     qt-mt323:qt-mt323.dll
 0002:00000390       __imp_?setAutoMask@QWidget@@UAEX_N@Z 10008390     qt-mt323:qt-mt323.dll
 0002:00000394       __imp_?setBackgroundColor@QWidget@@UAEXABVQColor@@@Z 10008394     qt-mt323:qt-mt323.dll
 0002:00000398       __imp_?setBackgroundMode@QWidget@@UAEXW4BackgroundMode@Qt@@@Z 10008398     qt-mt323:qt-mt323.dll
 0002:0000039c       __imp_?setBackgroundOrigin@QWidget@@UAEXW4BackgroundOrigin@1@@Z 1000839c     qt-mt323:qt-mt323.dll
 0002:000003a0       __imp_?setBackgroundPixmap@QWidget@@UAEXABVQPixmap@@@Z 100083a0     qt-mt323:qt-mt323.dll
 0002:000003a4       __imp_?setCaption@QDockWindow@@UAEXABVQString@@@Z 100083a4     qt-mt323:qt-mt323.dll
 0002:000003a8       __imp_?setCaption@QWidget@@UAEXABVQString@@@Z 100083a8     qt-mt323:qt-mt323.dll
 0002:000003ac       __imp_?setCheckable@QPopupMenu@@UAEX_N@Z 100083ac     qt-mt323:qt-mt323.dll
 0002:000003b0       __imp_?setCloseMode@QDockWindow@@UAEXH@Z 100083b0     qt-mt323:qt-mt323.dll
 0002:000003b4       __imp_?setCursor@QWidget@@UAEXABVQCursor@@@Z 100083b4     qt-mt323:qt-mt323.dll
 0002:000003b8       __imp_?setDragEnabled@QListViewItem@@UAEX_N@Z 100083b8     qt-mt323:qt-mt323.dll
 0002:000003bc       __imp_?setDropEnabled@QListViewItem@@UAEX_N@Z 100083bc     qt-mt323:qt-mt323.dll
 0002:000003c0       __imp_?setEnabled@QAction@@UAEX_N@Z 100083c0     qt-mt323:qt-mt323.dll
 0002:000003c4       __imp_?setEnabled@QListViewItem@@UAEX_N@Z 100083c4     qt-mt323:qt-mt323.dll
 0002:000003c8       __imp_?setEnabled@QWidget@@UAEX_N@Z 100083c8     qt-mt323:qt-mt323.dll
 0002:000003cc       __imp_?setEraseColor@QWidget@@UAEXABVQColor@@@Z 100083cc     qt-mt323:qt-mt323.dll
 0002:000003d0       __imp_?setErasePixmap@QWidget@@UAEXABVQPixmap@@@Z 100083d0     qt-mt323:qt-mt323.dll
 0002:000003d4       __imp_?setExpandable@QListViewItem@@UAEX_N@Z 100083d4     qt-mt323:qt-mt323.dll
 0002:000003d8       __imp_?setFirstItemActive@QPopupMenu@@EAEXXZ 100083d8     qt-mt323:qt-mt323.dll
 0002:000003dc       __imp_?setFixedExtentHeight@QDockWindow@@UAEXH@Z 100083dc     qt-mt323:qt-mt323.dll
 0002:000003e0       __imp_?setFixedExtentWidth@QDockWindow@@UAEXH@Z 100083e0     qt-mt323:qt-mt323.dll
 0002:000003e4       __imp_?setFocus@QWidget@@UAEXXZ 100083e4     qt-mt323:qt-mt323.dll
 0002:000003e8       __imp_?setFocusPolicy@QWidget@@UAEXW4FocusPolicy@1@@Z 100083e8     qt-mt323:qt-mt323.dll
 0002:000003ec       __imp_?setFocusProxy@QWidget@@UAEXPAV1@@Z 100083ec     qt-mt323:qt-mt323.dll
 0002:000003f0       __imp_?setFont@QPopupMenu@@UAEXABVQFont@@@Z 100083f0     qt-mt323:qt-mt323.dll
 0002:000003f4       __imp_?setFont@QWidget@@UAEXABVQFont@@@Z 100083f4     qt-mt323:qt-mt323.dll
 0002:000003f8       __imp_?setFrameRect@QFrame@@UAEXABVQRect@@@Z 100083f8     qt-mt323:qt-mt323.dll
 0002:000003fc       __imp_?setFrameStyle@QFrame@@UAEXH@Z 100083fc     qt-mt323:qt-mt323.dll
 0002:00000400       __imp_?setGeometry@QWidget@@UAEXABVQRect@@@Z 10008400     qt-mt323:qt-mt323.dll
 0002:00000404       __imp_?setGeometry@QWidget@@UAEXHHHH@Z 10008404     qt-mt323:qt-mt323.dll
 0002:00000408       __imp_?setHeight@QListViewItem@@MAEXH@Z 10008408     qt-mt323:qt-mt323.dll
 0002:0000040c       __imp_?setHorizontallyStretchable@QDockWindow@@UAEX_N@Z 1000840c     qt-mt323:qt-mt323.dll
 0002:00000410       __imp_?setIcon@QWidget@@UAEXABVQPixmap@@@Z 10008410     qt-mt323:qt-mt323.dll
 0002:00000414       __imp_?setIconSet@QAction@@UAEXABVQIconSet@@@Z 10008414     qt-mt323:qt-mt323.dll
 0002:00000418       __imp_?setIconText@QWidget@@UAEXABVQString@@@Z 10008418     qt-mt323:qt-mt323.dll
 0002:0000041c       __imp_?setId@QMenuData@@UAEXHH@Z 1000841c     qt-mt323:qt-mt323.dll
 0002:00000420       __imp_?setKeyCompression@QWidget@@MAEX_N@Z 10008420     qt-mt323:qt-mt323.dll
 0002:00000424       __imp_?setLabel@QToolBar@@UAEXABVQString@@@Z 10008424     qt-mt323:qt-mt323.dll
 0002:00000428       __imp_?setLineWidth@QFrame@@UAEXH@Z 10008428     qt-mt323:qt-mt323.dll
 0002:0000042c       __imp_?setMargin@QFrame@@UAEXH@Z 1000842c     qt-mt323:qt-mt323.dll
 0002:00000430       __imp_?setMask@QWidget@@UAEXABVQBitmap@@@Z 10008430     qt-mt323:qt-mt323.dll
 0002:00000434       __imp_?setMask@QWidget@@UAEXABVQRegion@@@Z 10008434     qt-mt323:qt-mt323.dll
 0002:00000438       __imp_?setMaximumSize@QWidget@@UAEXHH@Z 10008438     qt-mt323:qt-mt323.dll
 0002:0000043c       __imp_?setMenuText@QAction@@UAEXABVQString@@@Z 1000843c     qt-mt323:qt-mt323.dll
 0002:00000440       __imp_?setMicroFocusHint@QWidget@@MAEXHHHH_NPAVQFont@@@Z 10008440     qt-mt323:qt-mt323.dll
 0002:00000444       __imp_?setMidLineWidth@QFrame@@UAEXH@Z 10008444     qt-mt323:qt-mt323.dll
 0002:00000448       __imp_?setMinimumSize@QToolBar@@UAEXHH@Z 10008448     qt-mt323:qt-mt323.dll
 0002:0000044c       __imp_?setMinimumSize@QWidget@@UAEXHH@Z 1000844c     qt-mt323:qt-mt323.dll
 0002:00000450       __imp_?setMouseTracking@QWidget@@UAEX_N@Z 10008450     qt-mt323:qt-mt323.dll
 0002:00000454       __imp_?setMovingEnabled@QDockWindow@@UAEX_N@Z 10008454     qt-mt323:qt-mt323.dll
 0002:00000458       __imp_?setMultiLinesEnabled@QListViewItem@@UAEX_N@Z 10008458     qt-mt323:qt-mt323.dll
 0002:0000045c       __imp_?setName@QObject@@UAEXPBD@Z 1000845c     qt-mt323:qt-mt323.dll
 0002:00000460       __imp_?setNewLine@QDockWindow@@UAEX_N@Z 10008460     qt-mt323:qt-mt323.dll
 0002:00000464       __imp_?setOffset@QDockWindow@@UAEXH@Z 10008464     qt-mt323:qt-mt323.dll
 0002:00000468       __imp_?setOn@QAction@@UAEX_N@Z 10008468     qt-mt323:qt-mt323.dll
 0002:0000046c       __imp_?setOpaqueMoving@QDockWindow@@UAEX_N@Z 1000846c     qt-mt323:qt-mt323.dll
 0002:00000470       __imp_?setOpen@QListViewItem@@UAEX_N@Z 10008470     qt-mt323:qt-mt323.dll
 0002:00000474       __imp_?setOrientation@QToolBar@@UAEXW4Orientation@Qt@@@Z 10008474     qt-mt323:qt-mt323.dll
 0002:00000478       __imp_?setPalette@QWidget@@UAEXABVQPalette@@@Z 10008478     qt-mt323:qt-mt323.dll
 0002:0000047c       __imp_?setPaletteBackgroundColor@QWidget@@UAEXABVQColor@@@Z 1000847c     qt-mt323:qt-mt323.dll
 0002:00000480       __imp_?setPaletteBackgroundPixmap@QWidget@@UAEXABVQPixmap@@@Z 10008480     qt-mt323:qt-mt323.dll
 0002:00000484       __imp_?setPixmap@QListViewItem@@UAEXHABVQPixmap@@@Z 10008484     qt-mt323:qt-mt323.dll
 0002:00000488       __imp_?setProperty@QObject@@UAE_NPBDABVQVariant@@@Z 10008488     qt-mt323:qt-mt323.dll
 0002:0000048c       __imp_?setRenameEnabled@QListViewItem@@UAEXH_N@Z 1000848c     qt-mt323:qt-mt323.dll
 0002:00000490       __imp_?setResizeEnabled@QDockWindow@@UAEX_N@Z 10008490     qt-mt323:qt-mt323.dll
 0002:00000494       __imp_?setResolution@QPaintDevice@@UAEXH@Z 10008494     qt-mt323:qt-mt323.dll
 0002:00000498       __imp_?setSelectable@QListViewItem@@UAEX_N@Z 10008498     qt-mt323:qt-mt323.dll
 0002:0000049c       __imp_?setSelected@QListViewItem@@UAEX_N@Z 1000849c     qt-mt323:qt-mt323.dll
 0002:000004a0       __imp_?setSizeIncrement@QWidget@@UAEXHH@Z 100084a0     qt-mt323:qt-mt323.dll
 0002:000004a4       __imp_?setSizePolicy@QWidget@@UAEXVQSizePolicy@@@Z 100084a4     qt-mt323:qt-mt323.dll
 0002:000004a8       __imp_?setStatusTip@QAction@@UAEXABVQString@@@Z 100084a8     qt-mt323:qt-mt323.dll
 0002:000004ac       __imp_?setStretchableWidget@QToolBar@@UAEXPAVQWidget@@@Z 100084ac     qt-mt323:qt-mt323.dll
 0002:000004b0       __imp_?setText@QAction@@UAEXABVQString@@@Z 100084b0     qt-mt323:qt-mt323.dll
 0002:000004b4       __imp_?setText@QListViewItem@@UAEXHABVQString@@@Z 100084b4     qt-mt323:qt-mt323.dll
 0002:000004b8       __imp_?setToggleAction@QAction@@UAEX_N@Z 100084b8     qt-mt323:qt-mt323.dll
 0002:000004bc       __imp_?setToolTip@QAction@@UAEXABVQString@@@Z 100084bc     qt-mt323:qt-mt323.dll
 0002:000004c0       __imp_?setUpdatesEnabled@QWidget@@UAEX_N@Z 100084c0     qt-mt323:qt-mt323.dll
 0002:000004c4       __imp_?setVerticallyStretchable@QDockWindow@@UAEX_N@Z 100084c4     qt-mt323:qt-mt323.dll
 0002:000004c8       __imp_?setWFlags@QWidget@@MAEXI@Z 100084c8     qt-mt323:qt-mt323.dll
 0002:000004cc       __imp_?setWState@QWidget@@MAEXI@Z 100084cc     qt-mt323:qt-mt323.dll
 0002:000004d0       __imp_?setWhatsThis@QAction@@UAEXABVQString@@@Z 100084d0     qt-mt323:qt-mt323.dll
 0002:000004d4       __imp_?setWidget@QDockWindow@@UAEXPAVQWidget@@@Z 100084d4     qt-mt323:qt-mt323.dll
 0002:000004d8       __imp_?setup@QListViewItem@@UAEXXZ 100084d8     qt-mt323:qt-mt323.dll
 0002:000004dc       __imp_?show@QPopupMenu@@UAEXXZ 100084dc     qt-mt323:qt-mt323.dll
 0002:000004e0       __imp_?show@QToolBar@@UAEXXZ 100084e0     qt-mt323:qt-mt323.dll
 0002:000004e4       __imp_?show@QWidget@@UAEXXZ 100084e4     qt-mt323:qt-mt323.dll
 0002:000004e8       __imp_?showEvent@QDockWindow@@MAEXPAVQShowEvent@@@Z 100084e8     qt-mt323:qt-mt323.dll
 0002:000004ec       __imp_?showEvent@QWidget@@MAEXPAVQShowEvent@@@Z 100084ec     qt-mt323:qt-mt323.dll
 0002:000004f0       __imp_?showMaximized@QWidget@@UAEXXZ 100084f0     qt-mt323:qt-mt323.dll
 0002:000004f4       __imp_?showMinimized@QWidget@@UAEXXZ 100084f4     qt-mt323:qt-mt323.dll
 0002:000004f8       __imp_?showNormal@QWidget@@UAEXXZ 100084f8     qt-mt323:qt-mt323.dll
 0002:000004fc       __imp_?sizeHint@QDockWindow@@UBE?AVQSize@@XZ 100084fc     qt-mt323:qt-mt323.dll
 0002:00000500       __imp_?sizeHint@QPopupMenu@@UBE?AVQSize@@XZ 10008500     qt-mt323:qt-mt323.dll
 0002:00000504       __imp_?sizeHint@QWidget@@UBE?AVQSize@@XZ 10008504     qt-mt323:qt-mt323.dll
 0002:00000508       __imp_?sizePolicy@QWidget@@UBE?AVQSizePolicy@@XZ 10008508     qt-mt323:qt-mt323.dll
 0002:0000050c       __imp_?sort@QListViewItem@@UAEXXZ 1000850c     qt-mt323:qt-mt323.dll
 0002:00000510       __imp_?sortChildItems@QListViewItem@@UAEXH_N@Z 10008510     qt-mt323:qt-mt323.dll
 0002:00000514       __imp_?startRename@QListViewItem@@UAEXH@Z 10008514     qt-mt323:qt-mt323.dll
 0002:00000518       __imp_?styleChange@QPopupMenu@@MAEXAAVQStyle@@@Z 10008518     qt-mt323:qt-mt323.dll
 0002:0000051c       __imp_?styleChange@QToolBar@@MAEXAAVQStyle@@@Z 1000851c     qt-mt323:qt-mt323.dll
 0002:00000520       __imp_?styleChange@QWidget@@MAEXAAVQStyle@@@Z 10008520     qt-mt323:qt-mt323.dll
 0002:00000524       __imp_?tabletEvent@QWidget@@MAEXPAVQTabletEvent@@@Z 10008524     qt-mt323:qt-mt323.dll
 0002:00000528       __imp_??0QAction@@QAE@ABVQString@@ABVQIconSet@@0VQKeySequence@@PAVQObject@@PBD_N@Z 10008528     qt-mt323:qt-mt323.dll
 0002:0000052c       __imp_??0QStringList@@QAE@XZ 1000852c     qt-mt323:qt-mt323.dll
 0002:00000530       __imp_?timerEvent@QObject@@MAEXPAVQTimerEvent@@@Z 10008530     qt-mt323:qt-mt323.dll
 0002:00000534       __imp_?timerEvent@QPopupMenu@@MAEXPAVQTimerEvent@@@Z 10008534     qt-mt323:qt-mt323.dll
 0002:00000538       __imp_?undock@QDockWindow@@UAEXPAVQWidget@@@Z 10008538     qt-mt323:qt-mt323.dll
 0002:0000053c       __imp_?undock@QDockWindow@@UAEXXZ 1000853c     qt-mt323:qt-mt323.dll
 0002:00000540       __imp_?unsetCursor@QWidget@@UAEXXZ 10008540     qt-mt323:qt-mt323.dll
 0002:00000544       __imp_?updateItem@QPopupMenu@@UAEXH@Z 10008544     qt-mt323:qt-mt323.dll
 0002:00000548       __imp_?updateMask@QWidget@@MAEXXZ 10008548     qt-mt323:qt-mt323.dll
 0002:0000054c       __imp_?wheelEvent@QWidget@@MAEXPAVQWheelEvent@@@Z 1000854c     qt-mt323:qt-mt323.dll
 0002:00000550       __imp_?width@QListViewItem@@UBEHABVQFontMetrics@@PBVQListView@@H@Z 10008550     qt-mt323:qt-mt323.dll
 0002:00000554       __imp_?winEvent@QWidget@@MAE_NPAUtagMSG@@@Z 10008554     qt-mt323:qt-mt323.dll
 0002:00000558       __imp_?windowActivationChange@QWidget@@MAEX_N@Z 10008558     qt-mt323:qt-mt323.dll
 0002:0000055c       __imp_?write@QGDict@@MBEAAVQDataStream@@AAV2@PAX@Z 1000855c     qt-mt323:qt-mt323.dll
 0002:00000560       __imp_?write@QGList@@MBEAAVQDataStream@@AAV2@PAX@Z 10008560     qt-mt323:qt-mt323.dll
 0002:00000564       __imp_?null@QString@@2V1@A 10008564     qt-mt323:qt-mt323.dll
 0002:00000568       __imp_??_7?$QPtrList@VQDockWindow@@@@6B@ 10008568     qt-mt323:qt-mt323.dll
 0002:0000056c       __imp_??6?$QValueList@VQString@@@@QAEAAV0@ABVQString@@@Z 1000856c     qt-mt323:qt-mt323.dll
 0002:00000570       __imp_??0QPixmap@@QAE@XZ   10008570     qt-mt323:qt-mt323.dll
 0002:00000574       __imp_?setMinimumSize@QWidget@@QAEXABVQSize@@@Z 10008574     qt-mt323:qt-mt323.dll
 0002:00000578       __imp_?resize@QWidget@@QAEXABVQSize@@@Z 10008578     qt-mt323:qt-mt323.dll
 0002:0000057c       __imp_??0QPushButton@@QAE@PAVQWidget@@PBD@Z 1000857c     qt-mt323:qt-mt323.dll
 0002:00000580       __imp_??1QPushButton@@UAE@XZ 10008580     qt-mt323:qt-mt323.dll
 0002:00000584       __imp_??0QButtonGroup@@QAE@PAVQWidget@@PBD@Z 10008584     qt-mt323:qt-mt323.dll
 0002:00000588       __imp_??1QButtonGroup@@UAE@XZ 10008588     qt-mt323:qt-mt323.dll
 0002:0000058c       __imp_??0QLabel@@QAE@PAVQWidget@@PBDI@Z 1000858c     qt-mt323:qt-mt323.dll
 0002:00000590       __imp_??1QLabel@@UAE@XZ    10008590     qt-mt323:qt-mt323.dll
 0002:00000594       __imp_??0QListView@@QAE@PAVQWidget@@PBDI@Z 10008594     qt-mt323:qt-mt323.dll
 0002:00000598       __imp_??1QListView@@UAE@XZ 10008598     qt-mt323:qt-mt323.dll
 0002:0000059c       __imp_?header@QListView@@QBEPAVQHeader@@XZ 1000859c     qt-mt323:qt-mt323.dll
 0002:000005a0       __imp_??1QLayoutItem@@UAE@XZ 100085a0     qt-mt323:qt-mt323.dll
 0002:000005a4       __imp_??0QSpacerItem@@QAE@HHW4SizeType@QSizePolicy@@0@Z 100085a4     qt-mt323:qt-mt323.dll
 0002:000005a8       __imp_?addWidget@QBoxLayout@@QAEXPAVQWidget@@HH@Z 100085a8     qt-mt323:qt-mt323.dll
 0002:000005ac       __imp_?addLayout@QBoxLayout@@QAEXPAVQLayout@@H@Z 100085ac     qt-mt323:qt-mt323.dll
 0002:000005b0       __imp_??0QHBoxLayout@@QAE@PAVQWidget@@HHPBD@Z 100085b0     qt-mt323:qt-mt323.dll
 0002:000005b4       __imp_??1QHBoxLayout@@UAE@XZ 100085b4     qt-mt323:qt-mt323.dll
 0002:000005b8       __imp_??0QVBoxLayout@@QAE@PAVQWidget@@HHPBD@Z 100085b8     qt-mt323:qt-mt323.dll
 0002:000005bc       __imp_??0QVBoxLayout@@QAE@PAVQLayout@@HPBD@Z 100085bc     qt-mt323:qt-mt323.dll
 0002:000005c0       __imp_??1QVBoxLayout@@UAE@XZ 100085c0     qt-mt323:qt-mt323.dll
 0002:000005c4       __imp_?addChild@QScrollView@@UAEXPAVQWidget@@HH@Z 100085c4     qt-mt323:qt-mt323.dll
 0002:000005c8       __imp_?addColumn@QListView@@UAEHABVQIconSet@@ABVQString@@H@Z 100085c8     qt-mt323:qt-mt323.dll
 0002:000005cc       __imp_?addColumn@QListView@@UAEHABVQString@@H@Z 100085cc     qt-mt323:qt-mt323.dll
 0002:000005d0       __imp_?addItem@QBoxLayout@@UAEXPAVQLayoutItem@@@Z 100085d0     qt-mt323:qt-mt323.dll
 0002:000005d4       __imp_?childEvent@QGroupBox@@MAEXPAVQChildEvent@@@Z 100085d4     qt-mt323:qt-mt323.dll
 0002:000005d8       __imp_?childEvent@QLayout@@MAEXPAVQChildEvent@@@Z 100085d8     qt-mt323:qt-mt323.dll
 0002:000005dc       __imp_?className@QButtonGroup@@UBEPBDXZ 100085dc     qt-mt323:qt-mt323.dll
 0002:000005e0       __imp_?className@QHBoxLayout@@UBEPBDXZ 100085e0     qt-mt323:qt-mt323.dll
 0002:000005e4       __imp_?className@QLabel@@UBEPBDXZ 100085e4     qt-mt323:qt-mt323.dll
 0002:000005e8       __imp_?className@QListView@@UBEPBDXZ 100085e8     qt-mt323:qt-mt323.dll
 0002:000005ec       __imp_?className@QPushButton@@UBEPBDXZ 100085ec     qt-mt323:qt-mt323.dll
 0002:000005f0       __imp_?className@QVBoxLayout@@UBEPBDXZ 100085f0     qt-mt323:qt-mt323.dll
 0002:000005f4       __imp_?clear@QListView@@UAEXXZ 100085f4     qt-mt323:qt-mt323.dll
 0002:000005f8       __imp_?clearSelection@QListView@@UAEXXZ 100085f8     qt-mt323:qt-mt323.dll
 0002:000005fc       __imp_?contentsContextMenuEvent@QListView@@MAEXPAVQContextMenuEvent@@@Z 100085fc     qt-mt323:qt-mt323.dll
 0002:00000600       __imp_?contentsDragEnterEvent@QListView@@MAEXPAVQDragEnterEvent@@@Z 10008600     qt-mt323:qt-mt323.dll
 0002:00000604       __imp_?contentsDragLeaveEvent@QListView@@MAEXPAVQDragLeaveEvent@@@Z 10008604     qt-mt323:qt-mt323.dll
 0002:00000608       __imp_?contentsDragMoveEvent@QListView@@MAEXPAVQDragMoveEvent@@@Z 10008608     qt-mt323:qt-mt323.dll
 0002:0000060c       __imp_?contentsDropEvent@QListView@@MAEXPAVQDropEvent@@@Z 1000860c     qt-mt323:qt-mt323.dll
 0002:00000610       __imp_?contentsMouseDoubleClickEvent@QListView@@MAEXPAVQMouseEvent@@@Z 10008610     qt-mt323:qt-mt323.dll
 0002:00000614       __imp_?contentsMouseMoveEvent@QListView@@MAEXPAVQMouseEvent@@@Z 10008614     qt-mt323:qt-mt323.dll
 0002:00000618       __imp_?contentsMousePressEvent@QListView@@MAEXPAVQMouseEvent@@@Z 10008618     qt-mt323:qt-mt323.dll
 0002:0000061c       __imp_?contentsMouseReleaseEvent@QListView@@MAEXPAVQMouseEvent@@@Z 1000861c     qt-mt323:qt-mt323.dll
 0002:00000620       __imp_?contentsWheelEvent@QScrollView@@MAEXPAVQWheelEvent@@@Z 10008620     qt-mt323:qt-mt323.dll
 0002:00000624       __imp_?contextMenuEvent@QScrollView@@MAEXPAVQContextMenuEvent@@@Z 10008624     qt-mt323:qt-mt323.dll
 0002:00000628       __imp_?dragObject@QListView@@MAEPAVQDragObject@@XZ 10008628     qt-mt323:qt-mt323.dll
 0002:0000062c       __imp_?drawButton@QPushButton@@MAEXPAVQPainter@@@Z 1000862c     qt-mt323:qt-mt323.dll
 0002:00000630       __imp_?drawButtonLabel@QPushButton@@MAEXPAVQPainter@@@Z 10008630     qt-mt323:qt-mt323.dll
 0002:00000634       __imp_?drawContents@QFrame@@MAEXPAVQPainter@@@Z 10008634     qt-mt323:qt-mt323.dll
 0002:00000638       __imp_?drawContents@QLabel@@MAEXPAVQPainter@@@Z 10008638     qt-mt323:qt-mt323.dll
 0002:0000063c       __imp_?drawContents@QScrollView@@EAEXPAVQPainter@@@Z 1000863c     qt-mt323:qt-mt323.dll
 0002:00000640       __imp_?drawContents@QScrollView@@MAEXPAVQPainter@@HHHH@Z 10008640     qt-mt323:qt-mt323.dll
 0002:00000644       __imp_?drawContentsOffset@QListView@@MAEXPAVQPainter@@HHHHHH@Z 10008644     qt-mt323:qt-mt323.dll
 0002:00000648       __imp_?enabledChange@QButton@@MAEX_N@Z 10008648     qt-mt323:qt-mt323.dll
 0002:0000064c       __imp_?event@QButtonGroup@@MAE_NPAVQEvent@@@Z 1000864c     qt-mt323:qt-mt323.dll
 0002:00000650       __imp_?eventFilter@QLayout@@MAE_NPAVQObject@@PAVQEvent@@@Z 10008650     qt-mt323:qt-mt323.dll
 0002:00000654       __imp_?eventFilter@QListView@@UAE_NPAVQObject@@PAVQEvent@@@Z 10008654     qt-mt323:qt-mt323.dll
 0002:00000658       __imp_?expanding@QBoxLayout@@UBE?AW4ExpandData@QSizePolicy@@XZ 10008658     qt-mt323:qt-mt323.dll
 0002:0000065c       __imp_?expanding@QSpacerItem@@UBE?AW4ExpandData@QSizePolicy@@XZ 1000865c     qt-mt323:qt-mt323.dll
 0002:00000660       __imp_?focusInEvent@QGroupBox@@MAEXPAVQFocusEvent@@@Z 10008660     qt-mt323:qt-mt323.dll
 0002:00000664       __imp_?focusInEvent@QListView@@MAEXPAVQFocusEvent@@@Z 10008664     qt-mt323:qt-mt323.dll
 0002:00000668       __imp_?focusInEvent@QPushButton@@MAEXPAVQFocusEvent@@@Z 10008668     qt-mt323:qt-mt323.dll
 0002:0000066c       __imp_?focusNextPrevChild@QScrollView@@MAE_N_N@Z 1000866c     qt-mt323:qt-mt323.dll
 0002:00000670       __imp_?focusOutEvent@QListView@@MAEXPAVQFocusEvent@@@Z 10008670     qt-mt323:qt-mt323.dll
 0002:00000674       __imp_?focusOutEvent@QPushButton@@MAEXPAVQFocusEvent@@@Z 10008674     qt-mt323:qt-mt323.dll
 0002:00000678       __imp_?fontChange@QGroupBox@@MAEXABVQFont@@@Z 10008678     qt-mt323:qt-mt323.dll
 0002:0000067c       __imp_?fontChange@QLabel@@MAEXABVQFont@@@Z 1000867c     qt-mt323:qt-mt323.dll
 0002:00000680       __imp_?fontChange@QScrollView@@MAEXABVQFont@@@Z 10008680     qt-mt323:qt-mt323.dll
 0002:00000684       __imp_?frameChanged@QHBox@@MAEXXZ 10008684     qt-mt323:qt-mt323.dll
 0002:00000688       __imp_?frameChanged@QScrollView@@MAEXXZ 10008688     qt-mt323:qt-mt323.dll
 0002:0000068c       __imp_?geometry@QLayout@@UBE?AVQRect@@XZ 1000868c     qt-mt323:qt-mt323.dll
 0002:00000690       __imp_?geometry@QSpacerItem@@UBE?AVQRect@@XZ 10008690     qt-mt323:qt-mt323.dll
 0002:00000694       __imp_?hasHeightForWidth@QBoxLayout@@UBE_NXZ 10008694     qt-mt323:qt-mt323.dll
 0002:00000698       __imp_?hasHeightForWidth@QLayoutItem@@UBE_NXZ 10008698     qt-mt323:qt-mt323.dll
 0002:0000069c       __imp_?heightForWidth@QBoxLayout@@UBEHH@Z 1000869c     qt-mt323:qt-mt323.dll
 0002:000006a0       __imp_?heightForWidth@QLabel@@UBEHH@Z 100086a0     qt-mt323:qt-mt323.dll
 0002:000006a4       __imp_?heightForWidth@QLayoutItem@@UBEHH@Z 100086a4     qt-mt323:qt-mt323.dll
 0002:000006a8       __imp_?hitButton@QButton@@MBE_NABVQPoint@@@Z 100086a8     qt-mt323:qt-mt323.dll
 0002:000006ac       __imp_?insertItem@QListView@@UAEXPAVQListViewItem@@@Z 100086ac     qt-mt323:qt-mt323.dll
 0002:000006b0       __imp_?invalidate@QBoxLayout@@UAEXXZ 100086b0     qt-mt323:qt-mt323.dll
 0002:000006b4       __imp_?invalidate@QLayoutItem@@UAEXXZ 100086b4     qt-mt323:qt-mt323.dll
 0002:000006b8       __imp_?invertSelection@QListView@@UAEXXZ 100086b8     qt-mt323:qt-mt323.dll
 0002:000006bc       __imp_?isEmpty@QLayout@@UBE_NXZ 100086bc     qt-mt323:qt-mt323.dll
 0002:000006c0       __imp_?isEmpty@QSpacerItem@@UBE_NXZ 100086c0     qt-mt323:qt-mt323.dll
 0002:000006c4       __imp_?iterator@QBoxLayout@@UAE?AVQLayoutIterator@@XZ 100086c4     qt-mt323:qt-mt323.dll
 0002:000006c8       __imp_?iterator@QLayoutItem@@UAE?AVQLayoutIterator@@XZ 100086c8     qt-mt323:qt-mt323.dll
 0002:000006cc       __imp_?keyPressEvent@QButton@@MAEXPAVQKeyEvent@@@Z 100086cc     qt-mt323:qt-mt323.dll
 0002:000006d0       __imp_?keyPressEvent@QListView@@MAEXPAVQKeyEvent@@@Z 100086d0     qt-mt323:qt-mt323.dll
 0002:000006d4       __imp_?keyReleaseEvent@QButton@@MAEXPAVQKeyEvent@@@Z 100086d4     qt-mt323:qt-mt323.dll
 0002:000006d8       __imp_?layout@QLayout@@UAEPAV1@XZ 100086d8     qt-mt323:qt-mt323.dll
 0002:000006dc       __imp_?layout@QLayoutItem@@UAEPAVQLayout@@XZ 100086dc     qt-mt323:qt-mt323.dll
 0002:000006e0       __imp_?maximumSize@QBoxLayout@@UBE?AVQSize@@XZ 100086e0     qt-mt323:qt-mt323.dll
 0002:000006e4       __imp_?maximumSize@QSpacerItem@@UBE?AVQSize@@XZ 100086e4     qt-mt323:qt-mt323.dll
 0002:000006e8       __imp_?metaObject@QButtonGroup@@UBEPAVQMetaObject@@XZ 100086e8     qt-mt323:qt-mt323.dll
 0002:000006ec       __imp_?metaObject@QHBoxLayout@@UBEPAVQMetaObject@@XZ 100086ec     qt-mt323:qt-mt323.dll
 0002:000006f0       __imp_?metaObject@QLabel@@UBEPAVQMetaObject@@XZ 100086f0     qt-mt323:qt-mt323.dll
 0002:000006f4       __imp_?metaObject@QListView@@UBEPAVQMetaObject@@XZ 100086f4     qt-mt323:qt-mt323.dll
 0002:000006f8       __imp_?metaObject@QPushButton@@UBEPAVQMetaObject@@XZ 100086f8     qt-mt323:qt-mt323.dll
 0002:000006fc       __imp_?metaObject@QVBoxLayout@@UBEPAVQMetaObject@@XZ 100086fc     qt-mt323:qt-mt323.dll
 0002:00000700       __imp_?minimumSize@QBoxLayout@@UBE?AVQSize@@XZ 10008700     qt-mt323:qt-mt323.dll
 0002:00000704       __imp_?minimumSize@QSpacerItem@@UBE?AVQSize@@XZ 10008704     qt-mt323:qt-mt323.dll
 0002:00000708       __imp_?minimumSizeHint@QLabel@@UBE?AVQSize@@XZ 10008708     qt-mt323:qt-mt323.dll
 0002:0000070c       __imp_?minimumSizeHint@QListView@@UBE?AVQSize@@XZ 1000870c     qt-mt323:qt-mt323.dll
 0002:00000710       __imp_?mouseDoubleClickEvent@QScrollView@@MAEXPAVQMouseEvent@@@Z 10008710     qt-mt323:qt-mt323.dll
 0002:00000714       __imp_?mouseMoveEvent@QButton@@MAEXPAVQMouseEvent@@@Z 10008714     qt-mt323:qt-mt323.dll
 0002:00000718       __imp_?mouseMoveEvent@QScrollView@@MAEXPAVQMouseEvent@@@Z 10008718     qt-mt323:qt-mt323.dll
 0002:0000071c       __imp_?mousePressEvent@QButton@@MAEXPAVQMouseEvent@@@Z 1000871c     qt-mt323:qt-mt323.dll
 0002:00000720       __imp_?mousePressEvent@QScrollView@@MAEXPAVQMouseEvent@@@Z 10008720     qt-mt323:qt-mt323.dll
 0002:00000724       __imp_?mouseReleaseEvent@QButton@@MAEXPAVQMouseEvent@@@Z 10008724     qt-mt323:qt-mt323.dll
 0002:00000728       __imp_?mouseReleaseEvent@QScrollView@@MAEXPAVQMouseEvent@@@Z 10008728     qt-mt323:qt-mt323.dll
 0002:0000072c       __imp_?move@QPushButton@@UAEXHH@Z 1000872c     qt-mt323:qt-mt323.dll
 0002:00000730       __imp_?moveChild@QScrollView@@UAEXPAVQWidget@@HH@Z 10008730     qt-mt323:qt-mt323.dll
 0002:00000734       __imp_?moveFocus@QButtonGroup@@UAEXH@Z 10008734     qt-mt323:qt-mt323.dll
 0002:00000738       __imp_?paintEmptyArea@QListView@@MAEXPAVQPainter@@ABVQRect@@@Z 10008738     qt-mt323:qt-mt323.dll
 0002:0000073c       __imp_?paintEvent@QButton@@MAEXPAVQPaintEvent@@@Z 1000873c     qt-mt323:qt-mt323.dll
 0002:00000740       __imp_?paintEvent@QGroupBox@@MAEXPAVQPaintEvent@@@Z 10008740     qt-mt323:qt-mt323.dll
 0002:00000744       __imp_?qt_cast@QButtonGroup@@UAEPAXPBD@Z 10008744     qt-mt323:qt-mt323.dll
 0002:00000748       __imp_?qt_cast@QHBoxLayout@@UAEPAXPBD@Z 10008748     qt-mt323:qt-mt323.dll
 0002:0000074c       __imp_?qt_cast@QLabel@@UAEPAXPBD@Z 1000874c     qt-mt323:qt-mt323.dll
 0002:00000750       __imp_?qt_cast@QListView@@UAEPAXPBD@Z 10008750     qt-mt323:qt-mt323.dll
 0002:00000754       __imp_?qt_cast@QPushButton@@UAEPAXPBD@Z 10008754     qt-mt323:qt-mt323.dll
 0002:00000758       __imp_?qt_cast@QVBoxLayout@@UAEPAXPBD@Z 10008758     qt-mt323:qt-mt323.dll
 0002:0000075c       __imp_?qt_emit@QButtonGroup@@UAE_NHPAUQUObject@@@Z 1000875c     qt-mt323:qt-mt323.dll
 0002:00000760       __imp_?qt_emit@QHBoxLayout@@UAE_NHPAUQUObject@@@Z 10008760     qt-mt323:qt-mt323.dll
 0002:00000764       __imp_?qt_emit@QLabel@@UAE_NHPAUQUObject@@@Z 10008764     qt-mt323:qt-mt323.dll
 0002:00000768       __imp_?qt_emit@QListView@@UAE_NHPAUQUObject@@@Z 10008768     qt-mt323:qt-mt323.dll
 0002:0000076c       __imp_?qt_emit@QPushButton@@UAE_NHPAUQUObject@@@Z 1000876c     qt-mt323:qt-mt323.dll
 0002:00000770       __imp_?qt_emit@QVBoxLayout@@UAE_NHPAUQUObject@@@Z 10008770     qt-mt323:qt-mt323.dll
 0002:00000774       __imp_?qt_invoke@QButtonGroup@@UAE_NHPAUQUObject@@@Z 10008774     qt-mt323:qt-mt323.dll
 0002:00000778       __imp_?qt_invoke@QHBoxLayout@@UAE_NHPAUQUObject@@@Z 10008778     qt-mt323:qt-mt323.dll
 0002:0000077c       __imp_?qt_invoke@QLabel@@UAE_NHPAUQUObject@@@Z 1000877c     qt-mt323:qt-mt323.dll
 0002:00000780       __imp_?qt_invoke@QListView@@UAE_NHPAUQUObject@@@Z 10008780     qt-mt323:qt-mt323.dll
 0002:00000784       __imp_?qt_invoke@QPushButton@@UAE_NHPAUQUObject@@@Z 10008784     qt-mt323:qt-mt323.dll
 0002:00000788       __imp_?qt_invoke@QVBoxLayout@@UAE_NHPAUQUObject@@@Z 10008788     qt-mt323:qt-mt323.dll
 0002:0000078c       __imp_?qt_property@QButtonGroup@@UAE_NHHPAVQVariant@@@Z 1000878c     qt-mt323:qt-mt323.dll
 0002:00000790       __imp_?qt_property@QHBoxLayout@@UAE_NHHPAVQVariant@@@Z 10008790     qt-mt323:qt-mt323.dll
 0002:00000794       __imp_?qt_property@QLabel@@UAE_NHHPAVQVariant@@@Z 10008794     qt-mt323:qt-mt323.dll
 0002:00000798       __imp_?qt_property@QListView@@UAE_NHHPAVQVariant@@@Z 10008798     qt-mt323:qt-mt323.dll
 0002:0000079c       __imp_?qt_property@QPushButton@@UAE_NHHPAVQVariant@@@Z 1000879c     qt-mt323:qt-mt323.dll
 0002:000007a0       __imp_?qt_property@QVBoxLayout@@UAE_NHHPAVQVariant@@@Z 100087a0     qt-mt323:qt-mt323.dll
 0002:000007a4       __imp_?removeChild@QScrollView@@UAEXPAVQObject@@@Z 100087a4     qt-mt323:qt-mt323.dll
 0002:000007a8       __imp_?removeColumn@QListView@@UAEXH@Z 100087a8     qt-mt323:qt-mt323.dll
 0002:000007ac       __imp_?removeItem@QListView@@UAEXPAVQListViewItem@@@Z 100087ac     qt-mt323:qt-mt323.dll
 0002:000007b0       __imp_?resize@QPushButton@@UAEXHH@Z 100087b0     qt-mt323:qt-mt323.dll
 0002:000007b4       __imp_?resize@QScrollView@@UAEXHH@Z 100087b4     qt-mt323:qt-mt323.dll
 0002:000007b8       __imp_?resizeContents@QScrollView@@UAEXHH@Z 100087b8     qt-mt323:qt-mt323.dll
 0002:000007bc       __imp_?resizeEvent@QGroupBox@@MAEXPAVQResizeEvent@@@Z 100087bc     qt-mt323:qt-mt323.dll
 0002:000007c0       __imp_?resizeEvent@QLabel@@MAEXPAVQResizeEvent@@@Z 100087c0     qt-mt323:qt-mt323.dll
 0002:000007c4       __imp_?resizeEvent@QListView@@MAEXPAVQResizeEvent@@@Z 100087c4     qt-mt323:qt-mt323.dll
 0002:000007c8       __imp_?resizeEvent@QPushButton@@MAEXPAVQResizeEvent@@@Z 100087c8     qt-mt323:qt-mt323.dll
 0002:000007cc       __imp_?selectAll@QListView@@UAEX_N@Z 100087cc     qt-mt323:qt-mt323.dll
 0002:000007d0       __imp_?setAccel@QButton@@UAEXABVQKeySequence@@@Z 100087d0     qt-mt323:qt-mt323.dll
 0002:000007d4       __imp_?setAlignment@QGroupBox@@UAEXH@Z 100087d4     qt-mt323:qt-mt323.dll
 0002:000007d8       __imp_?setAlignment@QLabel@@UAEXH@Z 100087d8     qt-mt323:qt-mt323.dll
 0002:000007dc       __imp_?setAlignment@QLayoutItem@@UAEXH@Z 100087dc     qt-mt323:qt-mt323.dll
 0002:000007e0       __imp_?setAllColumnsShowFocus@QListView@@UAEX_N@Z 100087e0     qt-mt323:qt-mt323.dll
 0002:000007e4       __imp_?setAutoAdd@QLayout@@UAEX_N@Z 100087e4     qt-mt323:qt-mt323.dll
 0002:000007e8       __imp_?setAutoDefault@QPushButton@@UAEX_N@Z 100087e8     qt-mt323:qt-mt323.dll
 0002:000007ec       __imp_?setAutoRepeat@QButton@@UAEX_N@Z 100087ec     qt-mt323:qt-mt323.dll
 0002:000007f0       __imp_?setAutoResize@QLabel@@UAEX_N@Z 100087f0     qt-mt323:qt-mt323.dll
 0002:000007f4       __imp_?setBuddy@QLabel@@UAEXPAVQWidget@@@Z 100087f4     qt-mt323:qt-mt323.dll
 0002:000007f8       __imp_?setButton@QButtonGroup@@UAEXH@Z 100087f8     qt-mt323:qt-mt323.dll
 0002:000007fc       __imp_?setColumnAlignment@QListView@@UAEXHH@Z 100087fc     qt-mt323:qt-mt323.dll
 0002:00000800       __imp_?setColumnLayout@QGroupBox@@UAEXHW4Orientation@Qt@@@Z 10008800     qt-mt323:qt-mt323.dll
 0002:00000804       __imp_?setColumnText@QListView@@UAEXHABVQIconSet@@ABVQString@@@Z 10008804     qt-mt323:qt-mt323.dll
 0002:00000808       __imp_?setColumnText@QListView@@UAEXHABVQString@@@Z 10008808     qt-mt323:qt-mt323.dll
 0002:0000080c       __imp_?setColumnWidth@QListView@@UAEXHH@Z 1000880c     qt-mt323:qt-mt323.dll
 0002:00000810       __imp_?setColumnWidthMode@QListView@@UAEXHW4WidthMode@1@@Z 10008810     qt-mt323:qt-mt323.dll
 0002:00000814       __imp_?setContentsPos@QListView@@UAEXHH@Z 10008814     qt-mt323:qt-mt323.dll
 0002:00000818       __imp_?setCornerWidget@QScrollView@@UAEXPAVQWidget@@@Z 10008818     qt-mt323:qt-mt323.dll
 0002:0000081c       __imp_?setCurrentItem@QListView@@UAEXPAVQListViewItem@@@Z 1000881c     qt-mt323:qt-mt323.dll
 0002:00000820       __imp_?setDefault@QPushButton@@UAEX_N@Z 10008820     qt-mt323:qt-mt323.dll
 0002:00000824       __imp_?setDefaultRenameAction@QListView@@UAEXW4RenameAction@1@@Z 10008824     qt-mt323:qt-mt323.dll
 0002:00000828       __imp_?setDown@QButton@@UAEX_N@Z 10008828     qt-mt323:qt-mt323.dll
 0002:0000082c       __imp_?setDragAutoScroll@QScrollView@@UAEX_N@Z 1000882c     qt-mt323:qt-mt323.dll
 0002:00000830       __imp_?setEnabled@QGroupBox@@UAEX_N@Z 10008830     qt-mt323:qt-mt323.dll
 0002:00000834       __imp_?setEnabled@QScrollView@@UAEX_N@Z 10008834     qt-mt323:qt-mt323.dll
 0002:00000838       __imp_?setExclusive@QButtonGroup@@UAEX_N@Z 10008838     qt-mt323:qt-mt323.dll
 0002:0000083c       __imp_?setFont@QLabel@@UAEXABVQFont@@@Z 1000883c     qt-mt323:qt-mt323.dll
 0002:00000840       __imp_?setFont@QListView@@UAEXABVQFont@@@Z 10008840     qt-mt323:qt-mt323.dll
 0002:00000844       __imp_?setGeometry@QBoxLayout@@UAEXABVQRect@@@Z 10008844     qt-mt323:qt-mt323.dll
 0002:00000848       __imp_?setGeometry@QPushButton@@UAEXABVQRect@@@Z 10008848     qt-mt323:qt-mt323.dll
 0002:0000084c       __imp_?setGeometry@QPushButton@@UAEXHHHH@Z 1000884c     qt-mt323:qt-mt323.dll
 0002:00000850       __imp_?setGeometry@QSpacerItem@@UAEXABVQRect@@@Z 10008850     qt-mt323:qt-mt323.dll
 0002:00000854       __imp_?setGroup@QButton@@EAEXPAVQButtonGroup@@@Z 10008854     qt-mt323:qt-mt323.dll
 0002:00000858       __imp_?setHBarGeometry@QScrollView@@MAEXAAVQScrollBar@@HHHH@Z 10008858     qt-mt323:qt-mt323.dll
 0002:0000085c       __imp_?setHScrollBarMode@QScrollView@@UAEXW4ScrollBarMode@1@@Z 1000885c     qt-mt323:qt-mt323.dll
 0002:00000860       __imp_?setIsMenuButton@QPushButton@@UAEX_N@Z 10008860     qt-mt323:qt-mt323.dll
 0002:00000864       __imp_?setItemMargin@QListView@@UAEXH@Z 10008864     qt-mt323:qt-mt323.dll
 0002:00000868       __imp_?setMargin@QLayout@@UAEXH@Z 10008868     qt-mt323:qt-mt323.dll
 0002:0000086c       __imp_?setMargins@QScrollView@@MAEXHHHH@Z 1000886c     qt-mt323:qt-mt323.dll
 0002:00000870       __imp_?setMenuBar@QLayout@@UAEXPAVQMenuBar@@@Z 10008870     qt-mt323:qt-mt323.dll
 0002:00000874       __imp_?setMovie@QLabel@@UAEXABVQMovie@@@Z 10008874     qt-mt323:qt-mt323.dll
 0002:00000878       __imp_?setMultiSelection@QListView@@UAEX_N@Z 10008878     qt-mt323:qt-mt323.dll
 0002:0000087c       __imp_?setNum@QLabel@@UAEXH@Z 1000887c     qt-mt323:qt-mt323.dll
 0002:00000880       __imp_?setNum@QLabel@@UAEXN@Z 10008880     qt-mt323:qt-mt323.dll
 0002:00000884       __imp_?setOn@QPushButton@@UAEX_N@Z 10008884     qt-mt323:qt-mt323.dll
 0002:00000888       __imp_?setOpen@QListView@@UAEXPAVQListViewItem@@_N@Z 10008888     qt-mt323:qt-mt323.dll
 0002:0000088c       __imp_?setPalette@QListView@@UAEXABVQPalette@@@Z 1000888c     qt-mt323:qt-mt323.dll
 0002:00000890       __imp_?setPicture@QLabel@@UAEXABVQPicture@@@Z 10008890     qt-mt323:qt-mt323.dll
 0002:00000894       __imp_?setPixmap@QButton@@UAEXABVQPixmap@@@Z 10008894     qt-mt323:qt-mt323.dll
 0002:00000898       __imp_?setPixmap@QLabel@@UAEXABVQPixmap@@@Z 10008898     qt-mt323:qt-mt323.dll
 0002:0000089c       __imp_?setRadioButtonExclusive@QButtonGroup@@UAEX_N@Z 1000889c     qt-mt323:qt-mt323.dll
 0002:000008a0       __imp_?setResizeMode@QListView@@UAEXW4ResizeMode@1@@Z 100088a0     qt-mt323:qt-mt323.dll
 0002:000008a4       __imp_?setResizePolicy@QScrollView@@UAEXW4ResizePolicy@1@@Z 100088a4     qt-mt323:qt-mt323.dll
 0002:000008a8       __imp_?setRootIsDecorated@QListView@@UAEX_N@Z 100088a8     qt-mt323:qt-mt323.dll
 0002:000008ac       __imp_?setSelected@QListView@@UAEXPAVQListViewItem@@_N@Z 100088ac     qt-mt323:qt-mt323.dll
 0002:000008b0       __imp_?setShowSortIndicator@QListView@@UAEX_N@Z 100088b0     qt-mt323:qt-mt323.dll
 0002:000008b4       __imp_?setShowToolTips@QListView@@UAEX_N@Z 100088b4     qt-mt323:qt-mt323.dll
 0002:000008b8       __imp_?setSorting@QListView@@UAEXH_N@Z 100088b8     qt-mt323:qt-mt323.dll
 0002:000008bc       __imp_?setSpacing@QLayout@@UAEXH@Z 100088bc     qt-mt323:qt-mt323.dll
 0002:000008c0       __imp_?setState@QButton@@MAEXW4ToggleState@1@@Z 100088c0     qt-mt323:qt-mt323.dll
 0002:000008c4       __imp_?setText@QButton@@UAEXABVQString@@@Z 100088c4     qt-mt323:qt-mt323.dll
 0002:000008c8       __imp_?setText@QLabel@@UAEXABVQString@@@Z 100088c8     qt-mt323:qt-mt323.dll
 0002:000008cc       __imp_?setTitle@QGroupBox@@UAEXABVQString@@@Z 100088cc     qt-mt323:qt-mt323.dll
 0002:000008d0       __imp_?setToggleType@QButton@@MAEXW4ToggleType@1@@Z 100088d0     qt-mt323:qt-mt323.dll
 0002:000008d4       __imp_?setTreeStepSize@QListView@@UAEXH@Z 100088d4     qt-mt323:qt-mt323.dll
 0002:000008d8       __imp_?setVBarGeometry@QScrollView@@MAEXAAVQScrollBar@@HHHH@Z 100088d8     qt-mt323:qt-mt323.dll
 0002:000008dc       __imp_?setVScrollBarMode@QScrollView@@UAEXW4ScrollBarMode@1@@Z 100088dc     qt-mt323:qt-mt323.dll
 0002:000008e0       __imp_?show@QListView@@UAEXXZ 100088e0     qt-mt323:qt-mt323.dll
 0002:000008e4       __imp_?showEvent@QListView@@MAEXPAVQShowEvent@@@Z 100088e4     qt-mt323:qt-mt323.dll
 0002:000008e8       __imp_?sizeHint@QBoxLayout@@UBE?AVQSize@@XZ 100088e8     qt-mt323:qt-mt323.dll
 0002:000008ec       __imp_?sizeHint@QGroupBox@@UBE?AVQSize@@XZ 100088ec     qt-mt323:qt-mt323.dll
 0002:000008f0       __imp_?sizeHint@QHBox@@UBE?AVQSize@@XZ 100088f0     qt-mt323:qt-mt323.dll
 0002:000008f4       __imp_?sizeHint@QLabel@@UBE?AVQSize@@XZ 100088f4     qt-mt323:qt-mt323.dll
 0002:000008f8       __imp_?sizeHint@QListView@@UBE?AVQSize@@XZ 100088f8     qt-mt323:qt-mt323.dll
 0002:000008fc       __imp_?sizeHint@QPushButton@@UBE?AVQSize@@XZ 100088fc     qt-mt323:qt-mt323.dll
 0002:00000900       __imp_?sizeHint@QSpacerItem@@UBE?AVQSize@@XZ 10008900     qt-mt323:qt-mt323.dll
 0002:00000904       __imp_?sort@QListView@@UAEXXZ 10008904     qt-mt323:qt-mt323.dll
 0002:00000908       __imp_?spacerItem@QLayoutItem@@UAEPAVQSpacerItem@@XZ 10008908     qt-mt323:qt-mt323.dll
 0002:0000090c       __imp_?spacerItem@QSpacerItem@@UAEPAV1@XZ 1000890c     qt-mt323:qt-mt323.dll
 0002:00000910       __imp_?startDrag@QListView@@MAEXXZ 10008910     qt-mt323:qt-mt323.dll
 0002:00000914       __imp_?styleChange@QFrame@@MAEXAAVQStyle@@@Z 10008914     qt-mt323:qt-mt323.dll
 0002:00000918       __imp_?styleChange@QListView@@MAEXAAVQStyle@@@Z 10008918     qt-mt323:qt-mt323.dll
 0002:0000091c       __imp_?takeItem@QListView@@UAEXPAVQListViewItem@@@Z 1000891c     qt-mt323:qt-mt323.dll
 0002:00000920       __imp_?updateMask@QPushButton@@MAEXXZ 10008920     qt-mt323:qt-mt323.dll
 0002:00000924       __imp_?viewportContextMenuEvent@QScrollView@@MAEXPAVQContextMenuEvent@@@Z 10008924     qt-mt323:qt-mt323.dll
 0002:00000928       __imp_?viewportDragEnterEvent@QScrollView@@MAEXPAVQDragEnterEvent@@@Z 10008928     qt-mt323:qt-mt323.dll
 0002:0000092c       __imp_?viewportDragLeaveEvent@QScrollView@@MAEXPAVQDragLeaveEvent@@@Z 1000892c     qt-mt323:qt-mt323.dll
 0002:00000930       __imp_?viewportDragMoveEvent@QScrollView@@MAEXPAVQDragMoveEvent@@@Z 10008930     qt-mt323:qt-mt323.dll
 0002:00000934       __imp_?viewportDropEvent@QScrollView@@MAEXPAVQDropEvent@@@Z 10008934     qt-mt323:qt-mt323.dll
 0002:00000938       __imp_?viewportMouseDoubleClickEvent@QScrollView@@MAEXPAVQMouseEvent@@@Z 10008938     qt-mt323:qt-mt323.dll
 0002:0000093c       __imp_?viewportMouseMoveEvent@QScrollView@@MAEXPAVQMouseEvent@@@Z 1000893c     qt-mt323:qt-mt323.dll
 0002:00000940       __imp_?viewportMousePressEvent@QScrollView@@MAEXPAVQMouseEvent@@@Z 10008940     qt-mt323:qt-mt323.dll
 0002:00000944       __imp_?viewportMouseReleaseEvent@QScrollView@@MAEXPAVQMouseEvent@@@Z 10008944     qt-mt323:qt-mt323.dll
 0002:00000948       __imp_?viewportPaintEvent@QScrollView@@MAEXPAVQPaintEvent@@@Z 10008948     qt-mt323:qt-mt323.dll
 0002:0000094c       __imp_?viewportResizeEvent@QListView@@MAEXPAVQResizeEvent@@@Z 1000894c     qt-mt323:qt-mt323.dll
 0002:00000950       __imp_?viewportWheelEvent@QScrollView@@MAEXPAVQWheelEvent@@@Z 10008950     qt-mt323:qt-mt323.dll
 0002:00000954       __imp_?wheelEvent@QScrollView@@MAEXPAVQWheelEvent@@@Z 10008954     qt-mt323:qt-mt323.dll
 0002:00000958       __imp_?widget@QLayoutItem@@UAEPAVQWidget@@XZ 10008958     qt-mt323:qt-mt323.dll
 0002:0000095c       __imp_?windowActivationChange@QListView@@MAEX_N@Z 1000895c     qt-mt323:qt-mt323.dll
 0002:00000960       __imp_?qstrcmp@@YAHPBD0@Z  10008960     qt-mt323:qt-mt323.dll
 0002:00000964       __imp_?fromLatin1@QString@@SA?AV1@PBDH@Z 10008964     qt-mt323:qt-mt323.dll
 0002:00000968       __imp_?receivers@QObject@@IBEPAVQConnectionList@@H@Z 10008968     qt-mt323:qt-mt323.dll
 0002:0000096c       __imp_?activate_signal@QObject@@IAEXPAVQConnectionList@@PAUQUObject@@@Z 1000896c     qt-mt323:qt-mt323.dll
 0002:00000970       __imp_?staticMetaObject@QWidget@@SAPAVQMetaObject@@XZ 10008970     qt-mt323:qt-mt323.dll
 0002:00000974       __imp_?new_metaobject@QMetaObject@@SAPAV1@PBDPAV1@QBUQMetaData@@H2HQBVQMetaProperty@@HQBUQMetaEnum@@HQBUQClassInfo@@H@Z 10008974     qt-mt323:qt-mt323.dll
 0002:00000978       __imp_??0QMetaObjectCleanUp@@QAE@PBDP6APAVQMetaObject@@XZ@Z 10008978     qt-mt323:qt-mt323.dll
 0002:0000097c       __imp_??1QMetaObjectCleanUp@@QAE@XZ 1000897c     qt-mt323:qt-mt323.dll
 0002:00000980       __imp_?setMetaObject@QMetaObjectCleanUp@@QAEXAAPAVQMetaObject@@@Z 10008980     qt-mt323:qt-mt323.dll
 0002:00000984       __imp_?translate@QApplication@@QBE?AVQString@@PBD00W4Encoding@1@@Z 10008984     qt-mt323:qt-mt323.dll
 0002:00000988       __imp_??0QUObject@@QAE@XZ  10008988     qt-mt323:qt-mt323.dll
 0002:0000098c       __imp_??1QUObject@@QAE@XZ  1000898c     qt-mt323:qt-mt323.dll
 0002:00000990       __imp_?set@QUType_bool@@QAEXPAUQUObject@@_N@Z 10008990     qt-mt323:qt-mt323.dll
 0002:00000994       __imp_?set@QUType_QString@@QAEXPAUQUObject@@ABVQString@@@Z 10008994     qt-mt323:qt-mt323.dll
 0002:00000998       __imp_?qApp@@3PAVQApplication@@A 10008998     qt-mt323:qt-mt323.dll
 0002:0000099c       __imp_?static_QUType_bool@@3UQUType_bool@@A 1000899c     qt-mt323:qt-mt323.dll
 0002:000009a0       __imp_?static_QUType_QString@@3UQUType_QString@@A 100089a0     qt-mt323:qt-mt323.dll
 0002:000009a4       __imp_??1QIconSet@@UAE@XZ  100089a4     qt-mt323:qt-mt323.dll
 0002:000009a8       __imp_??0QKeySequence@@QAE@H@Z 100089a8     qt-mt323:qt-mt323.dll
 0002:000009ac       __imp_??0QIconSet@@QAE@ABVQPixmap@@W4Size@0@@Z 100089ac     qt-mt323:qt-mt323.dll
 0002:000009b0       __imp_??1QPixmap@@UAE@XZ   100089b0     qt-mt323:qt-mt323.dll
 0002:000009b4       __imp_??0QPixmap@@QAE@QAPBD@Z 100089b4     qt-mt323:qt-mt323.dll
 0002:000009b8       __imp_?critical@QMessageBox@@SAHPAVQWidget@@ABVQString@@1111HH@Z 100089b8     qt-mt323:qt-mt323.dll
 0002:000009bc       __imp_?information@QMessageBox@@SAHPAVQWidget@@ABVQString@@1111HH@Z 100089bc     qt-mt323:qt-mt323.dll
 0002:000009c0       __imp_?rect@QWidget@@QBE?AVQRect@@XZ 100089c0     qt-mt323:qt-mt323.dll
 0002:000009c4       __imp_?setName@QWidget@@UAEXPBD@Z 100089c4     qt-mt323:qt-mt323.dll
 0002:000009c8       __imp_??1QWidget@@UAE@XZ   100089c8     qt-mt323:qt-mt323.dll
 0002:000009cc       __imp_??0QWidget@@QAE@PAV0@PBDI@Z 100089cc     qt-mt323:qt-mt323.dll
 0002:000009d0       __imp_?latin1@QString@@QBEPBDXZ 100089d0     qt-mt323:qt-mt323.dll
 0002:000009d4       __imp_??1QStringList@@QAE@XZ 100089d4     qt-mt323:qt-mt323.dll
 0002:000009d8       __imp_?ascii@QString@@QBEPBDXZ 100089d8     qt-mt323:qt-mt323.dll
 0002:000009dc       __imp_?remove@QString@@QAEAAV1@ABV1@@Z 100089dc     qt-mt323:qt-mt323.dll
 0002:000009e0       __imp_?connect@QObject@@SA_NPBV1@PBD01@Z 100089e0     qt-mt323:qt-mt323.dll
 0002:000009e4       __imp_?clear@QGList@@MAEXXZ 100089e4     qt-mt323:qt-mt323.dll
 0002:000009e8       __imp_?append@QGList@@IAEXPAX@Z 100089e8     qt-mt323:qt-mt323.dll
 0002:000009ec       __imp_??1QGList@@MAE@XZ    100089ec     qt-mt323:qt-mt323.dll
 0002:000009f0       __imp_??0QGList@@IAE@XZ    100089f0     qt-mt323:qt-mt323.dll
 0002:000009f4       __imp_?detachInternal@?$QValueList@VQString@@@@AAEXXZ 100089f4     qt-mt323:qt-mt323.dll
 0002:000009f8       __imp_?contains@?$QValueList@VQString@@@@QBEIABVQString@@@Z 100089f8     qt-mt323:qt-mt323.dll
 0002:000009fc       __imp_?append@?$QValueList@VQString@@@@QAE?AV?$QValueListIterator@VQString@@@@ABVQString@@@Z 100089fc     qt-mt323:qt-mt323.dll
 0002:00000a00       __imp_?remove@?$QValueList@VQString@@@@QAEIABVQString@@@Z 10008a00     qt-mt323:qt-mt323.dll
 0002:00000a04       __imp_??H@YA?BVQString@@ABV0@D@Z 10008a04     qt-mt323:qt-mt323.dll
 0002:00000a08       __imp_??H@YA?BVQString@@PBDABV0@@Z 10008a08     qt-mt323:qt-mt323.dll
 0002:00000a0c       __imp_??H@YA?BVQString@@ABV0@PBD@Z 10008a0c     qt-mt323:qt-mt323.dll
 0002:00000a10       __imp_??H@YA?BVQString@@ABV0@0@Z 10008a10     qt-mt323:qt-mt323.dll
 0002:00000a14       __imp_??8@YA_NABVQString@@PBD@Z 10008a14     qt-mt323:qt-mt323.dll
 0002:00000a18       __imp_??8@YA_NABVQString@@0@Z 10008a18     qt-mt323:qt-mt323.dll
 0002:00000a1c       __imp_??9@YA_NABVQString@@0@Z 10008a1c     qt-mt323:qt-mt323.dll
 0002:00000a20       __imp_?endsWith@QString@@QBE_NABV1@@Z 10008a20     qt-mt323:qt-mt323.dll
 0002:00000a24       __imp_?text@QListViewItem@@UBE?AVQString@@H@Z 10008a24     qt-mt323:qt-mt323.dll
 0002:00000a28       __imp_?startsWith@QString@@QBE_NABV1@@Z 10008a28     qt-mt323:qt-mt323.dll
 0002:00000a2c       __imp_?insert@QString@@QAEAAV1@IABV1@@Z 10008a2c     qt-mt323:qt-mt323.dll
 0002:00000a30       __imp_??4QString@@QAEAAV0@PBD@Z 10008a30     qt-mt323:qt-mt323.dll
 0002:00000a34       __imp_??4QString@@QAEAAV0@ABV0@@Z 10008a34     qt-mt323:qt-mt323.dll
 0002:00000a38       __imp_??1QString@@QAE@XZ   10008a38     qt-mt323:qt-mt323.dll
 0002:00000a3c       __imp_??0QString@@QAE@PBD@Z 10008a3c     qt-mt323:qt-mt323.dll
 0002:00000a40       __imp_??0QString@@QAE@ABV0@@Z 10008a40     qt-mt323:qt-mt323.dll
 0002:00000a44       __imp_??0QString@@QAE@XZ   10008a44     qt-mt323:qt-mt323.dll
 0002:00000a48       __imp_?takeItem@QListViewItem@@UAEXPAV1@@Z 10008a48     qt-mt323:qt-mt323.dll
 0002:00000a4c       __imp_?qDebug@@YAXPBDZZ    10008a4c     qt-mt323:qt-mt323.dll
 0002:00000a50       \177qt-mt323_NULL_THUNK_DATA 10008a50     qt-mt323:qt-mt323.dll
 0002:00000a54       ___xc_a                    10008a54     MSVCRT:cinitexe.obj
 0002:00000a64       ___xc_z                    10008a64     MSVCRT:cinitexe.obj
 0002:00000a68       ___xi_a                    10008a68     MSVCRT:cinitexe.obj
 0002:00000a74       ___xi_z                    10008a74     MSVCRT:cinitexe.obj
 0002:00000a80       ??_C@_0CD@BFGBAEB@?5?5?5?514?5?5?5?514?5?5?5?5?5?5?5?54?5?5?5?5?5?5?5?5?5?5?5@ 10008a80     cfg_alarm_overview.obj
 0002:00000aa4       ??_C@_0M@EKMPMHDK@?4?5c?5?$CD040404?$AA@ 10008aa4     cfg_alarm_overview.obj
 0002:00000ab0       ??_C@_0M@NBLJLJNN@?$CD?5c?5?$CD808304?$AA@ 10008ab0     cfg_alarm_overview.obj
 0002:00000abc       ??_C@_0M@EAFJJBBG@a?5c?5?$CDbfc2bf?$AA@ 10008abc     cfg_alarm_overview.obj
 0002:00000ac8       ??_C@_08PBKCALNO@b?5c?5None?$AA@ 10008ac8     cfg_alarm_overview.obj
 0002:00000ad4       ??_C@_0P@HFKAALMG@?4?4?4?4?4?4?4?4?4?4?4?4?4?4?$AA@ 10008ad4     cfg_alarm_overview.obj
 0002:00000ae4       ??_C@_0P@LGBCEGMD@?4?$CD?4aaaaaaaa?4a?4?$AA@ 10008ae4     cfg_alarm_overview.obj
 0002:00000af4       ??_C@_0P@MNNEIMDO@?4?$CD?4aaaaaaaa?4?4?4?$AA@ 10008af4     cfg_alarm_overview.obj
 0002:00000b04       ??_C@_0P@MFAMBPGN@?4?$CD?4aaaaaaaa?4?$CD?4?$AA@ 10008b04     cfg_alarm_overview.obj
 0002:00000b14       ??_C@_0P@HPMEFAGN@?4?$CD?$CD?4?4?4?4?4?4?4?4?$CD?$CD?4?$AA@ 10008b14     cfg_alarm_overview.obj
 0002:00000b24       ??_C@_0P@JAJCNDBN@?4?$CD?$CD?$CD?$CD?$CD?$CD?$CD?$CD?$CD?$CD?$CD?$CD?4?$AA@ 10008b24     cfg_alarm_overview.obj
 0002:00000b34       ??_C@_0P@INKOIILA@?4?$CD?$CD?4?4?4?4?4?4?4?4?4?$CD?4?$AA@ 10008b34     cfg_alarm_overview.obj
 0002:00000b44       ??_C@_0P@KJADPPJB@?4?$CD?$CD?4?4?4?4?4?4aa?4?$CD?4?$AA@ 10008b44     cfg_alarm_overview.obj
 0002:00000b54       ??_C@_0P@PKKONJFP@b?4?4?4?4?4?4?4?4?4?4?4?4?4?$AA@ 10008b54     cfg_alarm_overview.obj
 0002:00000b64       ??_C@_09KDLGOOHH@16?516?54?51?$AA@ 10008b64     cfg_alarm_overview.obj
 0002:00000b70       ??_C@_0M@KEPPNGJB@?$CD?5c?5?$CD000000?$AA@ 10008b70     cfg_alarm_overview.obj
 0002:00000b7c       ??_C@_0M@BCKHMLG@b?5c?5?$CD000080?$AA@ 10008b7c     cfg_alarm_overview.obj
 0002:00000b88       ??_C@_08IMFNEMJ@?4?5c?5none?$AA@ 10008b88     cfg_alarm_overview.obj
 0002:00000b94       ??_C@_0M@DPJAAKFM@a?5c?5?$CDffffff?$AA@ 10008b94     cfg_alarm_overview.obj
 0002:00000ba0       ??_C@_0BB@DDKGLOCG@?4?4?4?4?4?4?4?4?4?4?4?4?4?4?4?4?$AA@ 10008ba0     cfg_alarm_overview.obj
 0002:00000bb4       ??_C@_0BB@GDAPNCLP@?4?$CD?$CD?$CD?$CD?$CD?$CD?4?4?4?4?4?4?4?4?4?$AA@ 10008bb4     cfg_alarm_overview.obj
 0002:00000bc8       ??_C@_0BB@FFNCKNDA@?4?$CDaaaa?$CD?$CD?4?4?4?4?4?4?4?4?$AA@ 10008bc8     cfg_alarm_overview.obj
 0002:00000bdc       ??_C@_0BB@DONCJNPK@?4?$CDaaaa?$CDa?$CD?4?4?4?4?4?4?4?$AA@ 10008bdc     cfg_alarm_overview.obj
 0002:00000bf0       ??_C@_0BB@HJAKJBPB@?4?$CDa?$CD?$CDa?$CDbbbbbb?4?4?4?$AA@ 10008bf0     cfg_alarm_overview.obj
 0002:00000c04       ??_C@_0BB@FLJEJCPD@?4?$CDaaaaabaaaabb?4?4?$AA@ 10008c04     cfg_alarm_overview.obj
 0002:00000c18       ??_C@_0BB@BPNLNHEE@?4?$CDa?$CD?$CD?$CD?$CDbaaaabab?4?$AA@ 10008c18     cfg_alarm_overview.obj
 0002:00000c2c       ??_C@_0BB@MGPEEHJO@?4?$CDaaaaaba?$CD?$CDabbbb?$AA@ 10008c2c     cfg_alarm_overview.obj
 0002:00000c40       ??_C@_0BB@GPBBDME@?4?$CDa?$CD?$CD?$CD?$CDbaaaaaaab?$AA@ 10008c40     cfg_alarm_overview.obj
 0002:00000c54       ??_C@_0BB@MABJBMAB@?4?$CDaaaaaba?$CD?$CD?$CD?$CD?$CDab?$AA@ 10008c54     cfg_alarm_overview.obj
 0002:00000c68       ??_C@_0BB@GEIMNJCI@?4?$CD?$CD?$CD?$CD?$CD?$CDbaaaaaaab?$AA@ 10008c68     cfg_alarm_overview.obj
 0002:00000c7c       ??_C@_0BB@NNLHCEIJ@?4?4?4?4?4?4?4ba?$CD?$CD?$CD?$CD?$CDab?$AA@ 10008c7c     cfg_alarm_overview.obj
 0002:00000c90       ??_C@_0BB@DECFLFLB@?4?4?4?4?4?4?4baaaaaaab?$AA@ 10008c90     cfg_alarm_overview.obj
 0002:00000ca4       ??_C@_0BB@GDAIINMD@?4?4?4?4?4?4?4bbbbbbbbb?$AA@ 10008ca4     cfg_alarm_overview.obj
 0002:00000cb8       ??_C@_09OJGAFBMP@16?516?58?51?$AA@ 10008cb8     cfg_alarm_overview.obj
 0002:00000cc4       ??_C@_0M@HFLCJFDJ@e?5c?5?$CD000080?$AA@ 10008cc4     cfg_alarm_overview.obj
 0002:00000cd0       ??_C@_0M@JHADGEMH@c?5c?5?$CD808000?$AA@ 10008cd0     cfg_alarm_overview.obj
 0002:00000cdc       ??_C@_0M@CLFHJBA@b?5c?5?$CD808080?$AA@ 10008cdc     cfg_alarm_overview.obj
 0002:00000ce8       ??_C@_0M@MHLPHELG@d?5c?5?$CDd4d0c8?$AA@ 10008ce8     cfg_alarm_overview.obj
 0002:00000cf4       ??_C@_0M@LLEAKCIM@a?5c?5?$CDffff00?$AA@ 10008cf4     cfg_alarm_overview.obj
 0002:00000d00       ??_C@_0M@ELAIODND@f?5c?5?$CDffffff?$AA@ 10008d00     cfg_alarm_overview.obj
 0002:00000d0c       ??_C@_0BB@GHIGIKBH@?4?4?4?4?4?4?$CD?$CD?$CD?$CD?4?4?4?4?4?4?$AA@ 10008d0c     cfg_alarm_overview.obj
 0002:00000d20       ??_C@_0BB@EIGJHLLO@?4?4?$CD?$CD?$CD?$CD?$CDaa?$CD?$CD?$CD?$CD?$CD?4?4?$AA@ 10008d20     cfg_alarm_overview.obj
 0002:00000d34       ??_C@_0BB@GFDBAPPE@?4?$CDbcb?$CDa?$CD?$CDa?$CDcbc?$CD?4?$AA@ 10008d34     cfg_alarm_overview.obj
 0002:00000d48       ??_C@_0BB@JBCPPMEE@?4?$CDcb?$CDdddddd?$CDcb?$CD?4?$AA@ 10008d48     cfg_alarm_overview.obj
 0002:00000d5c       ??_C@_0BB@OPOOCIAI@?4?$CDbc?$CD?$CD?$CD?$CD?$CD?$CD?$CD?$CDbc?$CD?4?$AA@ 10008d5c     cfg_alarm_overview.obj
 0002:00000d70       ??_C@_0BB@EEBHCOMC@?4?$CDcbcbcbcbcbcb?$CD?4?$AA@ 10008d70     cfg_alarm_overview.obj
 0002:00000d84       ??_C@_0BB@BABPPNAH@?4?$CDbcbcbeeeeeee?$CD?4?$AA@ 10008d84     cfg_alarm_overview.obj
 0002:00000d98       ??_C@_0BB@IAJPFFAE@?4?$CDcbcbcefffffee?4?$AA@ 10008d98     cfg_alarm_overview.obj
 0002:00000dac       ??_C@_0BB@DCBNANCH@?4?$CDbcbcbefffffefe?$AA@ 10008dac     cfg_alarm_overview.obj
 0002:00000dc0       ??_C@_0BB@KKOBKMBK@?4?$CDcbcbcefeeefeee?$AA@ 10008dc0     cfg_alarm_overview.obj
 0002:00000dd4       ??_C@_0BB@CAKIKCMJ@?4?$CDbcbcbefffffffe?$AA@ 10008dd4     cfg_alarm_overview.obj
 0002:00000de8       ??_C@_0BB@OPAHGIJD@?4?$CDcbcbcefeeeeefe?$AA@ 10008de8     cfg_alarm_overview.obj
 0002:00000dfc       ??_C@_0BB@FMOFIOAF@?4?4?$CD?$CD?$CD?$CD?$CDefffffffe?$AA@ 10008dfc     cfg_alarm_overview.obj
 0002:00000e10       ??_C@_0BB@FCCLJILH@?4?4?4?4?4?4?4eeeeeeeee?$AA@ 10008e10     cfg_alarm_overview.obj
 0002:00000e24       ??_C@_09DOGBNGMO@16?516?53?51?$AA@ 10008e24     cfg_alarm_overview.obj
 0002:00000e30       ??_C@_0M@KKOMIHCJ@?$CD?5c?5?$CD000080?$AA@ 10008e30     cfg_alarm_overview.obj
 0002:00000e3c       ??_C@_0M@HFCLKLOA@a?5c?5?$CD808080?$AA@ 10008e3c     cfg_alarm_overview.obj
 0002:00000e48       ??_C@_0BB@DDMLBOGJ@?4?4?4?4?4?4?4?$CD?$CD?$CD?$CDa?4?4?4?4?$AA@ 10008e48     cfg_alarm_overview.obj
 0002:00000e5c       ??_C@_0BB@JOKGMNA@?4?$CD?4?4?4?$CD?$CD?4?4?4?4?$CDa?4?4?4?$AA@ 10008e5c     cfg_alarm_overview.obj
 0002:00000e70       ??_C@_0BB@HJFOCKLM@?4?$CD?$CD?4?$CD?4?4?4?4?4?4?4?$CD?4?4?4?$AA@ 10008e70     cfg_alarm_overview.obj
 0002:00000e84       ??_C@_0BB@IJIIDKJJ@?4?$CD?$CD?$CD?4?4?4?4?4?4?4?4?$CD?4?4?4?$AA@ 10008e84     cfg_alarm_overview.obj
 0002:00000e98       ??_C@_0BB@MOKEFKOH@?4?$CD?$CD?$CD?$CD?4?4?4?4?4?4?4?$CD?4?4?4?$AA@ 10008e98     cfg_alarm_overview.obj
 0002:00000eac       ??_C@_0BB@MOKGEDPO@?4?$CD?$CD?$CD?$CD?$CD?4?4?4?4?4?$CDa?4?4?4?$AA@ 10008eac     cfg_alarm_overview.obj
 0002:00000ec0       ??_C@_0BB@DNHLKIGI@?4?4?4?4?4?4?4?4?4?4a?$CD?4?4?4?4?$AA@ 10008ec0     cfg_alarm_overview.obj
 0002:00000ed4       ??_C@_02GIPFHKNO@OK?$AA@   10008ed4     cfg_alarm_overview.obj
 0002:00000edc       ??_SQAction@@6B@           10008edc     cfg_alarm_overview.obj
 0002:00000f6c       ??_SQToolBar@@6BQObject@@@ 10008f6c     cfg_alarm_overview.obj
 0002:00001188       ??_SQToolBar@@6BQPaintDevice@@@ 10009188     cfg_alarm_overview.obj
 0002:000011ac       ??_SQListViewItem@@6B@     100091ac     cfg_alarm_overview.obj
 0002:00001248       ??_7QDockWindowList@@6B@   10009248     cfg_alarm_overview.obj
 0002:0000126c       ??_SQPopupMenu@@6BQObject@@@ 1000926c     cfg_alarm_overview.obj
 0002:0000144c       ??_SQPopupMenu@@6BQPaintDevice@@@ 1000944c     cfg_alarm_overview.obj
 0002:00001470       ??_SQPopupMenu@@6B@        10009470     cfg_alarm_overview.obj
 0002:00001494       ??_7?$QPtrList@VQPopupMenu@@@@6B@ 10009494     cfg_alarm_overview.obj
 0002:000014b8       ??_7QPopupMenuList@@6B@    100094b8     cfg_alarm_overview.obj
 0002:000014dc       ??_SQGuardedPtrPrivate@@6B@ 100094dc     cfg_alarm_overview.obj
 0002:00001530       ??_7config_plugin_base@@6BQObject@@@ 10009530     cfg_alarm_overview.obj
 0002:00001708       ??_7config_plugin_base@@6BQPaintDevice@@@ 10009708     cfg_alarm_overview.obj
 0002:00001728       ??_C@_0EB@GNDACMDJ@?$CC?5?9?5the?5author?5should?5have?5defin@ 10009728     cfg_alarm_overview.obj
 0002:0000176c       ??_C@_0CH@BDPDPLDP@This?5is?5the?5default?5?$CCAbout?$CC?5text@ 1000976c     cfg_alarm_overview.obj
 0002:00001798       ??_7?$QDict@VQAction@@@@6B@ 10009798     cfg_alarm_overview.obj
 0002:000017b8       ??_7?$QPtrList@VCInputFile@@@@6B@ 100097b8     cfg_alarm_overview.obj
 0002:000017dc       ??_7?$QPtrList@VCOutputFile@@@@6B@ 100097dc     cfg_alarm_overview.obj
 0002:00001800       ??_7cfg_alarm_overview@@6BQObject@@@ 10009800     cfg_alarm_overview.obj
 0002:000019d8       ??_7cfg_alarm_overview@@6BQPaintDevice@@@ 100099d8     cfg_alarm_overview.obj
 0002:000019f8       ??_C@_0BC@IMJEOOJP@config?1myfile?4txt?$AA@ 100099f8     cfg_alarm_overview.obj
 0002:00001a0c       ??_C@_09DBJAPGHN@?1textedit?$AA@ 10009a0c     cfg_alarm_overview.obj
 0002:00001a18       ??_C@_05LHMKEDEH@?$CGEdit?$AA@ 10009a18     cfg_alarm_overview.obj
 0002:00001a20       ??_C@_03CLCAEGCJ@new?$AA@  10009a20     cfg_alarm_overview.obj
 0002:00001a24       ??_C@_0BC@EEBCDLBD@?$CGNew?5Alarm?5System?$AA@ 10009a24     cfg_alarm_overview.obj
 0002:00001a38       ??_C@_07EJAINBEK@filenew?$AA@ 10009a38     cfg_alarm_overview.obj
 0002:00001a40       ??_C@_0BB@LJNMABFG@New?5Alarm?5System?$AA@ 10009a40     cfg_alarm_overview.obj
 0002:00001a54       ??_C@_0BB@JKFKKCEC@1menuNewSystem?$CI?$CJ?$AA@ 10009a54     cfg_alarm_overview.obj
 0002:00001a68       ??_C@_0N@KCMOKDBB@2activated?$CI?$CJ?$AA@ 10009a68     cfg_alarm_overview.obj
 0002:00001a78       ??_C@_06FOBLBEIN@delete?$AA@ 10009a78     cfg_alarm_overview.obj
 0002:00001a80       ??_C@_0BF@LKGBFPNM@?$CGDelete?5Alarm?5System?$AA@ 10009a80     cfg_alarm_overview.obj
 0002:00001a98       ??_C@_0L@BPDPNFLB@filedelete?$AA@ 10009a98     cfg_alarm_overview.obj
 0002:00001aa4       ??_C@_0BE@JFEFCBME@Delete?5Alarm?5System?$AA@ 10009aa4     cfg_alarm_overview.obj
 0002:00001ab8       ??_C@_0BP@KFJPMMLE@1selectSystem?$CIconst?5QString?5?$CG?$CJ?$AA@ 10009ab8     cfg_alarm_overview.obj
 0002:00001ad8       ??_C@_0BN@DDAIKEMB@2sysChanged?$CIconst?5QString?5?$CG?$CJ?$AA@ 10009ad8     cfg_alarm_overview.obj
 0002:00001af8       ??_C@_0BD@CJEHHDCP@1NavigatetoInput?$CI?$CJ?$AA@ 10009af8     cfg_alarm_overview.obj
 0002:00001b0c       ??_C@_0L@OELOHDKG@2clicked?$CI?$CJ?$AA@ 10009b0c     cfg_alarm_overview.obj
 0002:00001b18       ??_C@_0BD@GKDKEFEA@1NavigatetoProcs?$CI?$CJ?$AA@ 10009b18     cfg_alarm_overview.obj
 0002:00001b2c       ??_C@_0BE@KEIOPHAL@1NavigatetoOutput?$CI?$CJ?$AA@ 10009b2c     cfg_alarm_overview.obj
 0002:00001b40       ??_C@_0BD@JBOFMGJF@1createNewSystem?$CI?$CJ?$AA@ 10009b40     cfg_alarm_overview.obj
 0002:00001b54       ??_C@_06BNCCALCL@unlock?$AA@ 10009b54     cfg_alarm_overview.obj
 0002:00001b5c       ??_C@_08HNIAHLMM@download?$AA@ 10009b5c     cfg_alarm_overview.obj
 0002:00001b68       ??_C@_07MPPKIBJA@Error?3?6?$AA@ 10009b68     cfg_alarm_overview.obj
 0002:00001b70       ??_C@_05NAOIJFC@Error?$AA@ 10009b70     cfg_alarm_overview.obj
 0002:00001b78       ??_C@_07GEICGNKI@?1inputs?$AA@ 10009b78     cfg_alarm_overview.obj
 0002:00001b80       ??_C@_01KMDKNFGN@?1?$AA@   10009b80     cfg_alarm_overview.obj
 0002:00001b84       ??_C@_0O@MIFBLPDN@config?1alarms?$AA@ 10009b84     cfg_alarm_overview.obj
 0002:00001b94       ??_C@_08MKHFJBNK@?1inputs?1?$AA@ 10009b94     cfg_alarm_overview.obj
 0002:00001ba0       ??_C@_07NCIDFJOM@al_acq_?$AA@ 10009ba0     cfg_alarm_overview.obj
 0002:00001ba8       ??_C@_04IFJILJI@?4cfg?$AA@ 10009ba8     cfg_alarm_overview.obj
 0002:00001bad       ??_C@_00CNPNBAHC@?$AA@     10009bad     cfg_alarm_overview.obj
 0002:00001bb0       ??_C@_0L@FGNBINDG@ConfigTool?$AA@ 10009bb0     cfg_alarm_overview.obj
 0002:00001bbc       ??_C@_06JIODDOFH@System?$AA@ 10009bbc     cfg_alarm_overview.obj
 0002:00001bc4       ??_C@_04FABLJDN@Name?$AA@  10009bc4     cfg_alarm_overview.obj
 0002:00001bcc       ??_C@_08JBEPPOLH@?1outputs?$AA@ 10009bcc     cfg_alarm_overview.obj
 0002:00001bd8       ??_C@_09EHIIFBLM@?1outputs?1?$AA@ 10009bd8     cfg_alarm_overview.obj
 0002:00001be4       ??_C@_07BOAKCNCF@al_out_?$AA@ 10009be4     cfg_alarm_overview.obj
 0002:00001bec       ??_C@_0CN@EINONBEA@Download?5DONE?5for?5?8?$CFs?8?5create?5st@ 10009bec     cfg_alarm_overview.obj
 0002:00001c1c       ??_C@_04MKMCLCOO@lock?$AA@ 10009c1c     cfg_alarm_overview.obj
 0002:00001c24       ??_C@_0CC@OAGIAEAC@?6File?5will?5be?5available?5read?5onl@ 10009c24     cfg_alarm_overview.obj
 0002:00001c48       ??_C@_03NLJIHOMM@?5?9?5?$AA@ 10009c48     cfg_alarm_overview.obj
 0002:00001c4c       ??_C@_06JGFHLLHI@Lock?3?5?$AA@ 10009c4c     cfg_alarm_overview.obj
 0002:00001c54       ??_C@_04LADJNOK@Lock?$AA@  10009c54     cfg_alarm_overview.obj
 0002:00001c5c       ??_C@_0BA@HFGNGHNM@Got?5Lock?5for?5?$CFs?$AA@ 10009c5c     cfg_alarm_overview.obj
 0002:00001c6c       ??_C@_06KAOCKAGB@upload?$AA@ 10009c6c     cfg_alarm_overview.obj
 0002:00001c74       ??_C@_0BC@CLBPNFHH@reply?5from?5upload?$AA@ 10009c74     cfg_alarm_overview.obj
 0002:00001c88       ??_C@_03DAPAKLGM@dir?$AA@  10009c88     cfg_alarm_overview.obj
 0002:00001c8c       ??_C@_05CCAMFJOL@clean?$AA@ 10009c8c     cfg_alarm_overview.obj
 0002:00001c94       ??_C@_0BD@NLCMHLGP@UNLOCK?5RESPONSE?5?$CFs?$AA@ 10009c94     cfg_alarm_overview.obj
 0002:00001ca8       ??_C@_0CO@DMDPGOMC@Being?5asked?5to?5navigate?5to?5?$CFs?5wi@ 10009ca8     cfg_alarm_overview.obj
 0002:00001cd8       ??_C@_0CM@OJDNOHDO@ALARM?5OVERALL?3?9?5?9ACTIVATE?5ME?5?9?5r@ 10009cd8     cfg_alarm_overview.obj
 0002:00001d04       ??_C@_0BC@JENMCOAN@?$CFd?5dirs?5to?5upload?$AA@ 10009d04     cfg_alarm_overview.obj
 0002:00001d18       ??_C@_0O@JFGJGFB@syncDirUpload?$AA@ 10009d18     cfg_alarm_overview.obj
 0002:00001d28       ??_C@_0BH@DPGKGIAN@UPLOADING?5Directory?5?$CFs?$AA@ 10009d28     cfg_alarm_overview.obj
 0002:00001d40       ??_C@_0BI@LFOFOHH@Home?1Alarms?1Processes?0?5?$AA@ 10009d40     cfg_alarm_overview.obj
 0002:00001d58       ??_C@_08NCKPMOJE@navigate?$AA@ 10009d58     cfg_alarm_overview.obj
 0002:00001d64       ??_C@_0CH@JEBNGFIJ@Home?1Alarms?1Inputs?1cBNCS?5acquisi@ 10009d64     cfg_alarm_overview.obj
 0002:00001d8c       ??_C@_0CC@DCALHEBN@Home?1Alarms?1Outputs?1Bncs?5Output?0@ 10009d8c     cfg_alarm_overview.obj
 0002:00001db0       ??_C@_0BP@PIGHFONH@Home?1Alarms?1Outputs?1Database?0?5?$AA@ 10009db0     cfg_alarm_overview.obj
 0002:00001dd0       ??_C@_0DH@LBLKAOKI@ALARM?5OVERVIEW?5?5?9?5this?5is?5where?5@ 10009dd0     cfg_alarm_overview.obj
 0002:00001e08       ??_C@_0EB@CCFIPFO@ALARM?5OVERVIEW?5?9?5select?5system?5?9@ 10009e08     cfg_alarm_overview.obj
 0002:00001e4c       ??_C@_0BA@GNHMHBBC@syncDirDownload?$AA@ 10009e4c     cfg_alarm_overview.obj
 0002:00001e5c       ??_C@_0CB@JJNKHNCK@Nav?5to?5inputs?5tool?5?9?5?$CFs?0?5file?5?$CFs@ 10009e5c     cfg_alarm_overview.obj
 0002:00001e80       ??_C@_02LNAEAIDO@?$DL?5?$AA@ 10009e80     cfg_alarm_overview.obj
 0002:00001e84       ??_C@_01IHBHIGKO@?0?$AA@   10009e84     cfg_alarm_overview.obj
 0002:00001e88       ??_C@_0CC@FEOJNPF@Nav?5to?5outputs?5tool?5?9?5?$CFs?0?5file?5?$CF@ 10009e88     cfg_alarm_overview.obj
 0002:00001eac       ??_C@_0BP@IPJCMMAH@AL?5OVERVIEW?3?3Create?5New?5System?$AA@ 10009eac     cfg_alarm_overview.obj
 0002:00001ecc       ??_C@_0CI@PNLLFHOM@Enter?5the?5name?5for?5the?5New?5Alarm@ 10009ecc     cfg_alarm_overview.obj
 0002:00001ef4       ??_C@_0O@LOPHJEJO@Alarms?5Config?$AA@ 10009ef4     cfg_alarm_overview.obj
 0002:00001f04       ??_C@_0BE@JHCKMJAD@Checking?5out?5DIR?5?$CFs?$AA@ 10009f04     cfg_alarm_overview.obj
 0002:00001f18       ??_C@_0M@IKGKPMGN@checkoutDir?$AA@ 10009f18     cfg_alarm_overview.obj
 0002:00001f24       ??_C@_0BO@POGOIAFB@AL?5OVERALL?3?3MMMMMMmarkDirty?$CI?$CJ?$AA@ 10009f24     cfg_alarm_overview.obj
 0002:00001f44       ??_C@_05CFEJGMAI@dirty?$AA@ 10009f44     cfg_alarm_overview.obj
 0002:00001f4c       ??_C@_0N@LEBPCLIG@proc_def?4cfg?$AA@ 10009f4c     cfg_alarm_overview.obj
 0002:00001f5c       ??_C@_0BI@OGOMDAHM@CREATE?5NEW?5DIRECTORY?5?$CFs?$AA@ 10009f5c     cfg_alarm_overview.obj
 0002:00001f74       ??_C@_06HEJKKHEK@config?$AA@ 10009f74     cfg_alarm_overview.obj
 0002:00001f7c       ??_C@_0CA@KFPINNDD@Config?5DIR?5doesn?8t?5exist?$CB?$CB?$CB?$CB?5?$CFs?$AA@ 10009f7c     cfg_alarm_overview.obj
 0002:00001f9c       ??_C@_06BBBNOMFN@alarms?$AA@ 10009f9c     cfg_alarm_overview.obj
 0002:00001fa4       ??_C@_0CF@PCLBGGFK@ALARM?5DIR?5doesn?8t?5exist?5?9?5create@ 10009fa4     cfg_alarm_overview.obj
 0002:00001fcc       ??_C@_03GJCOJFLC@?4?6?6?$AA@ 10009fcc     cfg_alarm_overview.obj
 0002:00001fd0       ??_C@_0BM@CGOIHJMM@Could?5not?5Create?5directory?6?$AA@ 10009fd0     cfg_alarm_overview.obj
 0002:00001fec       ??_C@_0P@JCFHGIHA@Alarms?1Overall?$AA@ 10009fec     cfg_alarm_overview.obj
 0002:00001ffc       ??_C@_0BD@FLDAKHPB@New?5System?5Created?$AA@ 10009ffc     cfg_alarm_overview.obj
 0002:00002010       ??_C@_0BE@NNKFNLDF@Created?5Proc?5Def?5OK?$AA@ 1000a010     cfg_alarm_overview.obj
 0002:00002024       ??_C@_0BK@KENGENMD@FAILED?5to?5create?5proc_def?$AA@ 1000a024     cfg_alarm_overview.obj
 0002:00002040       ??_C@_0DG@NNMIHGBJ@?$CK?9?$CK?9?$CK?9?$CK?9?$CK?5Failed?5to?5create?5direc@ 1000a040     cfg_alarm_overview.obj
 0002:0000207c       ??_7dialog@@6BQObject@@@   1000a07c     dialogimpl.obj
 0002:00002234       ??_7dialog@@6BQPaintDevice@@@ 1000a234     dialogimpl.obj
 0002:00002258       ??_7CInputFile@@6B@        1000a258     InputFile.obj
 0002:00002260       ??_7COutputFile@@6B@       1000a260     OutputFile.obj
 0002:00002264       ??_C@_09HOMOKAL@15?516?53?51?$AA@ 1000a264     plugindesc.obj
 0002:00002270       ??_C@_0M@OCHFMIJJ@a?5c?5?$CDff0000?$AA@ 1000a270     plugindesc.obj
 0002:0000227c       ??_C@_0BA@HJHFMOKC@?4?4?4?4?4?4?4?4?4?4?4?4?4?4?4?$AA@ 1000a27c     plugindesc.obj
 0002:0000228c       ??_C@_0BA@HNMEKCEF@?4?4?4?4?4?4?$CD?$CD?4?4?4?4?4?4?4?$AA@ 1000a28c     plugindesc.obj
 0002:0000229c       ??_C@_0BA@LIAGGGKB@?4?4?4?4?$CD?$CDaa?$CD?$CD?4?4?4?4?4?$AA@ 1000a29c     plugindesc.obj
 0002:000022ac       ??_C@_0BA@KJOEDNIA@?4?4?4?$CDaaaaaa?$CD?4?4?4?4?$AA@ 1000a2ac     plugindesc.obj
 0002:000022bc       ??_C@_0BA@HJMPAGON@?4?4?$CDaaaaaaaa?$CD?4?4?4?$AA@ 1000a2bc     plugindesc.obj
 0002:000022cc       ??_C@_0BA@PFEPJEEJ@?4?$CDaaaaaaaaaa?$CD?4?4?$AA@ 1000a2cc     plugindesc.obj
 0002:000022dc       ??_C@_0BA@GIJBPHCG@?4?$CD?$CD?$CD?$CD?$CD?$CD?$CD?$CD?$CD?$CD?$CD?$CD?4?4?$AA@ 1000a2dc     plugindesc.obj
 0002:000022ec       ??_C@_0BA@BHOPFOFJ@?4?4?4?4?4?4aa?4?4?4?4?4?4?4?$AA@ 1000a2ec     plugindesc.obj
 0002:00002300       ??_7config_plugin_desc_base@@6B@ 1000a300     plugindesc.obj
 0002:00002314       ??_7plugindesc@@6B@        1000a314     plugindesc.obj
 0002:00002324       ??_C@_0BF@ECKGKBLE@Home?1Alarms?1Overview?$AA@ 1000a324     plugindesc.obj
 0002:00002340       ??_7dialogBase@@6BQObject@@@ 1000a340     dialog.obj
 0002:000024f8       ??_7dialogBase@@6BQPaintDevice@@@ 1000a4f8     dialog.obj
 0002:0000251c       ??_SQPushButton@@6BQObject@@@ 1000a51c     dialog.obj
 0002:0000270c       ??_SQPushButton@@6BQPaintDevice@@@ 1000a70c     dialog.obj
 0002:00002734       ??_SQButtonGroup@@6BQObject@@@ 1000a734     dialog.obj
 0002:00002924       ??_SQButtonGroup@@6BQPaintDevice@@@ 1000a924     dialog.obj
 0002:0000294c       ??_SQLabel@@6BQObject@@@   1000a94c     dialog.obj
 0002:00002b44       ??_SQLabel@@6BQPaintDevice@@@ 1000ab44     dialog.obj
 0002:00002b6c       ??_SQListView@@6BQObject@@@ 1000ab6c     dialog.obj
 0002:00002e50       ??_SQListView@@6BQPaintDevice@@@ 1000ae50     dialog.obj
 0002:00002e74       ??_SQSpacerItem@@6B@       1000ae74     dialog.obj
 0002:00002ebc       ??_SQHBoxLayout@@6BQObject@@@ 1000aebc     dialog.obj
 0002:00002f24       ??_SQHBoxLayout@@6BQLayoutItem@@@ 1000af24     dialog.obj
 0002:00002f6c       ??_SQVBoxLayout@@6BQObject@@@ 1000af6c     dialog.obj
 0002:00002fd4       ??_SQVBoxLayout@@6BQLayoutItem@@@ 1000afd4     dialog.obj
 0002:0000301c       ??_SCAlm_sys_select@@6BQObject@@@ 1000b01c     dialog.obj
 0002:000031f0       ??_SCAlm_sys_select@@6BQPaintDevice@@@ 1000b1f0     dialog.obj
 0002:00003210       ??_C@_0L@BCEAHFEK@dialogBase?$AA@ 1000b210     dialog.obj
 0002:0000321c       ??_C@_0BB@NFKKNJMG@dialogBaseLayout?$AA@ 1000b21c     dialog.obj
 0002:00003230       ??_C@_0O@GLGNKJNI@sSystemSelect?$AA@ 1000b230     dialog.obj
 0002:00003240       ??_C@_0O@PAOANHBM@buttonGroup18?$AA@ 1000b240     dialog.obj
 0002:00003250       ??_C@_0O@NCLNPPKP@newSystemPush?$AA@ 1000b250     dialog.obj
 0002:00003260       ??_C@_0N@MHEGOAAO@buttonGroup1?$AA@ 1000b260     dialog.obj
 0002:00003270       ??_C@_08POCADDJ@layout41?$AA@ 1000b270     dialog.obj
 0002:0000327c       ??_C@_0M@EACHACOL@inputsLabel?$AA@ 1000b27c     dialog.obj
 0002:00003288       ??_C@_0N@FIOKBJDD@processLabel?$AA@ 1000b288     dialog.obj
 0002:00003298       ??_C@_0N@FIEOLBFP@outputsLabel?$AA@ 1000b298     dialog.obj
 0002:000032a8       ??_C@_08NOCALIHA@layout48?$AA@ 1000b2a8     dialog.obj
 0002:000032b4       ??_C@_0P@GLJAELEN@inputsListView?$AA@ 1000b2b4     dialog.obj
 0002:000032c4       ??_C@_04KOACHJEN@Type?$AA@ 1000b2c4     dialog.obj
 0002:000032cc       ??_C@_0BA@FCEBDJBO@outputsListView?$AA@ 1000b2cc     dialog.obj
 0002:000032dc       ??_C@_08DNNEGBLL@layout43?$AA@ 1000b2dc     dialog.obj
 0002:000032e8       ??_C@_09LIPEGLAN@inputPush?$AA@ 1000b2e8     dialog.obj
 0002:000032f4       ??_C@_0M@BEHAACAP@processPush?$AA@ 1000b2f4     dialog.obj
 0002:00003300       ??_C@_0L@PHKJHJOA@outputPush?$AA@ 1000b300     dialog.obj
 0002:0000330c       ??_C@_06IOAEHBNO@dialog?$AA@ 1000b30c     dialog.obj
 0002:00003314       ??_C@_03ILBCOJBH@New?$AA@  1000b314     dialog.obj
 0002:00003318       ??_C@_0BA@LPNHLNAM@?$DMh1?$DOInputs?$DM?1h1?$DO?$AA@ 1000b318     dialog.obj
 0002:00003328       ??_C@_0BD@IGPEFHNN@?$DMh1?$DOProcesses?$DM?1h1?$DO?$AA@ 1000b328     dialog.obj
 0002:0000333c       ??_C@_0BB@LOGGEFLB@?$DMh1?$DOOutputs?$DM?1h1?$DO?$AA@ 1000b33c     dialog.obj
 0002:00003350       ??_C@_0BD@NAKBJAAM@Edit?5Selected?5File?$AA@ 1000b350     dialog.obj
 0002:00003364       ??_C@_0P@GNIMHNDI@Edit?5Processes?$AA@ 1000b364     dialog.obj
 0002:00003380       __xmm@0000002b0000005a000000140000000b 1000b380     dialog.obj
 0002:00003390       ??_C@_0BD@OMKHBCHI@cfg_alarm_overview?$AA@ 1000b390     moc_cfg_alarm_overview.obj
 0002:000033b0       ??_C@_05JLNEMJLN@dummy?$AA@ 1000b3b0     moc_cfg_alarm_overview.obj
 0002:000033b8       ??_C@_0L@DJNKAPEG@sNewSystem?$AA@ 1000b3b8     moc_cfg_alarm_overview.obj
 0002:000033d0       ??_C@_0BD@INLLCKAH@createNewDirectory?$AA@ 1000b3d0     moc_cfg_alarm_overview.obj
 0002:000033f0       ??_C@_09HIGIDEDO@markDirty?$AA@ 1000b3f0     moc_cfg_alarm_overview.obj
 0002:00003408       ??_C@_0BA@LKKBPBCL@createNewSystem?$AA@ 1000b408     moc_cfg_alarm_overview.obj
 0002:00003424       ??_C@_0BB@DBBIKKND@NavigatetoOutput?$AA@ 1000b424     moc_cfg_alarm_overview.obj
 0002:00003444       ??_C@_0BA@KOMOIPOE@NavigatetoProcs?$AA@ 1000b444     moc_cfg_alarm_overview.obj
 0002:00003460       ??_C@_0BA@HAJHKIPI@NavigatetoInput?$AA@ 1000b460     moc_cfg_alarm_overview.obj
 0002:00003470       ??_C@_07ECHCKIDD@sSystem?$AA@ 1000b470     moc_cfg_alarm_overview.obj
 0002:00003484       ??_C@_0N@JNMAEFDJ@selectSystem?$AA@ 1000b484     moc_cfg_alarm_overview.obj
 0002:000034a0       ??_C@_0O@ICMLCEAH@menuNewSystem?$AA@ 1000b4a0     moc_cfg_alarm_overview.obj
 0002:000034bc       ??_C@_0BE@MFJBJMAG@NavigateDatabaseOut?$AA@ 1000b4bc     moc_cfg_alarm_overview.obj
 0002:000034dc       ??_C@_0BA@KJNHHIM@NavigateBNCSOut?$AA@ 1000b4dc     moc_cfg_alarm_overview.obj
 0002:000034f8       ??_C@_0BA@IPJOCLDI@NavigateBNCSAcq?$AA@ 1000b4f8     moc_cfg_alarm_overview.obj
 0002:00003514       ??_C@_0O@LMAANOLM@NavigateProcs?$AA@ 1000b514     moc_cfg_alarm_overview.obj
 0002:000035c4       ??_C@_07MBMLLJIG@dummy?$CI?$CJ?$AA@ 1000b5c4     moc_cfg_alarm_overview.obj
 0002:000035cc       ??_C@_0BM@HGEJGCIP@createNewDirectory?$CIQString?$CJ?$AA@ 1000b5cc     moc_cfg_alarm_overview.obj
 0002:000035e8       ??_C@_0M@BCGJBPBD@markDirty?$CI?$CJ?$AA@ 1000b5e8     moc_cfg_alarm_overview.obj
 0002:000035f4       ??_C@_0BC@MONCANPB@createNewSystem?$CI?$CJ?$AA@ 1000b5f4     moc_cfg_alarm_overview.obj
 0002:00003608       ??_C@_0BD@OOAOGFIB@NavigatetoOutput?$CI?$CJ?$AA@ 1000b608     moc_cfg_alarm_overview.obj
 0002:0000361c       ??_C@_0BC@DFANIOCE@NavigatetoProcs?$CI?$CJ?$AA@ 1000b61c     moc_cfg_alarm_overview.obj
 0002:00003630       ??_C@_0BC@HGHALIEL@NavigatetoInput?$CI?$CJ?$AA@ 1000b630     moc_cfg_alarm_overview.obj
 0002:00003644       ??_C@_0BN@PCNKHLKL@selectSystem?$CIconst?5QString?$CG?$CJ?$AA@ 1000b644     moc_cfg_alarm_overview.obj
 0002:00003664       ??_C@_0BA@BFKHIGO@menuNewSystem?$CI?$CJ?$AA@ 1000b664     moc_cfg_alarm_overview.obj
 0002:00003674       ??_C@_0BG@NNPLDFML@NavigateDatabaseOut?$CI?$CJ?$AA@ 1000b674     moc_cfg_alarm_overview.obj
 0002:0000368c       ??_C@_0BC@CLEPLBPG@NavigateBNCSOut?$CI?$CJ?$AA@ 1000b68c     moc_cfg_alarm_overview.obj
 0002:000036a0       ??_C@_0BC@MJDLECJG@NavigateBNCSAcq?$CI?$CJ?$AA@ 1000b6a0     moc_cfg_alarm_overview.obj
 0002:000036b4       ??_C@_0BA@FLADCKNE@NavigateProcs?$CI?$CJ?$AA@ 1000b6b4     moc_cfg_alarm_overview.obj
 0002:000036d0       ??_C@_07KMMNMMFF@command?$AA@ 1000b6d0     moc_cfg_alarm_overview.obj
 0002:000036e4       ??_C@_0BJ@FEFNJDLM@command?$CIQString?0QString?$CJ?$AA@ 1000b6e4     moc_cfg_alarm_overview.obj
 0002:0000370c       ??_C@_0P@DMEOIADN@languageChange?$AA@ 1000b70c     moc_dialog.obj
 0002:00003728       ??_C@_0BB@PFEIHPGD@languageChange?$CI?$CJ?$AA@ 1000b728     moc_dialog.obj
 0002:00003740       ??_7type_info@@6B@         1000b740     MSVCRT:ti_inst.obj
 0002:00003744       __pRawDllMain              1000b744     MSVCRT:crtdll.obj
 0002:00003744       __pDefaultRawDllMain       1000b744     MSVCRT:crtdll.obj
 0002:00003750       __load_config_used         1000b750     MSVCRT:loadcfg.obj
 0002:00003798       ??_R3QShared@@8            1000b798     cfg_alarm_overview.obj
 0002:000037a8       ??_R2QShared@@8            1000b7a8     cfg_alarm_overview.obj
 0002:000037b0       ??_R1A@?0A@EA@QShared@@8   1000b7b0     cfg_alarm_overview.obj
 0002:000037cc       ??_R1A@?0A@EA@QGList@@8    1000b7cc     cfg_alarm_overview.obj
 0002:000037e8       ??_R3QGList@@8             1000b7e8     cfg_alarm_overview.obj
 0002:000037f8       ??_R2QGList@@8             1000b7f8     cfg_alarm_overview.obj
 0002:00003804       ??_R1A@?0A@EA@QPtrCollection@@8 1000b804     cfg_alarm_overview.obj
 0002:00003820       ??_R3QPtrCollection@@8     1000b820     cfg_alarm_overview.obj
 0002:00003830       ??_R2QPtrCollection@@8     1000b830     cfg_alarm_overview.obj
 0002:00003838       ??_R4QPopupMenu@@6BQObject@@@ 1000b838     cfg_alarm_overview.obj
 0002:0000384c       ??_R3QPopupMenu@@8         1000b84c     cfg_alarm_overview.obj
 0002:0000385c       ??_R2QPopupMenu@@8         1000b85c     cfg_alarm_overview.obj
 0002:0000387c       ??_R1A@?0A@EA@QPopupMenu@@8 1000b87c     cfg_alarm_overview.obj
 0002:00003898       ??_R1A@?0A@EA@QFrame@@8    1000b898     cfg_alarm_overview.obj
 0002:000038b4       ??_R3QFrame@@8             1000b8b4     cfg_alarm_overview.obj
 0002:000038c4       ??_R2QFrame@@8             1000b8c4     cfg_alarm_overview.obj
 0002:000038dc       ??_R1A@?0A@EA@QWidget@@8   1000b8dc     cfg_alarm_overview.obj
 0002:000038f8       ??_R3QWidget@@8            1000b8f8     cfg_alarm_overview.obj
 0002:00003908       ??_R2QWidget@@8            1000b908     cfg_alarm_overview.obj
 0002:0000391c       ??_R1A@?0A@EA@QObject@@8   1000b91c     cfg_alarm_overview.obj
 0002:00003938       ??_R3QObject@@8            1000b938     cfg_alarm_overview.obj
 0002:00003948       ??_R2QObject@@8            1000b948     cfg_alarm_overview.obj
 0002:00003954       ??_R13?0A@EA@Qt@@8         1000b954     cfg_alarm_overview.obj
 0002:00003970       ??_R3Qt@@8                 1000b970     cfg_alarm_overview.obj
 0002:00003980       ??_R2Qt@@8                 1000b980     cfg_alarm_overview.obj
 0002:00003988       ??_R1A@?0A@EA@Qt@@8        1000b988     cfg_alarm_overview.obj
 0002:000039a4       ??_R1CI@?0A@EA@QPaintDevice@@8 1000b9a4     cfg_alarm_overview.obj
 0002:000039c0       ??_R3QPaintDevice@@8       1000b9c0     cfg_alarm_overview.obj
 0002:000039d0       ??_R2QPaintDevice@@8       1000b9d0     cfg_alarm_overview.obj
 0002:000039d8       ??_R1A@?0A@EA@QPaintDevice@@8 1000b9d8     cfg_alarm_overview.obj
 0002:000039f4       ??_R1IM@?0A@EA@QMenuData@@8 1000b9f4     cfg_alarm_overview.obj
 0002:00003a10       ??_R3QMenuData@@8          1000ba10     cfg_alarm_overview.obj
 0002:00003a20       ??_R2QMenuData@@8          1000ba20     cfg_alarm_overview.obj
 0002:00003a28       ??_R1A@?0A@EA@QMenuData@@8 1000ba28     cfg_alarm_overview.obj
 0002:00003a44       ??_R4QPopupMenu@@6BQPaintDevice@@@ 1000ba44     cfg_alarm_overview.obj
 0002:00003a58       ??_R4QPopupMenu@@6B@       1000ba58     cfg_alarm_overview.obj
 0002:00003a6c       ??_R4QAction@@6B@          1000ba6c     cfg_alarm_overview.obj
 0002:00003a80       ??_R3QAction@@8            1000ba80     cfg_alarm_overview.obj
 0002:00003a90       ??_R2QAction@@8            1000ba90     cfg_alarm_overview.obj
 0002:00003aa0       ??_R1A@?0A@EA@QAction@@8   1000baa0     cfg_alarm_overview.obj
 0002:00003abc       ??_R4QToolBar@@6BQObject@@@ 1000babc     cfg_alarm_overview.obj
 0002:00003ad0       ??_R3QToolBar@@8           1000bad0     cfg_alarm_overview.obj
 0002:00003ae0       ??_R2QToolBar@@8           1000bae0     cfg_alarm_overview.obj
 0002:00003b00       ??_R1A@?0A@EA@QToolBar@@8  1000bb00     cfg_alarm_overview.obj
 0002:00003b1c       ??_R1A@?0A@EA@QDockWindow@@8 1000bb1c     cfg_alarm_overview.obj
 0002:00003b38       ??_R3QDockWindow@@8        1000bb38     cfg_alarm_overview.obj
 0002:00003b48       ??_R2QDockWindow@@8        1000bb48     cfg_alarm_overview.obj
 0002:00003b64       ??_R4QToolBar@@6BQPaintDevice@@@ 1000bb64     cfg_alarm_overview.obj
 0002:00003b78       ??_R4QListViewItem@@6B@    1000bb78     cfg_alarm_overview.obj
 0002:00003b8c       ??_R3QListViewItem@@8      1000bb8c     cfg_alarm_overview.obj
 0002:00003b9c       ??_R2QListViewItem@@8      1000bb9c     cfg_alarm_overview.obj
 0002:00003ba8       ??_R1A@?0A@EA@QListViewItem@@8 1000bba8     cfg_alarm_overview.obj
 0002:00003bc4       ??_R4QDockWindowList@@6B@  1000bbc4     cfg_alarm_overview.obj
 0002:00003bd8       ??_R3QDockWindowList@@8    1000bbd8     cfg_alarm_overview.obj
 0002:00003be8       ??_R2QDockWindowList@@8    1000bbe8     cfg_alarm_overview.obj
 0002:00003bfc       ??_R1A@?0A@EA@QDockWindowList@@8 1000bbfc     cfg_alarm_overview.obj
 0002:00003c18       ??_R1A@?0A@EA@?$QPtrList@VQDockWindow@@@@8 1000bc18     cfg_alarm_overview.obj
 0002:00003c34       ??_R3?$QPtrList@VQDockWindow@@@@8 1000bc34     cfg_alarm_overview.obj
 0002:00003c44       ??_R2?$QPtrList@VQDockWindow@@@@8 1000bc44     cfg_alarm_overview.obj
 0002:00003c54       ??_R4QPopupMenuList@@6B@   1000bc54     cfg_alarm_overview.obj
 0002:00003c68       ??_R3QPopupMenuList@@8     1000bc68     cfg_alarm_overview.obj
 0002:00003c78       ??_R2QPopupMenuList@@8     1000bc78     cfg_alarm_overview.obj
 0002:00003c8c       ??_R1A@?0A@EA@QPopupMenuList@@8 1000bc8c     cfg_alarm_overview.obj
 0002:00003ca8       ??_R1A@?0A@EA@?$QPtrList@VQPopupMenu@@@@8 1000bca8     cfg_alarm_overview.obj
 0002:00003cc4       ??_R3?$QPtrList@VQPopupMenu@@@@8 1000bcc4     cfg_alarm_overview.obj
 0002:00003cd4       ??_R2?$QPtrList@VQPopupMenu@@@@8 1000bcd4     cfg_alarm_overview.obj
 0002:00003ce4       ??_R4?$QPtrList@VQPopupMenu@@@@6B@ 1000bce4     cfg_alarm_overview.obj
 0002:00003cf8       ??_R4QGuardedPtrPrivate@@6B@ 1000bcf8     cfg_alarm_overview.obj
 0002:00003d0c       ??_R3QGuardedPtrPrivate@@8 1000bd0c     cfg_alarm_overview.obj
 0002:00003d1c       ??_R2QGuardedPtrPrivate@@8 1000bd1c     cfg_alarm_overview.obj
 0002:00003d30       ??_R1A@?0A@EA@QGuardedPtrPrivate@@8 1000bd30     cfg_alarm_overview.obj
 0002:00003d4c       ??_R1CI@?0A@EA@QShared@@8  1000bd4c     cfg_alarm_overview.obj
 0002:00003d68       ??_R1A@?0A@EA@QGDict@@8    1000bd68     cfg_alarm_overview.obj
 0002:00003d84       ??_R3QGDict@@8             1000bd84     cfg_alarm_overview.obj
 0002:00003d94       ??_R2QGDict@@8             1000bd94     cfg_alarm_overview.obj
 0002:00003da0       ??_R4config_plugin_base@@6BQObject@@@ 1000bda0     cfg_alarm_overview.obj
 0002:00003db4       ??_R3config_plugin_base@@8 1000bdb4     cfg_alarm_overview.obj
 0002:00003dc4       ??_R2config_plugin_base@@8 1000bdc4     cfg_alarm_overview.obj
 0002:00003ddc       ??_R1A@?0A@EA@config_plugin_base@@8 1000bddc     cfg_alarm_overview.obj
 0002:00003df8       ??_R4config_plugin_base@@6BQPaintDevice@@@ 1000bdf8     cfg_alarm_overview.obj
 0002:00003e0c       ??_R4cfg_alarm_overview@@6BQObject@@@ 1000be0c     cfg_alarm_overview.obj
 0002:00003e20       ??_R3cfg_alarm_overview@@8 1000be20     cfg_alarm_overview.obj
 0002:00003e30       ??_R2cfg_alarm_overview@@8 1000be30     cfg_alarm_overview.obj
 0002:00003e4c       ??_R1A@?0A@EA@cfg_alarm_overview@@8 1000be4c     cfg_alarm_overview.obj
 0002:00003e68       ??_R4cfg_alarm_overview@@6BQPaintDevice@@@ 1000be68     cfg_alarm_overview.obj
 0002:00003e7c       ??_R4?$QDict@VQAction@@@@6B@ 1000be7c     cfg_alarm_overview.obj
 0002:00003e90       ??_R3?$QDict@VQAction@@@@8 1000be90     cfg_alarm_overview.obj
 0002:00003ea0       ??_R2?$QDict@VQAction@@@@8 1000bea0     cfg_alarm_overview.obj
 0002:00003eb0       ??_R1A@?0A@EA@?$QDict@VQAction@@@@8 1000beb0     cfg_alarm_overview.obj
 0002:00003ecc       ??_R4?$QPtrList@VCInputFile@@@@6B@ 1000becc     cfg_alarm_overview.obj
 0002:00003ee0       ??_R3?$QPtrList@VCInputFile@@@@8 1000bee0     cfg_alarm_overview.obj
 0002:00003ef0       ??_R2?$QPtrList@VCInputFile@@@@8 1000bef0     cfg_alarm_overview.obj
 0002:00003f00       ??_R1A@?0A@EA@?$QPtrList@VCInputFile@@@@8 1000bf00     cfg_alarm_overview.obj
 0002:00003f1c       ??_R4?$QPtrList@VCOutputFile@@@@6B@ 1000bf1c     cfg_alarm_overview.obj
 0002:00003f30       ??_R3?$QPtrList@VCOutputFile@@@@8 1000bf30     cfg_alarm_overview.obj
 0002:00003f40       ??_R2?$QPtrList@VCOutputFile@@@@8 1000bf40     cfg_alarm_overview.obj
 0002:00003f50       ??_R1A@?0A@EA@?$QPtrList@VCOutputFile@@@@8 1000bf50     cfg_alarm_overview.obj
 0002:00003f6c       ??_R4dialog@@6BQObject@@@  1000bf6c     dialogimpl.obj
 0002:00003f80       ??_R3dialog@@8             1000bf80     dialogimpl.obj
 0002:00003f90       ??_R2dialog@@8             1000bf90     dialogimpl.obj
 0002:00003fac       ??_R1A@?0A@EA@dialog@@8    1000bfac     dialogimpl.obj
 0002:00003fc8       ??_R1A@?0A@EA@dialogBase@@8 1000bfc8     dialogimpl.obj
 0002:00003fe4       ??_R3dialogBase@@8         1000bfe4     dialogimpl.obj
 0002:00003ff4       ??_R2dialogBase@@8         1000bff4     dialogimpl.obj
 0002:0000400c       ??_R4dialog@@6BQPaintDevice@@@ 1000c00c     dialogimpl.obj
 0002:00004020       ??_R4CInputFile@@6B@       1000c020     InputFile.obj
 0002:00004034       ??_R3CInputFile@@8         1000c034     InputFile.obj
 0002:00004044       ??_R2CInputFile@@8         1000c044     InputFile.obj
 0002:0000404c       ??_R1A@?0A@EA@CInputFile@@8 1000c04c     InputFile.obj
 0002:00004068       ??_R4COutputFile@@6B@      1000c068     OutputFile.obj
 0002:0000407c       ??_R3COutputFile@@8        1000c07c     OutputFile.obj
 0002:0000408c       ??_R2COutputFile@@8        1000c08c     OutputFile.obj
 0002:00004094       ??_R1A@?0A@EA@COutputFile@@8 1000c094     OutputFile.obj
 0002:000040b0       ??_R4config_plugin_desc_base@@6B@ 1000c0b0     plugindesc.obj
 0002:000040c4       ??_R3config_plugin_desc_base@@8 1000c0c4     plugindesc.obj
 0002:000040d4       ??_R2config_plugin_desc_base@@8 1000c0d4     plugindesc.obj
 0002:000040dc       ??_R1A@?0A@EA@config_plugin_desc_base@@8 1000c0dc     plugindesc.obj
 0002:000040f8       ??_R4plugindesc@@6B@       1000c0f8     plugindesc.obj
 0002:0000410c       ??_R3plugindesc@@8         1000c10c     plugindesc.obj
 0002:0000411c       ??_R2plugindesc@@8         1000c11c     plugindesc.obj
 0002:00004128       ??_R1A@?0A@EA@plugindesc@@8 1000c128     plugindesc.obj
 0002:00004144       ??_R4QVBoxLayout@@6BQObject@@@ 1000c144     dialog.obj
 0002:00004158       ??_R3QVBoxLayout@@8        1000c158     dialog.obj
 0002:00004168       ??_R2QVBoxLayout@@8        1000c168     dialog.obj
 0002:00004184       ??_R1A@?0A@EA@QVBoxLayout@@8 1000c184     dialog.obj
 0002:000041a0       ??_R1A@?0A@EA@QBoxLayout@@8 1000c1a0     dialog.obj
 0002:000041bc       ??_R3QBoxLayout@@8         1000c1bc     dialog.obj
 0002:000041cc       ??_R2QBoxLayout@@8         1000c1cc     dialog.obj
 0002:000041e4       ??_R1A@?0A@EA@QLayout@@8   1000c1e4     dialog.obj
 0002:00004200       ??_R3QLayout@@8            1000c200     dialog.obj
 0002:00004210       ??_R2QLayout@@8            1000c210     dialog.obj
 0002:00004224       ??_R1CI@?0A@EA@QLayoutItem@@8 1000c224     dialog.obj
 0002:00004240       ??_R3QLayoutItem@@8        1000c240     dialog.obj
 0002:00004250       ??_R2QLayoutItem@@8        1000c250     dialog.obj
 0002:00004258       ??_R1A@?0A@EA@QLayoutItem@@8 1000c258     dialog.obj
 0002:00004274       ??_R4QVBoxLayout@@6BQLayoutItem@@@ 1000c274     dialog.obj
 0002:00004288       ??_R4QHBoxLayout@@6BQObject@@@ 1000c288     dialog.obj
 0002:0000429c       ??_R3QHBoxLayout@@8        1000c29c     dialog.obj
 0002:000042ac       ??_R2QHBoxLayout@@8        1000c2ac     dialog.obj
 0002:000042c8       ??_R1A@?0A@EA@QHBoxLayout@@8 1000c2c8     dialog.obj
 0002:000042e4       ??_R4QHBoxLayout@@6BQLayoutItem@@@ 1000c2e4     dialog.obj
 0002:000042f8       ??_R4CAlm_sys_select@@6BQObject@@@ 1000c2f8     dialog.obj
 0002:0000430c       ??_R3CAlm_sys_select@@8    1000c30c     dialog.obj
 0002:0000431c       ??_R2CAlm_sys_select@@8    1000c31c     dialog.obj
 0002:00004340       ??_R1A@?0A@EA@CAlm_sys_select@@8 1000c340     dialog.obj
 0002:0000435c       ??_R1A@?0A@EA@QVBox@@8     1000c35c     dialog.obj
 0002:00004378       ??_R3QVBox@@8              1000c378     dialog.obj
 0002:00004388       ??_R2QVBox@@8              1000c388     dialog.obj
 0002:000043a8       ??_R1A@?0A@EA@QHBox@@8     1000c3a8     dialog.obj
 0002:000043c4       ??_R3QHBox@@8              1000c3c4     dialog.obj
 0002:000043d4       ??_R2QHBox@@8              1000c3d4     dialog.obj
 0002:000043f0       ??_R4CAlm_sys_select@@6BQPaintDevice@@@ 1000c3f0     dialog.obj
 0002:00004404       ??_R4QButtonGroup@@6BQObject@@@ 1000c404     dialog.obj
 0002:00004418       ??_R3QButtonGroup@@8       1000c418     dialog.obj
 0002:00004428       ??_R2QButtonGroup@@8       1000c428     dialog.obj
 0002:00004448       ??_R1A@?0A@EA@QButtonGroup@@8 1000c448     dialog.obj
 0002:00004464       ??_R1A@?0A@EA@QGroupBox@@8 1000c464     dialog.obj
 0002:00004480       ??_R3QGroupBox@@8          1000c480     dialog.obj
 0002:00004490       ??_R2QGroupBox@@8          1000c490     dialog.obj
 0002:000044ac       ??_R4QButtonGroup@@6BQPaintDevice@@@ 1000c4ac     dialog.obj
 0002:000044c0       ??_R4QPushButton@@6BQObject@@@ 1000c4c0     dialog.obj
 0002:000044d4       ??_R3QPushButton@@8        1000c4d4     dialog.obj
 0002:000044e4       ??_R2QPushButton@@8        1000c4e4     dialog.obj
 0002:00004500       ??_R1A@?0A@EA@QPushButton@@8 1000c500     dialog.obj
 0002:0000451c       ??_R1A@?0A@EA@QButton@@8   1000c51c     dialog.obj
 0002:00004538       ??_R3QButton@@8            1000c538     dialog.obj
 0002:00004548       ??_R2QButton@@8            1000c548     dialog.obj
 0002:00004560       ??_R4QPushButton@@6BQPaintDevice@@@ 1000c560     dialog.obj
 0002:00004574       ??_R4QLabel@@6BQObject@@@  1000c574     dialog.obj
 0002:00004588       ??_R3QLabel@@8             1000c588     dialog.obj
 0002:00004598       ??_R2QLabel@@8             1000c598     dialog.obj
 0002:000045b4       ??_R1A@?0A@EA@QLabel@@8    1000c5b4     dialog.obj
 0002:000045d0       ??_R4QLabel@@6BQPaintDevice@@@ 1000c5d0     dialog.obj
 0002:000045e4       ??_R4QListView@@6BQObject@@@ 1000c5e4     dialog.obj
 0002:000045f8       ??_R3QListView@@8          1000c5f8     dialog.obj
 0002:00004608       ??_R2QListView@@8          1000c608     dialog.obj
 0002:00004628       ??_R1A@?0A@EA@QListView@@8 1000c628     dialog.obj
 0002:00004644       ??_R1A@?0A@EA@QScrollView@@8 1000c644     dialog.obj
 0002:00004660       ??_R3QScrollView@@8        1000c660     dialog.obj
 0002:00004670       ??_R2QScrollView@@8        1000c670     dialog.obj
 0002:0000468c       ??_R4QListView@@6BQPaintDevice@@@ 1000c68c     dialog.obj
 0002:000046a0       ??_R4dialogBase@@6BQObject@@@ 1000c6a0     dialog.obj
 0002:000046b4       ??_R4dialogBase@@6BQPaintDevice@@@ 1000c6b4     dialog.obj
 0002:000046c8       ??_R4QSpacerItem@@6B@      1000c6c8     dialog.obj
 0002:000046dc       ??_R3QSpacerItem@@8        1000c6dc     dialog.obj
 0002:000046ec       ??_R2QSpacerItem@@8        1000c6ec     dialog.obj
 0002:000046f8       ??_R1A@?0A@EA@QSpacerItem@@8 1000c6f8     dialog.obj
 0002:00004714       ??_R4type_info@@6B@        1000c714     MSVCRT:ti_inst.obj
 0002:00004728       ??_R3type_info@@8          1000c728     MSVCRT:ti_inst.obj
 0002:00004738       ??_R2type_info@@8          1000c738     MSVCRT:ti_inst.obj
 0002:00004740       ??_R1A@?0A@EA@type_info@@8 1000c740     MSVCRT:ti_inst.obj
 0002:00004760       ___safe_se_handler_table   1000c760     <linker-defined>
 0002:000047d0       ___rtc_iaa                 1000c7d0     MSVCRT:initsect.obj
 0002:000047d4       ___rtc_izz                 1000c7d4     MSVCRT:initsect.obj
 0002:000047d8       ___rtc_taa                 1000c7d8     MSVCRT:initsect.obj
 0002:000047dc       ___rtc_tzz                 1000c7dc     MSVCRT:initsect.obj
 0002:00005438       __IMPORT_DESCRIPTOR_qt-mt323 1000d438     qt-mt323:qt-mt323.dll
 0002:0000544c       __IMPORT_DESCRIPTOR_config_icons 1000d44c     config_icons:config_icons.dll
 0002:00005460       __IMPORT_DESCRIPTOR_alm_sys_select 1000d460     alm_sys_select:alm_sys_select.dll
 0002:00005474       __IMPORT_DESCRIPTOR_KERNEL32 1000d474     kernel32:KERNEL32.dll
 0002:00005488       __IMPORT_DESCRIPTOR_MSVCR120 1000d488     MSVCRT:MSVCR120.dll
 0002:0000549c       __NULL_IMPORT_DESCRIPTOR   1000d49c     qt-mt323:qt-mt323.dll
 0003:000001c0       ___security_cookie         100151c0     MSVCRT:gs_cookie.obj
 0003:000001c4       ___security_cookie_complement 100151c4     MSVCRT:gs_cookie.obj
 0003:000001d0       ___native_dllmain_reason   100151d0     MSVCRT:natstart.obj
 0003:000001d4       ??_R0?AUQShared@@@8        100151d4     cfg_alarm_overview.obj
 0003:000001ec       ??_R0?AVQGList@@@8         100151ec     cfg_alarm_overview.obj
 0003:00000204       ??_R0?AVQPtrCollection@@@8 10015204     cfg_alarm_overview.obj
 0003:00000224       ??_R0?AVQPopupMenu@@@8     10015224     cfg_alarm_overview.obj
 0003:00000240       ??_R0?AVQFrame@@@8         10015240     cfg_alarm_overview.obj
 0003:00000258       ??_R0?AVQWidget@@@8        10015258     cfg_alarm_overview.obj
 0003:00000270       ??_R0?AVQObject@@@8        10015270     cfg_alarm_overview.obj
 0003:00000288       ??_R0?AVQt@@@8             10015288     cfg_alarm_overview.obj
 0003:0000029c       ??_R0?AVQPaintDevice@@@8   1001529c     cfg_alarm_overview.obj
 0003:000002b8       ??_R0?AVQMenuData@@@8      100152b8     cfg_alarm_overview.obj
 0003:000002d0       ??_R0?AVQAction@@@8        100152d0     cfg_alarm_overview.obj
 0003:000002e8       ??_R0?AVQToolBar@@@8       100152e8     cfg_alarm_overview.obj
 0003:00000300       ??_R0?AVQDockWindow@@@8    10015300     cfg_alarm_overview.obj
 0003:0000031c       ??_R0?AVQListViewItem@@@8  1001531c     cfg_alarm_overview.obj
 0003:00000338       ??_R0?AVQDockWindowList@@@8 10015338     cfg_alarm_overview.obj
 0003:00000358       ??_R0?AV?$QPtrList@VQDockWindow@@@@@8 10015358     cfg_alarm_overview.obj
 0003:00000380       ??_R0?AVQPopupMenuList@@@8 10015380     cfg_alarm_overview.obj
 0003:000003a0       ??_R0?AV?$QPtrList@VQPopupMenu@@@@@8 100153a0     cfg_alarm_overview.obj
 0003:000003c8       ??_R0?AVQGuardedPtrPrivate@@@8 100153c8     cfg_alarm_overview.obj
 0003:000003ec       ??_R0?AVQGDict@@@8         100153ec     cfg_alarm_overview.obj
 0003:00000404       ??_R0?AVconfig_plugin_base@@@8 10015404     cfg_alarm_overview.obj
 0003:00000428       ??_R0?AVcfg_alarm_overview@@@8 10015428     cfg_alarm_overview.obj
 0003:0000044c       ??_R0?AV?$QDict@VQAction@@@@@8 1001544c     cfg_alarm_overview.obj
 0003:00000470       ??_R0?AV?$QPtrList@VCInputFile@@@@@8 10015470     cfg_alarm_overview.obj
 0003:00000498       ??_R0?AV?$QPtrList@VCOutputFile@@@@@8 10015498     cfg_alarm_overview.obj
 0003:000004c0       ??_R0?AVdialog@@@8         100154c0     dialogimpl.obj
 0003:000004d8       ??_R0?AVdialogBase@@@8     100154d8     dialogimpl.obj
 0003:000004f4       ??_R0?AVCInputFile@@@8     100154f4     InputFile.obj
 0003:00000510       ??_R0?AVCOutputFile@@@8    10015510     OutputFile.obj
 0003:0000052c       ??_R0?AVconfig_plugin_desc_base@@@8 1001552c     plugindesc.obj
 0003:00000554       ??_R0?AVplugindesc@@@8     10015554     plugindesc.obj
 0003:00000570       ??_R0?AVQVBoxLayout@@@8    10015570     dialog.obj
 0003:0000058c       ??_R0?AVQBoxLayout@@@8     1001558c     dialog.obj
 0003:000005a8       ??_R0?AVQLayout@@@8        100155a8     dialog.obj
 0003:000005c0       ??_R0?AVQLayoutItem@@@8    100155c0     dialog.obj
 0003:000005dc       ??_R0?AVQHBoxLayout@@@8    100155dc     dialog.obj
 0003:000005f8       ??_R0?AVCAlm_sys_select@@@8 100155f8     dialog.obj
 0003:00000618       ??_R0?AVQVBox@@@8          10015618     dialog.obj
 0003:0000062c       ??_R0?AVQHBox@@@8          1001562c     dialog.obj
 0003:00000640       ??_R0?AVQButtonGroup@@@8   10015640     dialog.obj
 0003:0000065c       ??_R0?AVQGroupBox@@@8      1001565c     dialog.obj
 0003:00000674       ??_R0?AVQPushButton@@@8    10015674     dialog.obj
 0003:00000690       ??_R0?AVQButton@@@8        10015690     dialog.obj
 0003:000006a8       ??_R0?AVQLabel@@@8         100156a8     dialog.obj
 0003:000006c0       ??_R0?AVQListView@@@8      100156c0     dialog.obj
 0003:000006d8       ??_R0?AVQScrollView@@@8    100156d8     dialog.obj
 0003:000006f4       ??_R0?AVQSpacerItem@@@8    100156f4     dialog.obj
 0003:00000710       ??_R0?AVtype_info@@@8      10015710     MSVCRT:ti_inst.obj
 0003:00000728       ?metaObj@cfg_alarm_overview@@0PAVQMetaObject@@A 10015728     moc_cfg_alarm_overview.obj
 0003:00000774       ?metaObj@dialogBase@@0PAVQMetaObject@@A 10015774     moc_dialog.obj
 0003:0000077c       ?metaObj@dialog@@0PAVQMetaObject@@A 1001577c     moc_dialogimpl.obj
 0003:00000aa8       ?__type_info_root_node@@3U__type_info_node@@A 10015aa8     MSVCRT:tncleanup.obj
 0003:00000ab0       ___native_startup_lock     10015ab0     <common>
 0003:00000ab4       ___native_startup_state    10015ab4     <common>
 0003:00000ab8       ___dyn_tls_init_callback   10015ab8     <common>
 0003:00000abc       ___onexitend               10015abc     <common>
 0003:00000ac0       ___onexitbegin             10015ac0     <common>

 entry point at        0001:00004f3a

 Static symbols

 0001:00000000       ??__EcleanUp_cfg_alarm_overview@@YAXXZ 10001000 f   moc_cfg_alarm_overview.obj
 0001:00000021       ??__EcleanUp_dialogBase@@YAXXZ 10001021 f   moc_dialog.obj
 0001:00000042       ??__EcleanUp_dialog@@YAXXZ 10001042 f   moc_dialogimpl.obj
 0001:00003b0f       $LN27                      10004b0f     moc_cfg_alarm_overview.obj
 0001:00004cf7       _pre_c_init                10005cf7 f   MSVCRT:crtdll.obj
 0001:00004f5d       ___DllMainCRTStartup       10005f5d f   MSVCRT:crtdll.obj
 0001:000051d0       $$000000                   100061d0     MSVCRT:sehprolg4.obj
 0001:000054ec       __unwindfunclet$?create@plugindesc@@UAEPAVconfig_plugin_base@@ABVQString@@00@Z$0 100064ec f   cfg_alarm_overview.obj
 0001:000054ec       __unwindfunclet$??4?$QGuardedPtr@VQDockWindow@@@@QAEAAV0@PAVQDockWindow@@@Z$0 100064ec f   cfg_alarm_overview.obj
 0001:000054ec       __unwindfunclet$??4?$QGuardedPtr@VQPopupMenu@@@@QAEAAV0@PAVQPopupMenu@@@Z$0 100064ec f   cfg_alarm_overview.obj
 0001:000054ec       __unwindfunclet$??0?$QGuardedPtr@VQDockWindow@@@@QAE@XZ$0 100064ec f   cfg_alarm_overview.obj
 0001:000054ec       __unwindfunclet$??0?$QGuardedPtr@VQPopupMenu@@@@QAE@XZ$0 100064ec f   cfg_alarm_overview.obj
 0001:000054f6       __ehhandler$??0?$QGuardedPtr@VQDockWindow@@@@QAE@XZ 100064f6 f   cfg_alarm_overview.obj
 0001:000054f6       __ehhandler$?create@plugindesc@@UAEPAVconfig_plugin_base@@ABVQString@@00@Z 100064f6 f   cfg_alarm_overview.obj
 0001:000054f6       __ehhandler$??4?$QGuardedPtr@VQPopupMenu@@@@QAEAAV0@PAVQPopupMenu@@@Z 100064f6 f   cfg_alarm_overview.obj
 0001:000054f6       __ehhandler$??0?$QGuardedPtr@VQPopupMenu@@@@QAE@XZ 100064f6 f   cfg_alarm_overview.obj
 0001:000054f6       __ehhandler$??4?$QGuardedPtr@VQDockWindow@@@@QAEAAV0@PAVQDockWindow@@@Z 100064f6 f   cfg_alarm_overview.obj
 0001:00005511       __unwindfunclet$??0cfg_alarm_overview@@QAE@ABVQString@@00@Z$0 10006511 f   cfg_alarm_overview.obj
 0001:00005519       __unwindfunclet$??0cfg_alarm_overview@@QAE@ABVQString@@00@Z$1 10006519 f   cfg_alarm_overview.obj
 0001:00005524       __unwindfunclet$??0cfg_alarm_overview@@QAE@ABVQString@@00@Z$2 10006524 f   cfg_alarm_overview.obj
 0001:0000552f       __unwindfunclet$??0cfg_alarm_overview@@QAE@ABVQString@@00@Z$3 1000652f f   cfg_alarm_overview.obj
 0001:0000553d       __unwindfunclet$??0cfg_alarm_overview@@QAE@ABVQString@@00@Z$4 1000653d f   cfg_alarm_overview.obj
 0001:0000554c       __unwindfunclet$??0cfg_alarm_overview@@QAE@ABVQString@@00@Z$5 1000654c f   cfg_alarm_overview.obj
 0001:0000555b       __unwindfunclet$??0cfg_alarm_overview@@QAE@ABVQString@@00@Z$6 1000655b f   cfg_alarm_overview.obj
 0001:0000556a       __unwindfunclet$??0cfg_alarm_overview@@QAE@ABVQString@@00@Z$7 1000656a f   cfg_alarm_overview.obj
 0001:00005579       __unwindfunclet$??0cfg_alarm_overview@@QAE@ABVQString@@00@Z$8 10006579 f   cfg_alarm_overview.obj
 0001:00005588       __unwindfunclet$??0cfg_alarm_overview@@QAE@ABVQString@@00@Z$9 10006588 f   cfg_alarm_overview.obj
 0001:00005596       __unwindfunclet$??0cfg_alarm_overview@@QAE@ABVQString@@00@Z$10 10006596 f   cfg_alarm_overview.obj
 0001:000055a4       __unwindfunclet$??0cfg_alarm_overview@@QAE@ABVQString@@00@Z$11 100065a4 f   cfg_alarm_overview.obj
 0001:000055b3       __unwindfunclet$??0cfg_alarm_overview@@QAE@ABVQString@@00@Z$12 100065b3 f   cfg_alarm_overview.obj
 0001:000055bd       __unwindfunclet$??0cfg_alarm_overview@@QAE@ABVQString@@00@Z$13 100065bd f   cfg_alarm_overview.obj
 0001:000055c7       __unwindfunclet$??0cfg_alarm_overview@@QAE@ABVQString@@00@Z$14 100065c7 f   cfg_alarm_overview.obj
 0001:000055d0       __unwindfunclet$??0cfg_alarm_overview@@QAE@ABVQString@@00@Z$15 100065d0 f   cfg_alarm_overview.obj
 0001:000055da       __unwindfunclet$??0cfg_alarm_overview@@QAE@ABVQString@@00@Z$16 100065da f   cfg_alarm_overview.obj
 0001:000055e4       __unwindfunclet$??0cfg_alarm_overview@@QAE@ABVQString@@00@Z$17 100065e4 f   cfg_alarm_overview.obj
 0001:000055fe       __unwindfunclet$??0cfg_alarm_overview@@QAE@ABVQString@@00@Z$18 100065fe f   cfg_alarm_overview.obj
 0001:00005618       __unwindfunclet$??0cfg_alarm_overview@@QAE@ABVQString@@00@Z$19 10006618 f   cfg_alarm_overview.obj
 0001:00005632       __unwindfunclet$??0cfg_alarm_overview@@QAE@ABVQString@@00@Z$20 10006632 f   cfg_alarm_overview.obj
 0001:0000564c       __unwindfunclet$??0cfg_alarm_overview@@QAE@ABVQString@@00@Z$22 1000664c f   cfg_alarm_overview.obj
 0001:00005656       __unwindfunclet$??0cfg_alarm_overview@@QAE@ABVQString@@00@Z$23 10006656 f   cfg_alarm_overview.obj
 0001:00005670       __unwindfunclet$??0cfg_alarm_overview@@QAE@ABVQString@@00@Z$24 10006670 f   cfg_alarm_overview.obj
 0001:0000568a       __unwindfunclet$??0cfg_alarm_overview@@QAE@ABVQString@@00@Z$25 1000668a f   cfg_alarm_overview.obj
 0001:000056a4       __unwindfunclet$??0cfg_alarm_overview@@QAE@ABVQString@@00@Z$26 100066a4 f   cfg_alarm_overview.obj
 0001:000056c3       __ehhandler$??0cfg_alarm_overview@@QAE@ABVQString@@00@Z 100066c3 f   cfg_alarm_overview.obj
 0001:000056de       __unwindfunclet$??0config_plugin_base@@QAE@ABVQString@@00@Z$0 100066de f   cfg_alarm_overview.obj
 0001:000056e7       __unwindfunclet$??0config_plugin_base@@QAE@ABVQString@@00@Z$1 100066e7 f   cfg_alarm_overview.obj
 0001:000056f3       __unwindfunclet$??0config_plugin_base@@QAE@ABVQString@@00@Z$2 100066f3 f   cfg_alarm_overview.obj
 0001:000056ff       __unwindfunclet$??0config_plugin_base@@QAE@ABVQString@@00@Z$3 100066ff f   cfg_alarm_overview.obj
 0001:0000570b       __ehhandler$??0config_plugin_base@@QAE@ABVQString@@00@Z 1000670b f   cfg_alarm_overview.obj
 0001:00005726       __unwindfunclet$??1?$QDict@VQAction@@@@UAE@XZ$0 10006726 f   cfg_alarm_overview.obj
 0001:0000572f       __ehhandler$??1?$QDict@VQAction@@@@UAE@XZ 1000672f f   cfg_alarm_overview.obj
 0001:0000574a       __unwindfunclet$??1?$QPtrList@VQPopupMenu@@@@UAE@XZ$0 1000674a f   cfg_alarm_overview.obj
 0001:0000574a       __unwindfunclet$??1?$QPtrList@VCOutputFile@@@@UAE@XZ$0 1000674a f   cfg_alarm_overview.obj
 0001:0000574a       __unwindfunclet$??1?$QPtrList@VCInputFile@@@@UAE@XZ$0 1000674a f   cfg_alarm_overview.obj
 0001:00005753       __ehhandler$??1?$QPtrList@VQPopupMenu@@@@UAE@XZ 10006753 f   cfg_alarm_overview.obj
 0001:00005753       __ehhandler$??1?$QPtrList@VCOutputFile@@@@UAE@XZ 10006753 f   cfg_alarm_overview.obj
 0001:00005753       __ehhandler$??1?$QPtrList@VCInputFile@@@@UAE@XZ 10006753 f   cfg_alarm_overview.obj
 0001:0000576e       __unwindfunclet$??1QDockWindowList@@UAE@XZ$0 1000676e f   cfg_alarm_overview.obj
 0001:00005777       __unwindfunclet$??1QDockWindowList@@UAE@XZ$1 10006777 f   cfg_alarm_overview.obj
 0001:00005780       __ehhandler$??1QDockWindowList@@UAE@XZ 10006780 f   cfg_alarm_overview.obj
 0001:0000579b       __unwindfunclet$??1QPopupMenuList@@UAE@XZ$0 1000679b f   cfg_alarm_overview.obj
 0001:000057a3       __ehhandler$??1QPopupMenuList@@UAE@XZ 100067a3 f   cfg_alarm_overview.obj
 0001:000057be       __unwindfunclet$??1cfg_alarm_overview@@UAE@XZ$0 100067be f   cfg_alarm_overview.obj
 0001:000057c6       __unwindfunclet$??1cfg_alarm_overview@@UAE@XZ$1 100067c6 f   cfg_alarm_overview.obj
 0001:000057d1       __unwindfunclet$??1cfg_alarm_overview@@UAE@XZ$2 100067d1 f   cfg_alarm_overview.obj
 0001:000057dc       __unwindfunclet$??1cfg_alarm_overview@@UAE@XZ$3 100067dc f   cfg_alarm_overview.obj
 0001:000057ea       __unwindfunclet$??1cfg_alarm_overview@@UAE@XZ$4 100067ea f   cfg_alarm_overview.obj
 0001:000057f9       __unwindfunclet$??1cfg_alarm_overview@@UAE@XZ$5 100067f9 f   cfg_alarm_overview.obj
 0001:00005808       __unwindfunclet$??1cfg_alarm_overview@@UAE@XZ$6 10006808 f   cfg_alarm_overview.obj
 0001:00005817       __unwindfunclet$??1cfg_alarm_overview@@UAE@XZ$7 10006817 f   cfg_alarm_overview.obj
 0001:00005826       __unwindfunclet$??1cfg_alarm_overview@@UAE@XZ$8 10006826 f   cfg_alarm_overview.obj
 0001:00005835       __unwindfunclet$??1cfg_alarm_overview@@UAE@XZ$9 10006835 f   cfg_alarm_overview.obj
 0001:00005843       __unwindfunclet$??1cfg_alarm_overview@@UAE@XZ$10 10006843 f   cfg_alarm_overview.obj
 0001:00005851       __unwindfunclet$??1cfg_alarm_overview@@UAE@XZ$11 10006851 f   cfg_alarm_overview.obj
 0001:00005860       __ehhandler$??1cfg_alarm_overview@@UAE@XZ 10006860 f   cfg_alarm_overview.obj
 0001:0000587b       __unwindfunclet$??1config_plugin_base@@UAE@XZ$0 1000687b f   cfg_alarm_overview.obj
 0001:00005884       __unwindfunclet$??1config_plugin_base@@UAE@XZ$1 10006884 f   cfg_alarm_overview.obj
 0001:00005890       __unwindfunclet$??1config_plugin_base@@UAE@XZ$2 10006890 f   cfg_alarm_overview.obj
 0001:0000589c       __ehhandler$??1config_plugin_base@@UAE@XZ 1000689c f   cfg_alarm_overview.obj
 0001:000058b7       __unwindfunclet$?NavigatetoProcs@cfg_alarm_overview@@QAEXXZ$0 100068b7 f   cfg_alarm_overview.obj
 0001:000058b7       __unwindfunclet$?markDirty@cfg_alarm_overview@@QAEXXZ$0 100068b7 f   cfg_alarm_overview.obj
 0001:000058b7       __unwindfunclet$?NavigateProcs@cfg_alarm_overview@@QAEXXZ$0 100068b7 f   cfg_alarm_overview.obj
 0001:000058b7       __unwindfunclet$?NavigateBNCSOut@cfg_alarm_overview@@QAEXXZ$0 100068b7 f   cfg_alarm_overview.obj
 0001:000058b7       __unwindfunclet$?NavigateBNCSAcq@cfg_alarm_overview@@QAEXXZ$0 100068b7 f   cfg_alarm_overview.obj
 0001:000058b7       __unwindfunclet$?NavigateDatabaseOut@cfg_alarm_overview@@QAEXXZ$0 100068b7 f   cfg_alarm_overview.obj
 0001:000058c0       __ehhandler$?markDirty@cfg_alarm_overview@@QAEXXZ 100068c0 f   cfg_alarm_overview.obj
 0001:000058c0       __ehhandler$?NavigateBNCSAcq@cfg_alarm_overview@@QAEXXZ 100068c0 f   cfg_alarm_overview.obj
 0001:000058c0       __ehhandler$?NavigatetoProcs@cfg_alarm_overview@@QAEXXZ 100068c0 f   cfg_alarm_overview.obj
 0001:000058c0       __ehhandler$?NavigateProcs@cfg_alarm_overview@@QAEXXZ 100068c0 f   cfg_alarm_overview.obj
 0001:000058c0       __ehhandler$?NavigateBNCSOut@cfg_alarm_overview@@QAEXXZ 100068c0 f   cfg_alarm_overview.obj
 0001:000058c0       __ehhandler$?NavigateDatabaseOut@cfg_alarm_overview@@QAEXXZ 100068c0 f   cfg_alarm_overview.obj
 0001:000058db       __unwindfunclet$?NavigatetoOutput@cfg_alarm_overview@@QAEXXZ$0 100068db f   cfg_alarm_overview.obj
 0001:000058db       __unwindfunclet$?NavigatetoInput@cfg_alarm_overview@@QAEXXZ$0 100068db f   cfg_alarm_overview.obj
 0001:000058e4       __unwindfunclet$?NavigatetoOutput@cfg_alarm_overview@@QAEXXZ$1 100068e4 f   cfg_alarm_overview.obj
 0001:000058e4       __unwindfunclet$?NavigatetoInput@cfg_alarm_overview@@QAEXXZ$1 100068e4 f   cfg_alarm_overview.obj
 0001:000058ed       __unwindfunclet$?NavigatetoInput@cfg_alarm_overview@@QAEXXZ$2 100068ed f   cfg_alarm_overview.obj
 0001:000058ed       __unwindfunclet$?NavigatetoOutput@cfg_alarm_overview@@QAEXXZ$2 100068ed f   cfg_alarm_overview.obj
 0001:000058f6       __unwindfunclet$?NavigatetoInput@cfg_alarm_overview@@QAEXXZ$3 100068f6 f   cfg_alarm_overview.obj
 0001:000058f6       __unwindfunclet$?NavigatetoOutput@cfg_alarm_overview@@QAEXXZ$3 100068f6 f   cfg_alarm_overview.obj
 0001:000058ff       __unwindfunclet$?NavigatetoOutput@cfg_alarm_overview@@QAEXXZ$4 100068ff f   cfg_alarm_overview.obj
 0001:000058ff       __unwindfunclet$?NavigatetoInput@cfg_alarm_overview@@QAEXXZ$4 100068ff f   cfg_alarm_overview.obj
 0001:00005908       __unwindfunclet$?NavigatetoOutput@cfg_alarm_overview@@QAEXXZ$5 10006908 f   cfg_alarm_overview.obj
 0001:00005908       __unwindfunclet$?NavigatetoInput@cfg_alarm_overview@@QAEXXZ$5 10006908 f   cfg_alarm_overview.obj
 0001:00005911       __unwindfunclet$?NavigatetoInput@cfg_alarm_overview@@QAEXXZ$6 10006911 f   cfg_alarm_overview.obj
 0001:00005911       __unwindfunclet$?NavigatetoOutput@cfg_alarm_overview@@QAEXXZ$6 10006911 f   cfg_alarm_overview.obj
 0001:0000591a       __unwindfunclet$?NavigatetoInput@cfg_alarm_overview@@QAEXXZ$7 1000691a f   cfg_alarm_overview.obj
 0001:0000591a       __unwindfunclet$?NavigatetoOutput@cfg_alarm_overview@@QAEXXZ$7 1000691a f   cfg_alarm_overview.obj
 0001:00005923       __unwindfunclet$?NavigatetoInput@cfg_alarm_overview@@QAEXXZ$8 10006923 f   cfg_alarm_overview.obj
 0001:00005923       __unwindfunclet$?NavigatetoOutput@cfg_alarm_overview@@QAEXXZ$8 10006923 f   cfg_alarm_overview.obj
 0001:0000592c       __ehhandler$?NavigatetoInput@cfg_alarm_overview@@QAEXXZ 1000692c f   cfg_alarm_overview.obj
 0001:0000592c       __ehhandler$?NavigatetoOutput@cfg_alarm_overview@@QAEXXZ 1000692c f   cfg_alarm_overview.obj
 0001:00005947       __unwindfunclet$?about@config_plugin_base@@UAE?AVQString@@XZ$0 10006947 f   cfg_alarm_overview.obj
 0001:00005950       __unwindfunclet$?about@config_plugin_base@@UAE?AVQString@@XZ$1 10006950 f   cfg_alarm_overview.obj
 0001:0000596a       __ehhandler$?about@config_plugin_base@@UAE?AVQString@@XZ 1000696a f   cfg_alarm_overview.obj
 0001:00005985       __unwindfunclet$?activate@cfg_alarm_overview@@UAEX_N@Z$0 10006985 f   cfg_alarm_overview.obj
 0001:0000598e       __unwindfunclet$?activate@cfg_alarm_overview@@UAEX_N@Z$3 1000698e f   cfg_alarm_overview.obj
 0001:00005997       __ehhandler$?activate@cfg_alarm_overview@@UAEX_N@Z 10006997 f   cfg_alarm_overview.obj
 0001:000059b2       __unwindfunclet$?apply@cfg_alarm_overview@@UAEXXZ$0 100069b2 f   cfg_alarm_overview.obj
 0001:000059b2       __unwindfunclet$?closeEvent@cfg_alarm_overview@@UAEXPAVQCloseEvent@@@Z$0 100069b2 f   cfg_alarm_overview.obj
 0001:000059bb       __ehhandler$?apply@cfg_alarm_overview@@UAEXXZ 100069bb f   cfg_alarm_overview.obj
 0001:000059bb       __ehhandler$?closeEvent@cfg_alarm_overview@@UAEXPAVQCloseEvent@@@Z 100069bb f   cfg_alarm_overview.obj
 0001:000059d6       __unwindfunclet$?createNewDirectory@cfg_alarm_overview@@QAE_NVQString@@@Z$0 100069d6 f   cfg_alarm_overview.obj
 0001:000059df       __unwindfunclet$?createNewDirectory@cfg_alarm_overview@@QAE_NVQString@@@Z$1 100069df f   cfg_alarm_overview.obj
 0001:000059eb       __unwindfunclet$?createNewDirectory@cfg_alarm_overview@@QAE_NVQString@@@Z$2 100069eb f   cfg_alarm_overview.obj
 0001:000059f4       __unwindfunclet$?createNewDirectory@cfg_alarm_overview@@QAE_NVQString@@@Z$3 100069f4 f   cfg_alarm_overview.obj
 0001:000059fd       __unwindfunclet$?createNewDirectory@cfg_alarm_overview@@QAE_NVQString@@@Z$4 100069fd f   cfg_alarm_overview.obj
 0001:00005a06       __unwindfunclet$?createNewDirectory@cfg_alarm_overview@@QAE_NVQString@@@Z$5 10006a06 f   cfg_alarm_overview.obj
 0001:00005a0f       __unwindfunclet$?createNewDirectory@cfg_alarm_overview@@QAE_NVQString@@@Z$6 10006a0f f   cfg_alarm_overview.obj
 0001:00005a18       __unwindfunclet$?createNewDirectory@cfg_alarm_overview@@QAE_NVQString@@@Z$7 10006a18 f   cfg_alarm_overview.obj
 0001:00005a21       __unwindfunclet$?createNewDirectory@cfg_alarm_overview@@QAE_NVQString@@@Z$8 10006a21 f   cfg_alarm_overview.obj
 0001:00005a2a       __unwindfunclet$?createNewDirectory@cfg_alarm_overview@@QAE_NVQString@@@Z$9 10006a2a f   cfg_alarm_overview.obj
 0001:00005a33       __unwindfunclet$?createNewDirectory@cfg_alarm_overview@@QAE_NVQString@@@Z$10 10006a33 f   cfg_alarm_overview.obj
 0001:00005a3c       __unwindfunclet$?createNewDirectory@cfg_alarm_overview@@QAE_NVQString@@@Z$11 10006a3c f   cfg_alarm_overview.obj
 0001:00005a45       __unwindfunclet$?createNewDirectory@cfg_alarm_overview@@QAE_NVQString@@@Z$12 10006a45 f   cfg_alarm_overview.obj
 0001:00005a4e       __unwindfunclet$?createNewDirectory@cfg_alarm_overview@@QAE_NVQString@@@Z$13 10006a4e f   cfg_alarm_overview.obj
 0001:00005a57       __unwindfunclet$?createNewDirectory@cfg_alarm_overview@@QAE_NVQString@@@Z$14 10006a57 f   cfg_alarm_overview.obj
 0001:00005a60       __unwindfunclet$?createNewDirectory@cfg_alarm_overview@@QAE_NVQString@@@Z$15 10006a60 f   cfg_alarm_overview.obj
 0001:00005a69       __unwindfunclet$?createNewDirectory@cfg_alarm_overview@@QAE_NVQString@@@Z$16 10006a69 f   cfg_alarm_overview.obj
 0001:00005a72       __unwindfunclet$?createNewDirectory@cfg_alarm_overview@@QAE_NVQString@@@Z$17 10006a72 f   cfg_alarm_overview.obj
 0001:00005a7b       __unwindfunclet$?createNewDirectory@cfg_alarm_overview@@QAE_NVQString@@@Z$18 10006a7b f   cfg_alarm_overview.obj
 0001:00005a84       __unwindfunclet$?createNewDirectory@cfg_alarm_overview@@QAE_NVQString@@@Z$19 10006a84 f   cfg_alarm_overview.obj
 0001:00005a8d       __unwindfunclet$?createNewDirectory@cfg_alarm_overview@@QAE_NVQString@@@Z$20 10006a8d f   cfg_alarm_overview.obj
 0001:00005a96       __unwindfunclet$?createNewDirectory@cfg_alarm_overview@@QAE_NVQString@@@Z$21 10006a96 f   cfg_alarm_overview.obj
 0001:00005a9f       __unwindfunclet$?createNewDirectory@cfg_alarm_overview@@QAE_NVQString@@@Z$22 10006a9f f   cfg_alarm_overview.obj
 0001:00005aa8       __unwindfunclet$?createNewDirectory@cfg_alarm_overview@@QAE_NVQString@@@Z$23 10006aa8 f   cfg_alarm_overview.obj
 0001:00005ab1       __unwindfunclet$?createNewDirectory@cfg_alarm_overview@@QAE_NVQString@@@Z$24 10006ab1 f   cfg_alarm_overview.obj
 0001:00005aba       __unwindfunclet$?createNewDirectory@cfg_alarm_overview@@QAE_NVQString@@@Z$25 10006aba f   cfg_alarm_overview.obj
 0001:00005ac6       __unwindfunclet$?createNewDirectory@cfg_alarm_overview@@QAE_NVQString@@@Z$26 10006ac6 f   cfg_alarm_overview.obj
 0001:00005acf       __ehhandler$?createNewDirectory@cfg_alarm_overview@@QAE_NVQString@@@Z 10006acf f   cfg_alarm_overview.obj
 0001:00005aed       __unwindfunclet$?createNewSystem@cfg_alarm_overview@@QAEXXZ$0 10006aed f   cfg_alarm_overview.obj
 0001:00005af6       __unwindfunclet$?createNewSystem@cfg_alarm_overview@@QAEXXZ$1 10006af6 f   cfg_alarm_overview.obj
 0001:00005aff       __unwindfunclet$?createNewSystem@cfg_alarm_overview@@QAEXXZ$2 10006aff f   cfg_alarm_overview.obj
 0001:00005b08       __unwindfunclet$?createNewSystem@cfg_alarm_overview@@QAEXXZ$3 10006b08 f   cfg_alarm_overview.obj
 0001:00005b11       __unwindfunclet$?createNewSystem@cfg_alarm_overview@@QAEXXZ$4 10006b11 f   cfg_alarm_overview.obj
 0001:00005b1a       __unwindfunclet$?createNewSystem@cfg_alarm_overview@@QAEXXZ$5 10006b1a f   cfg_alarm_overview.obj
 0001:00005b23       __unwindfunclet$?createNewSystem@cfg_alarm_overview@@QAEXXZ$6 10006b23 f   cfg_alarm_overview.obj
 0001:00005b2c       __unwindfunclet$?createNewSystem@cfg_alarm_overview@@QAEXXZ$7 10006b2c f   cfg_alarm_overview.obj
 0001:00005b35       __unwindfunclet$?createNewSystem@cfg_alarm_overview@@QAEXXZ$8 10006b35 f   cfg_alarm_overview.obj
 0001:00005b3e       __unwindfunclet$?createNewSystem@cfg_alarm_overview@@QAEXXZ$9 10006b3e f   cfg_alarm_overview.obj
 0001:00005b47       __ehhandler$?createNewSystem@cfg_alarm_overview@@QAEXXZ 10006b47 f   cfg_alarm_overview.obj
 0001:00005b62       __unwindfunclet$?menus@cfg_alarm_overview@@UAE?AVQPopupMenuList@@XZ$0 10006b62 f   cfg_alarm_overview.obj
 0001:00005b7b       __ehhandler$?menus@cfg_alarm_overview@@UAE?AVQPopupMenuList@@XZ 10006b7b f   cfg_alarm_overview.obj
 0001:00005b96       __unwindfunclet$?reply@cfg_alarm_overview@@UAEXPAVresponse@@@Z$0 10006b96 f   cfg_alarm_overview.obj
 0001:00005ba2       __unwindfunclet$?reply@cfg_alarm_overview@@UAEXPAVresponse@@@Z$1 10006ba2 f   cfg_alarm_overview.obj
 0001:00005bae       __unwindfunclet$?reply@cfg_alarm_overview@@UAEXPAVresponse@@@Z$3 10006bae f   cfg_alarm_overview.obj
 0001:00005bba       __unwindfunclet$?reply@cfg_alarm_overview@@UAEXPAVresponse@@@Z$4 10006bba f   cfg_alarm_overview.obj
 0001:00005bc6       __unwindfunclet$?reply@cfg_alarm_overview@@UAEXPAVresponse@@@Z$5 10006bc6 f   cfg_alarm_overview.obj
 0001:00005bd2       __unwindfunclet$?reply@cfg_alarm_overview@@UAEXPAVresponse@@@Z$6 10006bd2 f   cfg_alarm_overview.obj
 0001:00005bde       __unwindfunclet$?reply@cfg_alarm_overview@@UAEXPAVresponse@@@Z$7 10006bde f   cfg_alarm_overview.obj
 0001:00005bea       __unwindfunclet$?reply@cfg_alarm_overview@@UAEXPAVresponse@@@Z$8 10006bea f   cfg_alarm_overview.obj
 0001:00005bf6       __unwindfunclet$?reply@cfg_alarm_overview@@UAEXPAVresponse@@@Z$9 10006bf6 f   cfg_alarm_overview.obj
 0001:00005c02       __unwindfunclet$?reply@cfg_alarm_overview@@UAEXPAVresponse@@@Z$10 10006c02 f   cfg_alarm_overview.obj
 0001:00005c0e       __unwindfunclet$?reply@cfg_alarm_overview@@UAEXPAVresponse@@@Z$11 10006c0e f   cfg_alarm_overview.obj
 0001:00005c1a       __unwindfunclet$?reply@cfg_alarm_overview@@UAEXPAVresponse@@@Z$12 10006c1a f   cfg_alarm_overview.obj
 0001:00005c26       __unwindfunclet$?reply@cfg_alarm_overview@@UAEXPAVresponse@@@Z$13 10006c26 f   cfg_alarm_overview.obj
 0001:00005c49       __unwindfunclet$?reply@cfg_alarm_overview@@UAEXPAVresponse@@@Z$14 10006c49 f   cfg_alarm_overview.obj
 0001:00005c6c       __unwindfunclet$?reply@cfg_alarm_overview@@UAEXPAVresponse@@@Z$15 10006c6c f   cfg_alarm_overview.obj
 0001:00005c78       __unwindfunclet$?reply@cfg_alarm_overview@@UAEXPAVresponse@@@Z$16 10006c78 f   cfg_alarm_overview.obj
 0001:00005c85       __unwindfunclet$?reply@cfg_alarm_overview@@UAEXPAVresponse@@@Z$17 10006c85 f   cfg_alarm_overview.obj
 0001:00005c92       __unwindfunclet$?reply@cfg_alarm_overview@@UAEXPAVresponse@@@Z$18 10006c92 f   cfg_alarm_overview.obj
 0001:00005c9e       __unwindfunclet$?reply@cfg_alarm_overview@@UAEXPAVresponse@@@Z$19 10006c9e f   cfg_alarm_overview.obj
 0001:00005caa       __unwindfunclet$?reply@cfg_alarm_overview@@UAEXPAVresponse@@@Z$20 10006caa f   cfg_alarm_overview.obj
 0001:00005cb6       __unwindfunclet$?reply@cfg_alarm_overview@@UAEXPAVresponse@@@Z$21 10006cb6 f   cfg_alarm_overview.obj
 0001:00005cc2       __unwindfunclet$?reply@cfg_alarm_overview@@UAEXPAVresponse@@@Z$22 10006cc2 f   cfg_alarm_overview.obj
 0001:00005cce       __unwindfunclet$?reply@cfg_alarm_overview@@UAEXPAVresponse@@@Z$23 10006cce f   cfg_alarm_overview.obj
 0001:00005cda       __unwindfunclet$?reply@cfg_alarm_overview@@UAEXPAVresponse@@@Z$24 10006cda f   cfg_alarm_overview.obj
 0001:00005ce6       __unwindfunclet$?reply@cfg_alarm_overview@@UAEXPAVresponse@@@Z$26 10006ce6 f   cfg_alarm_overview.obj
 0001:00005cf2       __unwindfunclet$?reply@cfg_alarm_overview@@UAEXPAVresponse@@@Z$27 10006cf2 f   cfg_alarm_overview.obj
 0001:00005cfe       __unwindfunclet$?reply@cfg_alarm_overview@@UAEXPAVresponse@@@Z$28 10006cfe f   cfg_alarm_overview.obj
 0001:00005d0a       __unwindfunclet$?reply@cfg_alarm_overview@@UAEXPAVresponse@@@Z$29 10006d0a f   cfg_alarm_overview.obj
 0001:00005d16       __unwindfunclet$?reply@cfg_alarm_overview@@UAEXPAVresponse@@@Z$30 10006d16 f   cfg_alarm_overview.obj
 0001:00005d22       __unwindfunclet$?reply@cfg_alarm_overview@@UAEXPAVresponse@@@Z$31 10006d22 f   cfg_alarm_overview.obj
 0001:00005d2e       __unwindfunclet$?reply@cfg_alarm_overview@@UAEXPAVresponse@@@Z$32 10006d2e f   cfg_alarm_overview.obj
 0001:00005d3a       __unwindfunclet$?reply@cfg_alarm_overview@@UAEXPAVresponse@@@Z$33 10006d3a f   cfg_alarm_overview.obj
 0001:00005d46       __unwindfunclet$?reply@cfg_alarm_overview@@UAEXPAVresponse@@@Z$34 10006d46 f   cfg_alarm_overview.obj
 0001:00005d69       __unwindfunclet$?reply@cfg_alarm_overview@@UAEXPAVresponse@@@Z$35 10006d69 f   cfg_alarm_overview.obj
 0001:00005d8c       __unwindfunclet$?reply@cfg_alarm_overview@@UAEXPAVresponse@@@Z$36 10006d8c f   cfg_alarm_overview.obj
 0001:00005d98       __unwindfunclet$?reply@cfg_alarm_overview@@UAEXPAVresponse@@@Z$37 10006d98 f   cfg_alarm_overview.obj
 0001:00005da5       __unwindfunclet$?reply@cfg_alarm_overview@@UAEXPAVresponse@@@Z$38 10006da5 f   cfg_alarm_overview.obj
 0001:00005db2       __unwindfunclet$?reply@cfg_alarm_overview@@UAEXPAVresponse@@@Z$39 10006db2 f   cfg_alarm_overview.obj
 0001:00005dbe       __unwindfunclet$?reply@cfg_alarm_overview@@UAEXPAVresponse@@@Z$40 10006dbe f   cfg_alarm_overview.obj
 0001:00005dca       __unwindfunclet$?reply@cfg_alarm_overview@@UAEXPAVresponse@@@Z$41 10006dca f   cfg_alarm_overview.obj
 0001:00005dd6       __unwindfunclet$?reply@cfg_alarm_overview@@UAEXPAVresponse@@@Z$42 10006dd6 f   cfg_alarm_overview.obj
 0001:00005de2       __unwindfunclet$?reply@cfg_alarm_overview@@UAEXPAVresponse@@@Z$43 10006de2 f   cfg_alarm_overview.obj
 0001:00005dee       __unwindfunclet$?reply@cfg_alarm_overview@@UAEXPAVresponse@@@Z$44 10006dee f   cfg_alarm_overview.obj
 0001:00005dfa       __unwindfunclet$?reply@cfg_alarm_overview@@UAEXPAVresponse@@@Z$45 10006dfa f   cfg_alarm_overview.obj
 0001:00005e06       __unwindfunclet$?reply@cfg_alarm_overview@@UAEXPAVresponse@@@Z$48 10006e06 f   cfg_alarm_overview.obj
 0001:00005e12       __unwindfunclet$?reply@cfg_alarm_overview@@UAEXPAVresponse@@@Z$49 10006e12 f   cfg_alarm_overview.obj
 0001:00005e1e       __unwindfunclet$?reply@cfg_alarm_overview@@UAEXPAVresponse@@@Z$50 10006e1e f   cfg_alarm_overview.obj
 0001:00005e2a       __unwindfunclet$?reply@cfg_alarm_overview@@UAEXPAVresponse@@@Z$51 10006e2a f   cfg_alarm_overview.obj
 0001:00005e36       __unwindfunclet$?reply@cfg_alarm_overview@@UAEXPAVresponse@@@Z$52 10006e36 f   cfg_alarm_overview.obj
 0001:00005e42       __unwindfunclet$?reply@cfg_alarm_overview@@UAEXPAVresponse@@@Z$53 10006e42 f   cfg_alarm_overview.obj
 0001:00005e4e       __unwindfunclet$?reply@cfg_alarm_overview@@UAEXPAVresponse@@@Z$55 10006e4e f   cfg_alarm_overview.obj
 0001:00005e5a       __unwindfunclet$?reply@cfg_alarm_overview@@UAEXPAVresponse@@@Z$57 10006e5a f   cfg_alarm_overview.obj
 0001:00005e66       __ehhandler$?reply@cfg_alarm_overview@@UAEXPAVresponse@@@Z 10006e66 f   cfg_alarm_overview.obj
 0001:00005e8e       __unwindfunclet$?selectSystem@cfg_alarm_overview@@QAEXABVQString@@@Z$0 10006e8e f   cfg_alarm_overview.obj
 0001:00005e97       __unwindfunclet$?selectSystem@cfg_alarm_overview@@QAEXABVQString@@@Z$1 10006e97 f   cfg_alarm_overview.obj
 0001:00005ea0       __unwindfunclet$?selectSystem@cfg_alarm_overview@@QAEXABVQString@@@Z$2 10006ea0 f   cfg_alarm_overview.obj
 0001:00005ea9       __unwindfunclet$?selectSystem@cfg_alarm_overview@@QAEXABVQString@@@Z$3 10006ea9 f   cfg_alarm_overview.obj
 0001:00005eb2       __unwindfunclet$?selectSystem@cfg_alarm_overview@@QAEXABVQString@@@Z$4 10006eb2 f   cfg_alarm_overview.obj
 0001:00005ebb       __unwindfunclet$?selectSystem@cfg_alarm_overview@@QAEXABVQString@@@Z$5 10006ebb f   cfg_alarm_overview.obj
 0001:00005ec4       __unwindfunclet$?selectSystem@cfg_alarm_overview@@QAEXABVQString@@@Z$6 10006ec4 f   cfg_alarm_overview.obj
 0001:00005ecd       __unwindfunclet$?selectSystem@cfg_alarm_overview@@QAEXABVQString@@@Z$7 10006ecd f   cfg_alarm_overview.obj
 0001:00005ed6       __unwindfunclet$?selectSystem@cfg_alarm_overview@@QAEXABVQString@@@Z$9 10006ed6 f   cfg_alarm_overview.obj
 0001:00005edf       __unwindfunclet$?selectSystem@cfg_alarm_overview@@QAEXABVQString@@@Z$10 10006edf f   cfg_alarm_overview.obj
 0001:00005ee8       __unwindfunclet$?selectSystem@cfg_alarm_overview@@QAEXABVQString@@@Z$11 10006ee8 f   cfg_alarm_overview.obj
 0001:00005ef1       __unwindfunclet$?selectSystem@cfg_alarm_overview@@QAEXABVQString@@@Z$12 10006ef1 f   cfg_alarm_overview.obj
 0001:00005efa       __unwindfunclet$?selectSystem@cfg_alarm_overview@@QAEXABVQString@@@Z$13 10006efa f   cfg_alarm_overview.obj
 0001:00005f03       __unwindfunclet$?selectSystem@cfg_alarm_overview@@QAEXABVQString@@@Z$14 10006f03 f   cfg_alarm_overview.obj
 0001:00005f0c       __unwindfunclet$?selectSystem@cfg_alarm_overview@@QAEXABVQString@@@Z$15 10006f0c f   cfg_alarm_overview.obj
 0001:00005f15       __unwindfunclet$?selectSystem@cfg_alarm_overview@@QAEXABVQString@@@Z$16 10006f15 f   cfg_alarm_overview.obj
 0001:00005f1e       __ehhandler$?selectSystem@cfg_alarm_overview@@QAEXABVQString@@@Z 10006f1e f   cfg_alarm_overview.obj
 0001:00005f39       __unwindfunclet$?toolbars@cfg_alarm_overview@@UAE?AVQDockWindowList@@XZ$0 10006f39 f   cfg_alarm_overview.obj
 0001:00005f52       __ehhandler$?toolbars@cfg_alarm_overview@@UAE?AVQDockWindowList@@XZ 10006f52 f   cfg_alarm_overview.obj
 0001:00005f6d       __unwindfunclet$??0COutputFile@@QAE@XZ$0 10006f6d f   OutputFile.obj
 0001:00005f6d       __unwindfunclet$??0CInputFile@@QAE@XZ$0 10006f6d f   OutputFile.obj
 0001:00005f6d       __unwindfunclet$??1COutputFile@@UAE@XZ$0 10006f6d f   OutputFile.obj
 0001:00005f6d       __unwindfunclet$??1CInputFile@@UAE@XZ$0 10006f6d f   OutputFile.obj
 0001:00005f79       __unwindfunclet$??1COutputFile@@UAE@XZ$1 10006f79 f   OutputFile.obj
 0001:00005f79       __unwindfunclet$??0CInputFile@@QAE@XZ$1 10006f79 f   OutputFile.obj
 0001:00005f79       __unwindfunclet$??0COutputFile@@QAE@XZ$1 10006f79 f   OutputFile.obj
 0001:00005f79       __unwindfunclet$??1CInputFile@@UAE@XZ$1 10006f79 f   OutputFile.obj
 0001:00005f85       __ehhandler$??1CInputFile@@UAE@XZ 10006f85 f   OutputFile.obj
 0001:00005f85       __ehhandler$??0CInputFile@@QAE@XZ 10006f85 f   OutputFile.obj
 0001:00005f85       __ehhandler$??0COutputFile@@QAE@XZ 10006f85 f   OutputFile.obj
 0001:00005f85       __ehhandler$??1COutputFile@@UAE@XZ 10006f85 f   OutputFile.obj
 0001:00005fa0       __unwindfunclet$?keys@plugindesc@@UAE?AVQStringList@@ABVQString@@0@Z$0 10006fa0 f   plugindesc.obj
 0001:00005fba       __unwindfunclet$?keys@plugindesc@@UAE?AVQStringList@@ABVQString@@0@Z$1 10006fba f   plugindesc.obj
 0001:00005fc3       __ehhandler$?keys@plugindesc@@UAE?AVQStringList@@ABVQString@@0@Z 10006fc3 f   plugindesc.obj
 0001:00005fde       __unwindfunclet$??0dialogBase@@QAE@PAVQWidget@@PBDI@Z$0 10006fde f   dialog.obj
 0001:00005fe7       __unwindfunclet$??0dialogBase@@QAE@PAVQWidget@@PBDI@Z$1 10006fe7 f   dialog.obj
 0001:00005ff6       __unwindfunclet$??0dialogBase@@QAE@PAVQWidget@@PBDI@Z$2 10006ff6 f   dialog.obj
 0001:00006000       __unwindfunclet$??0dialogBase@@QAE@PAVQWidget@@PBDI@Z$3 10007000 f   dialog.obj
 0001:0000600a       __unwindfunclet$??0dialogBase@@QAE@PAVQWidget@@PBDI@Z$4 1000700a f   dialog.obj
 0001:00006014       __unwindfunclet$??0dialogBase@@QAE@PAVQWidget@@PBDI@Z$5 10007014 f   dialog.obj
 0001:0000601e       __unwindfunclet$??0dialogBase@@QAE@PAVQWidget@@PBDI@Z$6 1000701e f   dialog.obj
 0001:00006028       __unwindfunclet$??0dialogBase@@QAE@PAVQWidget@@PBDI@Z$7 10007028 f   dialog.obj
 0001:00006032       __unwindfunclet$??0dialogBase@@QAE@PAVQWidget@@PBDI@Z$8 10007032 f   dialog.obj
 0001:0000603c       __unwindfunclet$??0dialogBase@@QAE@PAVQWidget@@PBDI@Z$9 1000703c f   dialog.obj
 0001:00006046       __unwindfunclet$??0dialogBase@@QAE@PAVQWidget@@PBDI@Z$10 10007046 f   dialog.obj
 0001:00006050       __unwindfunclet$??0dialogBase@@QAE@PAVQWidget@@PBDI@Z$11 10007050 f   dialog.obj
 0001:0000605a       __unwindfunclet$??0dialogBase@@QAE@PAVQWidget@@PBDI@Z$12 1000705a f   dialog.obj
 0001:00006064       __unwindfunclet$??0dialogBase@@QAE@PAVQWidget@@PBDI@Z$13 10007064 f   dialog.obj
 0001:0000606e       __unwindfunclet$??0dialogBase@@QAE@PAVQWidget@@PBDI@Z$14 1000706e f   dialog.obj
 0001:00006077       __unwindfunclet$??0dialogBase@@QAE@PAVQWidget@@PBDI@Z$15 10007077 f   dialog.obj
 0001:00006080       __unwindfunclet$??0dialogBase@@QAE@PAVQWidget@@PBDI@Z$16 10007080 f   dialog.obj
 0001:0000608a       __unwindfunclet$??0dialogBase@@QAE@PAVQWidget@@PBDI@Z$17 1000708a f   dialog.obj
 0001:00006094       __unwindfunclet$??0dialogBase@@QAE@PAVQWidget@@PBDI@Z$18 10007094 f   dialog.obj
 0001:0000609d       __unwindfunclet$??0dialogBase@@QAE@PAVQWidget@@PBDI@Z$19 1000709d f   dialog.obj
 0001:000060a6       __unwindfunclet$??0dialogBase@@QAE@PAVQWidget@@PBDI@Z$20 100070a6 f   dialog.obj
 0001:000060b0       __unwindfunclet$??0dialogBase@@QAE@PAVQWidget@@PBDI@Z$21 100070b0 f   dialog.obj
 0001:000060ba       __unwindfunclet$??0dialogBase@@QAE@PAVQWidget@@PBDI@Z$22 100070ba f   dialog.obj
 0001:000060c4       __unwindfunclet$??0dialogBase@@QAE@PAVQWidget@@PBDI@Z$23 100070c4 f   dialog.obj
 0001:000060ce       __unwindfunclet$??0dialogBase@@QAE@PAVQWidget@@PBDI@Z$24 100070ce f   dialog.obj
 0001:000060d8       __ehhandler$??0dialogBase@@QAE@PAVQWidget@@PBDI@Z 100070d8 f   dialog.obj
 0001:000060f3       __unwindfunclet$??1dialogBase@@UAE@XZ$0 100070f3 f   dialog.obj
 0001:000060fc       __ehhandler$??1dialogBase@@UAE@XZ 100070fc f   dialog.obj
 0001:00006117       __unwindfunclet$?languageChange@dialogBase@@MAEXXZ$0 10007117 f   dialog.obj
 0001:00006120       __unwindfunclet$?languageChange@dialogBase@@MAEXXZ$1 10007120 f   dialog.obj
 0001:00006129       __unwindfunclet$?languageChange@dialogBase@@MAEXXZ$2 10007129 f   dialog.obj
 0001:00006132       __unwindfunclet$?languageChange@dialogBase@@MAEXXZ$3 10007132 f   dialog.obj
 0001:0000613b       __unwindfunclet$?languageChange@dialogBase@@MAEXXZ$4 1000713b f   dialog.obj
 0001:00006144       __unwindfunclet$?languageChange@dialogBase@@MAEXXZ$5 10007144 f   dialog.obj
 0001:0000614d       __unwindfunclet$?languageChange@dialogBase@@MAEXXZ$6 1000714d f   dialog.obj
 0001:00006156       __unwindfunclet$?languageChange@dialogBase@@MAEXXZ$7 10007156 f   dialog.obj
 0001:0000615f       __unwindfunclet$?languageChange@dialogBase@@MAEXXZ$8 1000715f f   dialog.obj
 0001:00006168       __unwindfunclet$?languageChange@dialogBase@@MAEXXZ$9 10007168 f   dialog.obj
 0001:00006171       __unwindfunclet$?languageChange@dialogBase@@MAEXXZ$10 10007171 f   dialog.obj
 0001:0000617a       __unwindfunclet$?languageChange@dialogBase@@MAEXXZ$11 1000717a f   dialog.obj
 0001:00006183       __unwindfunclet$?languageChange@dialogBase@@MAEXXZ$12 10007183 f   dialog.obj
 0001:0000618c       __ehhandler$?languageChange@dialogBase@@MAEXXZ 1000718c f   dialog.obj
 0001:000061a7       __unwindfunclet$?command@cfg_alarm_overview@@IAEXVQString@@0@Z$0 100071a7 f   moc_cfg_alarm_overview.obj
 0001:000061b0       __unwindfunclet$?command@cfg_alarm_overview@@IAEXVQString@@0@Z$1 100071b0 f   moc_cfg_alarm_overview.obj
 0001:000061b9       __unwindfunclet$?command@cfg_alarm_overview@@IAEXVQString@@0@Z$2 100071b9 f   moc_cfg_alarm_overview.obj
 0001:000061cd       __ehhandler$?command@cfg_alarm_overview@@IAEXVQString@@0@Z 100071cd f   moc_cfg_alarm_overview.obj
 0001:000061f2       __unwindfunclet$?qt_emit@cfg_alarm_overview@@UAE_NHPAUQUObject@@@Z$0 100071f2 f   moc_cfg_alarm_overview.obj
 0001:000061fb       __ehhandler$?qt_emit@cfg_alarm_overview@@UAE_NHPAUQUObject@@@Z 100071fb f   moc_cfg_alarm_overview.obj
 0001:00006216       ??__FcleanUp_cfg_alarm_overview@@YAXXZ 10007216 f   moc_cfg_alarm_overview.obj
 0001:00006221       ??__FcleanUp_dialogBase@@YAXXZ 10007221 f   moc_dialog.obj
 0001:0000622c       ??__FcleanUp_dialog@@YAXXZ 1000722c f   moc_dialogimpl.obj
 0002:00000a58       _cleanUp_cfg_alarm_overview$initializer$ 10008a58     moc_cfg_alarm_overview.obj
 0002:00000a5c       _cleanUp_dialogBase$initializer$ 10008a5c     moc_dialog.obj
 0002:00000a60       _cleanUp_dialog$initializer$ 10008a60     moc_dialogimpl.obj
 0002:00000a6c       _pcinit                    10008a6c     MSVCRT:crtdll.obj
 0002:00000a70       _pinit                     10008a70     MSVCRT:atonexit.obj
 0002:000033a4       ?slot_0@?3??staticMetaObject@cfg_alarm_overview@@SAPAVQMetaObject@@XZ@4UQUMethod@@B 1000b3a4     moc_cfg_alarm_overview.obj
 0002:000033c4       ?slot_1@?3??staticMetaObject@cfg_alarm_overview@@SAPAVQMetaObject@@XZ@4UQUMethod@@B 1000b3c4     moc_cfg_alarm_overview.obj
 0002:000033e4       ?slot_2@?3??staticMetaObject@cfg_alarm_overview@@SAPAVQMetaObject@@XZ@4UQUMethod@@B 1000b3e4     moc_cfg_alarm_overview.obj
 0002:000033fc       ?slot_3@?3??staticMetaObject@cfg_alarm_overview@@SAPAVQMetaObject@@XZ@4UQUMethod@@B 1000b3fc     moc_cfg_alarm_overview.obj
 0002:00003418       ?slot_4@?3??staticMetaObject@cfg_alarm_overview@@SAPAVQMetaObject@@XZ@4UQUMethod@@B 1000b418     moc_cfg_alarm_overview.obj
 0002:00003438       ?slot_5@?3??staticMetaObject@cfg_alarm_overview@@SAPAVQMetaObject@@XZ@4UQUMethod@@B 1000b438     moc_cfg_alarm_overview.obj
 0002:00003454       ?slot_6@?3??staticMetaObject@cfg_alarm_overview@@SAPAVQMetaObject@@XZ@4UQUMethod@@B 1000b454     moc_cfg_alarm_overview.obj
 0002:00003478       ?slot_7@?3??staticMetaObject@cfg_alarm_overview@@SAPAVQMetaObject@@XZ@4UQUMethod@@B 1000b478     moc_cfg_alarm_overview.obj
 0002:00003494       ?slot_8@?3??staticMetaObject@cfg_alarm_overview@@SAPAVQMetaObject@@XZ@4UQUMethod@@B 1000b494     moc_cfg_alarm_overview.obj
 0002:000034b0       ?slot_9@?3??staticMetaObject@cfg_alarm_overview@@SAPAVQMetaObject@@XZ@4UQUMethod@@B 1000b4b0     moc_cfg_alarm_overview.obj
 0002:000034d0       ?slot_10@?3??staticMetaObject@cfg_alarm_overview@@SAPAVQMetaObject@@XZ@4UQUMethod@@B 1000b4d0     moc_cfg_alarm_overview.obj
 0002:000034ec       ?slot_11@?3??staticMetaObject@cfg_alarm_overview@@SAPAVQMetaObject@@XZ@4UQUMethod@@B 1000b4ec     moc_cfg_alarm_overview.obj
 0002:00003508       ?slot_12@?3??staticMetaObject@cfg_alarm_overview@@SAPAVQMetaObject@@XZ@4UQUMethod@@B 1000b508     moc_cfg_alarm_overview.obj
 0002:00003528       ?slot_tbl@?3??staticMetaObject@cfg_alarm_overview@@SAPAVQMetaObject@@XZ@4QBUQMetaData@@B 1000b528     moc_cfg_alarm_overview.obj
 0002:000036c4       ?signal_0@?3??staticMetaObject@cfg_alarm_overview@@SAPAVQMetaObject@@XZ@4UQUMethod@@B 1000b6c4     moc_cfg_alarm_overview.obj
 0002:000036d8       ?signal_tbl@?3??staticMetaObject@cfg_alarm_overview@@SAPAVQMetaObject@@XZ@4QBUQMetaData@@B 1000b6d8     moc_cfg_alarm_overview.obj
 0002:00003700       ?slot_0@?3??staticMetaObject@dialogBase@@SAPAVQMetaObject@@XZ@4UQUMethod@@B 1000b700     moc_dialog.obj
 0002:0000371c       ?slot_tbl@?3??staticMetaObject@dialogBase@@SAPAVQMetaObject@@XZ@4QBUQMetaData@@B 1000b71c     moc_dialog.obj
 0002:00003748       _GS_ExceptionPointers      1000b748     MSVCRT:gs_report.obj
 0002:000047e0       __unwindtable$??1QDockWindowList@@UAE@XZ 1000c7e0     cfg_alarm_overview.obj
 0002:000047f0       __ehfuncinfo$??1QDockWindowList@@UAE@XZ 1000c7f0     cfg_alarm_overview.obj
 0002:00004814       __unwindtable$??1?$QPtrList@VCInputFile@@@@UAE@XZ 1000c814     cfg_alarm_overview.obj
 0002:00004814       __unwindtable$??1?$QPtrList@VCOutputFile@@@@UAE@XZ 1000c814     cfg_alarm_overview.obj
 0002:00004814       __unwindtable$??1?$QPtrList@VQPopupMenu@@@@UAE@XZ 1000c814     cfg_alarm_overview.obj
 0002:0000481c       __ehfuncinfo$??1?$QPtrList@VCOutputFile@@@@UAE@XZ 1000c81c     cfg_alarm_overview.obj
 0002:0000481c       __ehfuncinfo$??1?$QPtrList@VQPopupMenu@@@@UAE@XZ 1000c81c     cfg_alarm_overview.obj
 0002:0000481c       __ehfuncinfo$??1?$QPtrList@VCInputFile@@@@UAE@XZ 1000c81c     cfg_alarm_overview.obj
 0002:00004840       __unwindtable$??1QPopupMenuList@@UAE@XZ 1000c840     cfg_alarm_overview.obj
 0002:00004848       __ehfuncinfo$??1QPopupMenuList@@UAE@XZ 1000c848     cfg_alarm_overview.obj
 0002:0000486c       __unwindtable$??0config_plugin_base@@QAE@ABVQString@@00@Z 1000c86c     cfg_alarm_overview.obj
 0002:0000488c       __ehfuncinfo$??0config_plugin_base@@QAE@ABVQString@@00@Z 1000c88c     cfg_alarm_overview.obj
 0002:000048b0       __unwindtable$??1config_plugin_base@@UAE@XZ 1000c8b0     cfg_alarm_overview.obj
 0002:000048c8       __ehfuncinfo$??1config_plugin_base@@UAE@XZ 1000c8c8     cfg_alarm_overview.obj
 0002:000048ec       __unwindtable$?about@config_plugin_base@@UAE?AVQString@@XZ 1000c8ec     cfg_alarm_overview.obj
 0002:000048fc       __ehfuncinfo$?about@config_plugin_base@@UAE?AVQString@@XZ 1000c8fc     cfg_alarm_overview.obj
 0002:00004920       __ehfuncinfo$??0cfg_alarm_overview@@QAE@ABVQString@@00@Z 1000c920     cfg_alarm_overview.obj
 0002:00004944       __unwindtable$??0cfg_alarm_overview@@QAE@ABVQString@@00@Z 1000c944     cfg_alarm_overview.obj
 0002:00004a54       __ehfuncinfo$??1cfg_alarm_overview@@UAE@XZ 1000ca54     cfg_alarm_overview.obj
 0002:00004a78       __unwindtable$??1cfg_alarm_overview@@UAE@XZ 1000ca78     cfg_alarm_overview.obj
 0002:00004ad8       __unwindtable$?toolbars@cfg_alarm_overview@@UAE?AVQDockWindowList@@XZ 1000cad8     cfg_alarm_overview.obj
 0002:00004ae0       __ehfuncinfo$?toolbars@cfg_alarm_overview@@UAE?AVQDockWindowList@@XZ 1000cae0     cfg_alarm_overview.obj
 0002:00004b04       __unwindtable$?menus@cfg_alarm_overview@@UAE?AVQPopupMenuList@@XZ 1000cb04     cfg_alarm_overview.obj
 0002:00004b0c       __ehfuncinfo$?menus@cfg_alarm_overview@@UAE?AVQPopupMenuList@@XZ 1000cb0c     cfg_alarm_overview.obj
 0002:00004b30       __ehfuncinfo$?reply@cfg_alarm_overview@@UAEXPAVresponse@@@Z 1000cb30     cfg_alarm_overview.obj
 0002:00004b54       __unwindtable$?reply@cfg_alarm_overview@@UAEXPAVresponse@@@Z 1000cb54     cfg_alarm_overview.obj
 0002:00004cfc       __unwindtable$?activate@cfg_alarm_overview@@UAEX_N@Z 1000ccfc     cfg_alarm_overview.obj
 0002:00004d0c       __ehfuncinfo$?activate@cfg_alarm_overview@@UAEX_N@Z 1000cd0c     cfg_alarm_overview.obj
 0002:00004d30       __unwindtable$?closeEvent@cfg_alarm_overview@@UAEXPAVQCloseEvent@@@Z 1000cd30     cfg_alarm_overview.obj
 0002:00004d30       __unwindtable$?apply@cfg_alarm_overview@@UAEXXZ 1000cd30     cfg_alarm_overview.obj
 0002:00004d38       __ehfuncinfo$?closeEvent@cfg_alarm_overview@@UAEXPAVQCloseEvent@@@Z 1000cd38     cfg_alarm_overview.obj
 0002:00004d38       __ehfuncinfo$?apply@cfg_alarm_overview@@UAEXXZ 1000cd38     cfg_alarm_overview.obj
 0002:00004d5c       __ehfuncinfo$?createNewDirectory@cfg_alarm_overview@@QAE_NVQString@@@Z 1000cd5c     cfg_alarm_overview.obj
 0002:00004d80       __unwindtable$?createNewDirectory@cfg_alarm_overview@@QAE_NVQString@@@Z 1000cd80     cfg_alarm_overview.obj
 0002:00004e70       __ehfuncinfo$?createNewSystem@cfg_alarm_overview@@QAEXXZ 1000ce70     cfg_alarm_overview.obj
 0002:00004e94       __unwindtable$?createNewSystem@cfg_alarm_overview@@QAEXXZ 1000ce94     cfg_alarm_overview.obj
 0002:00004ef4       __ehfuncinfo$?NavigatetoOutput@cfg_alarm_overview@@QAEXXZ 1000cef4     cfg_alarm_overview.obj
 0002:00004ef4       __ehfuncinfo$?NavigatetoInput@cfg_alarm_overview@@QAEXXZ 1000cef4     cfg_alarm_overview.obj
 0002:00004f18       __unwindtable$?NavigatetoOutput@cfg_alarm_overview@@QAEXXZ 1000cf18     cfg_alarm_overview.obj
 0002:00004f18       __unwindtable$?NavigatetoInput@cfg_alarm_overview@@QAEXXZ 1000cf18     cfg_alarm_overview.obj
 0002:00004f60       __ehfuncinfo$?selectSystem@cfg_alarm_overview@@QAEXABVQString@@@Z 1000cf60     cfg_alarm_overview.obj
 0002:00004f84       __unwindtable$?selectSystem@cfg_alarm_overview@@QAEXABVQString@@@Z 1000cf84     cfg_alarm_overview.obj
 0002:00005004       __unwindtable$?NavigateProcs@cfg_alarm_overview@@QAEXXZ 1000d004     cfg_alarm_overview.obj
 0002:00005004       __unwindtable$?NavigateDatabaseOut@cfg_alarm_overview@@QAEXXZ 1000d004     cfg_alarm_overview.obj
 0002:00005004       __unwindtable$?NavigateBNCSAcq@cfg_alarm_overview@@QAEXXZ 1000d004     cfg_alarm_overview.obj
 0002:00005004       __unwindtable$?markDirty@cfg_alarm_overview@@QAEXXZ 1000d004     cfg_alarm_overview.obj
 0002:00005004       __unwindtable$?NavigateBNCSOut@cfg_alarm_overview@@QAEXXZ 1000d004     cfg_alarm_overview.obj
 0002:00005004       __unwindtable$?NavigatetoProcs@cfg_alarm_overview@@QAEXXZ 1000d004     cfg_alarm_overview.obj
 0002:0000500c       __ehfuncinfo$?NavigateProcs@cfg_alarm_overview@@QAEXXZ 1000d00c     cfg_alarm_overview.obj
 0002:0000500c       __ehfuncinfo$?markDirty@cfg_alarm_overview@@QAEXXZ 1000d00c     cfg_alarm_overview.obj
 0002:0000500c       __ehfuncinfo$?NavigateDatabaseOut@cfg_alarm_overview@@QAEXXZ 1000d00c     cfg_alarm_overview.obj
 0002:0000500c       __ehfuncinfo$?NavigateBNCSOut@cfg_alarm_overview@@QAEXXZ 1000d00c     cfg_alarm_overview.obj
 0002:0000500c       __ehfuncinfo$?NavigateBNCSAcq@cfg_alarm_overview@@QAEXXZ 1000d00c     cfg_alarm_overview.obj
 0002:0000500c       __ehfuncinfo$?NavigatetoProcs@cfg_alarm_overview@@QAEXXZ 1000d00c     cfg_alarm_overview.obj
 0002:00005030       __unwindtable$??4?$QGuardedPtr@VQPopupMenu@@@@QAEAAV0@PAVQPopupMenu@@@Z 1000d030     cfg_alarm_overview.obj
 0002:00005030       __unwindtable$??0?$QGuardedPtr@VQDockWindow@@@@QAE@XZ 1000d030     cfg_alarm_overview.obj
 0002:00005030       __unwindtable$??4?$QGuardedPtr@VQDockWindow@@@@QAEAAV0@PAVQDockWindow@@@Z 1000d030     cfg_alarm_overview.obj
 0002:00005030       __unwindtable$?create@plugindesc@@UAEPAVconfig_plugin_base@@ABVQString@@00@Z 1000d030     cfg_alarm_overview.obj
 0002:00005030       __unwindtable$??0?$QGuardedPtr@VQPopupMenu@@@@QAE@XZ 1000d030     cfg_alarm_overview.obj
 0002:00005038       __ehfuncinfo$??4?$QGuardedPtr@VQPopupMenu@@@@QAEAAV0@PAVQPopupMenu@@@Z 1000d038     cfg_alarm_overview.obj
 0002:00005038       __ehfuncinfo$??0?$QGuardedPtr@VQDockWindow@@@@QAE@XZ 1000d038     cfg_alarm_overview.obj
 0002:00005038       __ehfuncinfo$??4?$QGuardedPtr@VQDockWindow@@@@QAEAAV0@PAVQDockWindow@@@Z 1000d038     cfg_alarm_overview.obj
 0002:00005038       __ehfuncinfo$?create@plugindesc@@UAEPAVconfig_plugin_base@@ABVQString@@00@Z 1000d038     cfg_alarm_overview.obj
 0002:00005038       __ehfuncinfo$??0?$QGuardedPtr@VQPopupMenu@@@@QAE@XZ 1000d038     cfg_alarm_overview.obj
 0002:0000505c       __unwindtable$??1?$QDict@VQAction@@@@UAE@XZ 1000d05c     cfg_alarm_overview.obj
 0002:00005064       __ehfuncinfo$??1?$QDict@VQAction@@@@UAE@XZ 1000d064     cfg_alarm_overview.obj
 0002:00005088       __unwindtable$??1CInputFile@@UAE@XZ 1000d088     OutputFile.obj
 0002:00005088       __unwindtable$??0CInputFile@@QAE@XZ 1000d088     OutputFile.obj
 0002:00005088       __unwindtable$??1COutputFile@@UAE@XZ 1000d088     OutputFile.obj
 0002:00005088       __unwindtable$??0COutputFile@@QAE@XZ 1000d088     OutputFile.obj
 0002:00005098       __ehfuncinfo$??0COutputFile@@QAE@XZ 1000d098     OutputFile.obj
 0002:00005098       __ehfuncinfo$??1COutputFile@@UAE@XZ 1000d098     OutputFile.obj
 0002:00005098       __ehfuncinfo$??0CInputFile@@QAE@XZ 1000d098     OutputFile.obj
 0002:00005098       __ehfuncinfo$??1CInputFile@@UAE@XZ 1000d098     OutputFile.obj
 0002:000050bc       __unwindtable$?keys@plugindesc@@UAE?AVQStringList@@ABVQString@@0@Z 1000d0bc     plugindesc.obj
 0002:000050cc       __ehfuncinfo$?keys@plugindesc@@UAE?AVQStringList@@ABVQString@@0@Z 1000d0cc     plugindesc.obj
 0002:000050f0       __ehfuncinfo$??0dialogBase@@QAE@PAVQWidget@@PBDI@Z 1000d0f0     dialog.obj
 0002:00005114       __unwindtable$??0dialogBase@@QAE@PAVQWidget@@PBDI@Z 1000d114     dialog.obj
 0002:000051dc       __unwindtable$??1dialogBase@@UAE@XZ 1000d1dc     dialog.obj
 0002:000051e4       __ehfuncinfo$??1dialogBase@@UAE@XZ 1000d1e4     dialog.obj
 0002:00005208       __ehfuncinfo$?languageChange@dialogBase@@MAEXXZ 1000d208     dialog.obj
 0002:0000522c       __unwindtable$?languageChange@dialogBase@@MAEXXZ 1000d22c     dialog.obj
 0002:00005294       __unwindtable$?qt_emit@cfg_alarm_overview@@UAE_NHPAUQUObject@@@Z 1000d294     moc_cfg_alarm_overview.obj
 0002:0000529c       __ehfuncinfo$?qt_emit@cfg_alarm_overview@@UAE_NHPAUQUObject@@@Z 1000d29c     moc_cfg_alarm_overview.obj
 0002:000052c0       __unwindtable$?command@cfg_alarm_overview@@IAEXVQString@@0@Z 1000d2c0     moc_cfg_alarm_overview.obj
 0002:000052d8       __ehfuncinfo$?command@cfg_alarm_overview@@IAEXVQString@@0@Z 1000d2d8     moc_cfg_alarm_overview.obj
 0002:00005300       __sehtable$??_L@YGXPAXIHP6EX0@Z1@Z 1000d300     MSVCRT:ehvecctr.obj
 0002:00005320       __sehtable$??_M@YGXPAXIHP6EX0@Z@Z 1000d320     MSVCRT:ehvecdtr.obj
 0002:00005340       __sehtable$?__ArrayUnwind@@YGXPAXIHP6EX0@Z@Z 1000d340     MSVCRT:ehvecdtr.obj
 0002:00005360       __sehtable$__onexit        1000d360     MSVCRT:atonexit.obj
 0002:00005380       __sehtable$___DllMainCRTStartup 1000d380     MSVCRT:crtdll.obj
 0002:000053a8       __sehtable$__IsNonwritableInCurrentImage 1000d3a8     MSVCRT:pesect.obj
 0002:000053d0       .edata                     1000d3d0     config_alm_overview.exp
 0002:000053f8       rgpv                       1000d3f8     config_alm_overview.exp
 0002:000053fc       rgszName                   1000d3fc     config_alm_overview.exp
 0002:00005400       rgwOrd                     1000d400     config_alm_overview.exp
 0002:00005402       szName                     1000d402     config_alm_overview.exp
 0002:0000541a       $N00001                    1000d41a     config_alm_overview.exp
 0002:0000c4fc       .idata$6                   100144fc     qt-mt323:qt-mt323.dll
 0002:0000c52a       .idata$6                   1001452a     config_icons:config_icons.dll
 0002:0000c714       .idata$6                   10014714     alm_sys_select:alm_sys_select.dll
 0002:0000c744       .idata$6                   10014744     kernel32:KERNEL32.dll
 0002:0000c794       .idata$6                   10014794     MSVCRT:MSVCR120.dll
 0003:00000000       _filesave                  10015000     cfg_alarm_overview.obj
 0003:00000050       _copy                      10015050     cfg_alarm_overview.obj
 0003:000000a8       _paste                     100150a8     cfg_alarm_overview.obj
 0003:00000110       _undo                      10015110     cfg_alarm_overview.obj
 0003:00000160       _bell                      10015160     plugindesc.obj
 0003:000001b0       ?param_slot_7@?3??staticMetaObject@cfg_alarm_overview@@SAPAVQMetaObject@@XZ@4QBUQUParameter@@B 100151b0     moc_cfg_alarm_overview.obj
 0003:0000072c       _cleanUp_cfg_alarm_overview 1001572c     moc_cfg_alarm_overview.obj
 0003:00000730       ?param_slot_1@?3??staticMetaObject@cfg_alarm_overview@@SAPAVQMetaObject@@XZ@4QBUQUParameter@@B 10015730     moc_cfg_alarm_overview.obj
 0003:00000750       ?$S1@?3??staticMetaObject@cfg_alarm_overview@@SAPAVQMetaObject@@XZ@4IA 10015750     moc_cfg_alarm_overview.obj
 0003:00000754       ?param_signal_0@?3??staticMetaObject@cfg_alarm_overview@@SAPAVQMetaObject@@XZ@4QBUQUParameter@@B 10015754     moc_cfg_alarm_overview.obj
 0003:00000778       _cleanUp_dialogBase        10015778     moc_dialog.obj
 0003:00000780       _cleanUp_dialog            10015780     moc_dialogimpl.obj
 0003:00000784       ___proc_attached           10015784     MSVCRT:crtdll.obj
 0003:00000788       _GS_ExceptionRecord        10015788     MSVCRT:gs_report.obj
 0003:000007d8       _GS_ContextRecord          100157d8     MSVCRT:gs_report.obj
 0003:00000aa4       _DebuggerWasPresent        10015aa4     MSVCRT:gs_report.obj
 0004:000000a0       $R000000                   100160a0     version.res
 0004:00000558       $R0004B8                   10016558     version.res
